Component: ARM Compiler 5.06 update 6 (build 750) Tool: armlink [4d35ed]

==============================================================================

Section Cross References

    main.o(i.Button_state) refers to nrf_log_frontend.o(i.nrf_log_frontend_std_0) for nrf_log_frontend_std_0
    main.o(i.Button_state) refers to main.o(i.nrf_gpio_pin_toggle) for nrf_gpio_pin_toggle
    main.o(i.Button_state) refers to nrf_log_frontend.o(i.nrf_log_frontend_std_1) for nrf_log_frontend_std_1
    main.o(i.Button_state) refers to main.o(.data) for .data
    main.o(i.Button_state) refers to nrf_log_frontend.o(log_const_data) for m_nrf_log_app_logs_data_const
    main.o(i.NRF_GetTick) refers to main.o(.data) for .data
    main.o(i.SysTick_Handler) refers to main.o(.data) for .data
    main.o(i.TIMER2_IRQHandler) refers to main.o(i.saadc_start) for saadc_start
    main.o(i.TIMER2_IRQHandler) refers to printf1.o(i.__0sprintf$1) for __2sprintf
    main.o(i.TIMER2_IRQHandler) refers to strlen.o(.text) for strlen
    main.o(i.TIMER2_IRQHandler) refers to main.o(.data) for .data
    main.o(i.TIMER2_IRQHandler) refers to main.o(.bss) for .bss
    main.o(i.ble_evt_handler) refers to nrf_log_frontend.o(i.nrf_log_frontend_std_0) for nrf_log_frontend_std_0
    main.o(i.ble_evt_handler) refers to bsp.o(i.bsp_indication_set) for bsp_indication_set
    main.o(i.ble_evt_handler) refers to app_error.o(i.app_error_handler_bare) for app_error_handler_bare
    main.o(i.ble_evt_handler) refers to nrf_ble_qwr.o(i.nrf_ble_qwr_conn_handle_assign) for nrf_ble_qwr_conn_handle_assign
    main.o(i.ble_evt_handler) refers to main.o(.data) for .data
    main.o(i.ble_evt_handler) refers to nrf_log_frontend.o(log_const_data) for m_nrf_log_app_logs_data_const
==============================================================================

Removing Unused input sections from the image.

    Removing main.o(.rev16_text), (4 bytes).
    Removing main.o(.revsh_text), (4 bytes).
    Removing main.o(.rrx_text), (6 bytes).
    Removing main.o(i.NRF_GetTick), (12 bytes).
    Removing main.o(i.gatt_evt_handler), (92 bytes).
    Removing main.o(.bss), (40 bytes).
    Removing main.o(.constdata), (4 bytes).
    Removing main.o(.data), (6 bytes).
    Removing main.o(.data), (6 bytes).
    Removing main.o(.data), (2 bytes).
    Removing main.o(.data), (2 bytes).
    Removing boards.o(.rev16_text), (4 bytes).
    Removing boards.o(.revsh_text), (4 bytes).
    Removing boards.o(.rrx_text), (6 bytes).
    Removing boards.o(i.bsp_board_button_state_get), (32 bytes).
    Removing boards.o(i.bsp_board_init), (84 bytes).
    Removing boards.o(i.bsp_board_led_idx_to_pin), (12 bytes).
    Removing boards.o(i.bsp_board_pin_to_led_idx), (36 bytes).
==============================================================================

Image Symbol Table

    Local Symbols

    Symbol Name                              Value     Ov Type        Size  Object(Section)

    ../clib/../cmprslib/zerorunl2.c          0x00000000   Number         0  __dczerorl2.o ABSOLUTE
    ../clib/microlib/ctype/ctype.c           0x00000000   Number         0  iscntrl_o.o ABSOLUTE
    ../clib/microlib/ctype/ctype.c           0x00000000   Number         0  isupper_o.o ABSOLUTE
    ../clib/microlib/ctype/ctype.c           0x00000000   Number         0  isxdigit_o.o ABSOLUTE
    ../clib/microlib/ctype/ctype.c           0x00000000   Number         0  isgraph_o.o ABSOLUTE
    ../clib/microlib/ctype/ctype.c           0x00000000   Number         0  isdigit_o.o ABSOLUTE
    ../clib/microlib/ctype/ctype.c           0x00000000   Number         0  isprint_o.o ABSOLUTE
    ../clib/microlib/ctype/ctype.c           0x00000000   Number         0  isblank_o.o ABSOLUTE
    ../clib/microlib/ctype/ctype.c           0x00000000   Number         0  isalpha_o.o ABSOLUTE
    ../clib/microlib/ctype/ctype.c           0x00000000   Number         0  isalnum_o.o ABSOLUTE
    ../clib/microlib/ctype/ctype.c           0x00000000   Number         0  ctype_o.o ABSOLUTE
    ../clib/microlib/ctype/ctype.c           0x00000000   Number         0  islower_o.o ABSOLUTE
    ../clib/microlib/ctype/ctype.c           0x00000000   Number         0  ispunct_o.o ABSOLUTE
    ../clib/microlib/ctype/ctype.c           0x00000000   Number         0  isspace_o.o ABSOLUTE
    ../clib/microlib/division.c              0x00000000   Number         0  uidiv.o ABSOLUTE
    ../clib/microlib/division.c              0x00000000   Number         0  uldiv.o ABSOLUTE
    ../clib/microlib/init/entry.s            0x00000000   Number         0  entry2.o ABSOLUTE
    ../clib/microlib/init/entry.s            0x00000000   Number         0  entry10b.o ABSOLUTE
    ../clib/microlib/init/entry.s            0x00000000   Number         0  entry11a.o ABSOLUTE
    ../clib/microlib/init/entry.s            0x00000000   Number         0  entry9a.o ABSOLUTE
    ../clib/microlib/init/entry.s            0x00000000   Number         0  entry7a.o ABSOLUTE
    ../clib/microlib/init/entry.s            0x00000000   Number         0  entry11b.o ABSOLUTE
    ../clib/microlib/init/entry.s            0x00000000   Number         0  entry9b.o ABSOLUTE
    ../clib/microlib/init/entry.s            0x00000000   Number         0  entry8b.o ABSOLUTE
    ../clib/microlib/init/entry.s            0x00000000   Number         0  entry8a.o ABSOLUTE
    ../clib/microlib/init/entry.s            0x00000000   Number         0  entry10a.o ABSOLUTE
    ../clib/microlib/init/entry.s            0x00000000   Number         0  entry.o ABSOLUTE
    ../clib/microlib/init/entry.s            0x00000000   Number         0  entry7b.o ABSOLUTE
    ../clib/microlib/init/entry.s            0x00000000   Number         0  entry5.o ABSOLUTE
    ../clib/microlib/longlong.c              0x00000000   Number         0  llushr.o ABSOLUTE
    ../clib/microlib/longlong.c              0x00000000   Number         0  llshl.o ABSOLUTE
    ../clib/microlib/longlong.c              0x00000000   Number         0  llsshr.o ABSOLUTE
    ../clib/microlib/printf/printf.c         0x00000000   Number         0  printf6.o ABSOLUTE
    ../clib/microlib/printf/printf.c         0x00000000   Number         0  printf2.o ABSOLUTE
    ../clib/microlib/printf/printf.c         0x00000000   Number         0  printf8.o ABSOLUTE
    ../clib/microlib/printf/printf.c         0x00000000   Number         0  printf7.o ABSOLUTE
    ../clib/microlib/printf/printf.c         0x00000000   Number         0  printfa.o ABSOLUTE
    ../clib/microlib/printf/printf.c         0x00000000   Number         0  printf4.o ABSOLUTE
    ../clib/microlib/printf/printf.c         0x00000000   Number         0  printfb.o ABSOLUTE
    ../clib/microlib/printf/printf.c         0x00000000   Number         0  printf3.o ABSOLUTE
    ../clib/microlib/printf/printf.c         0x00000000   Number         0  printf0.o ABSOLUTE
    ../clib/microlib/printf/printf.c         0x00000000   Number         0  printf5.o ABSOLUTE
    ../clib/microlib/printf/printf.c         0x00000000   Number         0  printf1.o ABSOLUTE
    ../clib/microlib/printf/stubs.s          0x00000000   Number         0  stubs.o ABSOLUTE
    ../clib/microlib/string/memcmp.c         0x00000000   Number         0  memcmp.o ABSOLUTE
    ../clib/microlib/string/memcpy.c         0x00000000   Number         0  memcpyb.o ABSOLUTE
    ../clib/microlib/string/memcpy.c         0x00000000   Number         0  memcpya.o ABSOLUTE
    ../clib/microlib/string/memset.c         0x00000000   Number         0  memseta.o ABSOLUTE
    ../clib/microlib/string/strcpy.c         0x00000000   Number         0  strcpy.o ABSOLUTE
    ../clib/microlib/string/strlen.c         0x00000000   Number         0  strlen.o ABSOLUTE
    ../clib/microlib/stubs.s                 0x00000000   Number         0  iusefp.o ABSOLUTE
    ../fplib/microlib/fpadd.c                0x00000000   Number         0  dadd.o ABSOLUTE
    ../fplib/microlib/fpdiv.c                0x00000000   Number         0  ddiv.o ABSOLUTE
    ../fplib/microlib/fpepilogue.c           0x00000000   Number         0  depilogue.o ABSOLUTE
    ../fplib/microlib/fpfix.c                0x00000000   Number         0  dfixul.o ABSOLUTE
    ../fplib/microlib/fpmul.c                0x00000000   Number         0  dmul.o ABSOLUTE
    ..\..\..\..\..\..\components\ble\ble_advertising\ble_advertising.c 0x00000000   Number         0  ble_advertising.o ABSOLUTE
    ..\..\..\..\..\..\components\ble\ble_link_ctx_manager\ble_link_ctx_manager.c 0x00000000   Number         0  ble_link_ctx_manager.o ABSOLUTE
    ..\..\..\..\..\..\components\ble\ble_services\ble_nus\ble_nus.c 0x00000000   Number         0  ble_nus.o ABSOLUTE
    ..\..\..\..\..\..\components\ble\common\ble_advdata.c 0x00000000   Number         0  ble_advdata.o ABSOLUTE
    ..\..\..\..\..\..\components\ble\common\ble_conn_params.c 0x00000000   Number         0  ble_conn_params.o ABSOLUTE
    ..\..\..\..\..\..\components\ble\common\ble_conn_state.c 0x00000000   Number         0  ble_conn_state.o ABSOLUTE
    ..\..\..\..\..\..\components\ble\common\ble_srv_common.c 0x00000000   Number         0  ble_srv_common.o ABSOLUTE
    ..\..\..\..\..\..\components\ble\nrf_ble_gatt\nrf_ble_gatt.c 0x00000000   Number         0  nrf_ble_gatt.o ABSOLUTE
    ..\..\..\..\..\..\components\ble\nrf_ble_qwr\nrf_ble_qwr.c 0x00000000   Number         0  nrf_ble_qwr.o ABSOLUTE
    ..\..\..\..\..\..\components\boards\boards.c 0x00000000   Number         0  boards.o ABSOLUTE
    ..\..\..\..\..\..\components\libraries\atomic\nrf_atomic.c 0x00000000   Number         0  nrf_atomic.o ABSOLUTE
    ..\..\..\..\..\..\components\libraries\atomic_fifo\nrf_atfifo.c 0x00000000   Number         0  nrf_atfifo.o ABSOLUTE
    ..\..\..\..\..\..\components\libraries\atomic_flags\nrf_atflags.c 0x00000000   Number         0  nrf_atflags.o ABSOLUTE
    ..\..\..\..\..\..\components\libraries\balloc\nrf_balloc.c 0x00000000   Number         0  nrf_balloc.o ABSOLUTE
    ..\..\..\..\..\..\components\libraries\block_dev\sdc\nrf_block_dev_sdc.c 0x00000000   Number         0  nrf_block_dev_sdc.o ABSOLUTE
    ..\..\..\..\..\..\components\libraries\bsp\bsp.c 0x00000000   Number         0  bsp.o ABSOLUTE
    ..\..\..\..\..\..\components\libraries\bsp\bsp_btn_ble.c 0x00000000   Number         0  bsp_btn_ble.o ABSOLUTE
    ..\..\..\..\..\..\components\libraries\button\app_button.c 0x00000000   Number         0  app_button.o ABSOLUTE
    ..\..\..\..\..\..\components\libraries\experimental_section_vars\nrf_section_iter.c 0x00000000   Number         0  nrf_section_iter.o ABSOLUTE
    ..\..\..\..\..\..\components\libraries\fifo\app_fifo.c 0x00000000   Number         0  app_fifo.o ABSOLUTE
    ..\..\..\..\..\..\components\libraries\hardfault\hardfault_implementation.c 0x00000000   Number         0  hardfault_implementation.o ABSOLUTE
    ..\..\..\..\..\..\components\libraries\log\src\nrf_log_backend_rtt.c 0x00000000   Number         0  nrf_log_backend_rtt.o ABSOLUTE
    ..\..\..\..\..\..\components\libraries\log\src\nrf_log_backend_serial.c 0x00000000   Number         0  nrf_log_backend_serial.o ABSOLUTE
    ..\..\..\..\..\..\components\libraries\log\src\nrf_log_backend_uart.c 0x00000000   Number         0  nrf_log_backend_uart.o ABSOLUTE
    ..\..\..\..\..\..\components\libraries\log\src\nrf_log_default_backends.c 0x00000000   Number         0  nrf_log_default_backends.o ABSOLUTE
    ..\..\..\..\..\..\components\libraries\log\src\nrf_log_frontend.c 0x00000000   Number         0  nrf_log_frontend.o ABSOLUTE
    ..\..\..\..\..\..\components\libraries\log\src\nrf_log_str_formatter.c 0x00000000   Number         0  nrf_log_str_formatter.o ABSOLUTE
    ..\..\..\..\..\..\components\libraries\memobj\nrf_memobj.c 0x00000000   Number         0  nrf_memobj.o ABSOLUTE
    ..\..\..\..\..\..\components\libraries\pwr_mgmt\nrf_pwr_mgmt.c 0x00000000   Number         0  nrf_pwr_mgmt.o ABSOLUTE
    ..\..\..\..\..\..\components\libraries\ringbuf\nrf_ringbuf.c 0x00000000   Number         0  nrf_ringbuf.o ABSOLUTE
    ..\..\..\..\..\..\components\libraries\scheduler\app_scheduler.c 0x00000000   Number         0  app_scheduler.o ABSOLUTE
    ..\..\..\..\..\..\components\libraries\sdcard\app_sdcard.c 0x00000000   Number         0  app_sdcard.o ABSOLUTE
    ..\..\..\..\..\..\components\libraries\sortlist\nrf_sortlist.c 0x00000000   Number         0  nrf_sortlist.o ABSOLUTE
    ..\..\..\..\..\..\components\libraries\strerror\nrf_strerror.c 0x00000000   Number         0  nrf_strerror.o ABSOLUTE
    ..\..\..\..\..\..\components\libraries\timer\app_timer2.c 0x00000000   Number         0  app_timer2.o ABSOLUTE
    ..\..\..\..\..\..\components\libraries\timer\drv_rtc.c 0x00000000   Number         0  drv_rtc.o ABSOLUTE
    ..\..\..\..\..\..\components\libraries\uart\app_uart_fifo.c 0x00000000   Number         0  app_uart_fifo.o ABSOLUTE
    ..\..\..\..\..\..\components\libraries\uart\retarget.c 0x00000000   Number         0  retarget.o ABSOLUTE
    ..\..\..\..\..\..\components\libraries\util\app_error.c 0x00000000   Number         0  app_error.o ABSOLUTE
    ..\..\..\..\..\..\components\libraries\util\app_error_handler_keil.c 0x00000000   Number         0  app_error_handler_keil.o ABSOLUTE
    ..\..\..\..\..\..\components\libraries\util\app_error_weak.c 0x00000000   Number         0  app_error_weak.o ABSOLUTE
    ..\..\..\..\..\..\components\libraries\util\app_util_platform.c 0x00000000   Number         0  app_util_platform.o ABSOLUTE
    ..\..\..\..\..\..\components\libraries\util\nrf_assert.c 0x00000000   Number         0  nrf_assert.o ABSOLUTE
    ..\..\..\..\..\..\components\softdevice\common\nrf_sdh.c 0x00000000   Number         0  nrf_sdh.o ABSOLUTE
    ..\..\..\..\..\..\components\softdevice\common\nrf_sdh_ble.c 0x00000000   Number         0  nrf_sdh_ble.o ABSOLUTE
    ..\..\..\..\..\..\components\softdevice\common\nrf_sdh_soc.c 0x00000000   Number         0  nrf_sdh_soc.o ABSOLUTE
    ..\..\..\..\..\..\external\fatfs\port\diskio_blkdev.c 0x00000000   Number         0  diskio_blkdev.o ABSOLUTE
    ..\..\..\..\..\..\external\fatfs\src\ff.c 0x00000000   Number         0  ff.o ABSOLUTE
    ..\..\..\..\..\..\external\fprintf\nrf_fprintf.c 0x00000000   Number         0  nrf_fprintf.o ABSOLUTE
    ..\..\..\..\..\..\external\fprintf\nrf_fprintf_format.c 0x00000000   Number         0  nrf_fprintf_format.o ABSOLUTE
    ..\..\..\..\..\..\external\segger_rtt\SEGGER_RTT.c 0x00000000   Number         0  segger_rtt.o ABSOLUTE
    ..\..\..\..\..\..\external\segger_rtt\SEGGER_RTT_Syscalls_KEIL.c 0x00000000   Number         0  segger_rtt_syscalls_keil.o ABSOLUTE
    ..\..\..\..\..\..\external\segger_rtt\SEGGER_RTT_printf.c 0x00000000   Number         0  segger_rtt_printf.o ABSOLUTE
    ..\..\..\..\..\..\external\utf_converter\utf.c 0x00000000   Number         0  utf.o ABSOLUTE
    ..\..\..\..\..\..\integration\nrfx\legacy\nrf_drv_clock.c 0x00000000   Number         0  nrf_drv_clock.o ABSOLUTE
    ..\..\..\..\..\..\integration\nrfx\legacy\nrf_drv_spi.c 0x00000000   Number         0  nrf_drv_spi.o ABSOLUTE
    ..\..\..\..\..\..\integration\nrfx\legacy\nrf_drv_uart.c 0x00000000   Number         0  nrf_drv_uart.o ABSOLUTE
    ..\..\..\..\..\..\modules\nrfx\drivers\src\nrfx_clock.c 0x00000000   Number         0  nrfx_clock.o ABSOLUTE
    ..\..\..\..\..\..\modules\nrfx\drivers\src\nrfx_gpiote.c 0x00000000   Number         0  nrfx_gpiote.o ABSOLUTE
    ..\..\..\..\..\..\modules\nrfx\drivers\src\nrfx_spi.c 0x00000000   Number         0  nrfx_spi.o ABSOLUTE
    ..\..\..\..\..\..\modules\nrfx\drivers\src\nrfx_spim.c 0x00000000   Number         0  nrfx_spim.o ABSOLUTE
    ..\..\..\..\..\..\modules\nrfx\drivers\src\nrfx_uart.c 0x00000000   Number         0  nrfx_uart.o ABSOLUTE
    ..\..\..\..\..\..\modules\nrfx\drivers\src\nrfx_uarte.c 0x00000000   Number         0  nrfx_uarte.o ABSOLUTE
    ..\..\..\..\..\..\modules\nrfx\drivers\src\prs\nrfx_prs.c 0x00000000   Number         0  nrfx_prs.o ABSOLUTE
    ..\..\..\..\..\..\modules\nrfx\soc\nrfx_atomic.c 0x00000000   Number         0  nrfx_atomic.o ABSOLUTE
    ..\..\..\main.c                          0x00000000   Number         0  main.o ABSOLUTE
    ..\\..\\..\\..\\..\\..\\components\\ble\\ble_advertising\\ble_advertising.c 0x00000000   Number         0  ble_advertising.o ABSOLUTE
    ..\\..\\..\\..\\..\\..\\components\\ble\\ble_link_ctx_manager\\ble_link_ctx_manager.c 0x00000000   Number         0  ble_link_ctx_manager.o ABSOLUTE
    ..\\..\\..\\..\\..\\..\\components\\ble\\ble_services\\ble_nus\\ble_nus.c 0x00000000   Number         0  ble_nus.o ABSOLUTE
    ..\\..\\..\\..\\..\\..\\components\\ble\\common\\ble_advdata.c 0x00000000   Number         0  ble_advdata.o ABSOLUTE
    ..\\..\\..\\..\\..\\..\\components\\ble\\common\\ble_conn_params.c 0x00000000   Number         0  ble_conn_params.o ABSOLUTE
    ..\\..\\..\\..\\..\\..\\components\\ble\\common\\ble_conn_state.c 0x00000000   Number         0  ble_conn_state.o ABSOLUTE
    ..\\..\\..\\..\\..\\..\\components\\ble\\common\\ble_srv_common.c 0x00000000   Number         0  ble_srv_common.o ABSOLUTE
    ..\\..\\..\\..\\..\\..\\components\\ble\\nrf_ble_gatt\\nrf_ble_gatt.c 0x00000000   Number         0  nrf_ble_gatt.o ABSOLUTE
    ..\\..\\..\\..\\..\\..\\components\\ble\\nrf_ble_qwr\\nrf_ble_qwr.c 0x00000000   Number         0  nrf_ble_qwr.o ABSOLUTE
    ..\\..\\..\\..\\..\\..\\components\\boards\\boards.c 0x00000000   Number         0  boards.o ABSOLUTE
    ..\\..\\..\\..\\..\\..\\components\\libraries\\atomic\\nrf_atomic.c 0x00000000   Number         0  nrf_atomic.o ABSOLUTE
    ..\\..\\..\\..\\..\\..\\components\\libraries\\atomic_fifo\\nrf_atfifo.c 0x00000000   Number         0  nrf_atfifo.o ABSOLUTE
    ..\\..\\..\\..\\..\\..\\components\\libraries\\atomic_flags\\nrf_atflags.c 0x00000000   Number         0  nrf_atflags.o ABSOLUTE
    ..\\..\\..\\..\\..\\..\\components\\libraries\\balloc\\nrf_balloc.c 0x00000000   Number         0  nrf_balloc.o ABSOLUTE
    ..\\..\\..\\..\\..\\..\\components\\libraries\\block_dev\\sdc\\nrf_block_dev_sdc.c 0x00000000   Number         0  nrf_block_dev_sdc.o ABSOLUTE
    ..\\..\\..\\..\\..\\..\\components\\libraries\\bsp\\bsp.c 0x00000000   Number         0  bsp.o ABSOLUTE
    ..\\..\\..\\..\\..\\..\\components\\libraries\\bsp\\bsp_btn_ble.c 0x00000000   Number         0  bsp_btn_ble.o ABSOLUTE
    ..\\..\\..\\..\\..\\..\\components\\libraries\\button\\app_button.c 0x00000000   Number         0  app_button.o ABSOLUTE
    ..\\..\\..\\..\\..\\..\\components\\libraries\\experimental_section_vars\\nrf_section_iter.c 0x00000000   Number         0  nrf_section_iter.o ABSOLUTE
    ..\\..\\..\\..\\..\\..\\components\\libraries\\fifo\\app_fifo.c 0x00000000   Number         0  app_fifo.o ABSOLUTE
    ..\\..\\..\\..\\..\\..\\components\\libraries\\hardfault\\hardfault_implementation.c 0x00000000   Number         0  hardfault_implementation.o ABSOLUTE
    ..\\..\\..\\..\\..\\..\\components\\libraries\\log\\src\\nrf_log_backend_rtt.c 0x00000000   Number         0  nrf_log_backend_rtt.o ABSOLUTE
    ..\\..\\..\\..\\..\\..\\components\\libraries\\log\\src\\nrf_log_backend_serial.c 0x00000000   Number         0  nrf_log_backend_serial.o ABSOLUTE
    ..\\..\\..\\..\\..\\..\\components\\libraries\\log\\src\\nrf_log_backend_uart.c 0x00000000   Number         0  nrf_log_backend_uart.o ABSOLUTE
    ..\\..\\..\\..\\..\\..\\components\\libraries\\log\\src\\nrf_log_default_backends.c 0x00000000   Number         0  nrf_log_default_backends.o ABSOLUTE
    ..\\..\\..\\..\\..\\..\\components\\libraries\\log\\src\\nrf_log_frontend.c 0x00000000   Number         0  nrf_log_frontend.o ABSOLUTE
    ..\\..\\..\\..\\..\\..\\components\\libraries\\log\\src\\nrf_log_str_formatter.c 0x00000000   Number         0  nrf_log_str_formatter.o ABSOLUTE
    ..\\..\\..\\..\\..\\..\\components\\libraries\\memobj\\nrf_memobj.c 0x00000000   Number         0  nrf_memobj.o ABSOLUTE
    ..\\..\\..\\..\\..\\..\\components\\libraries\\pwr_mgmt\\nrf_pwr_mgmt.c 0x00000000   Number         0  nrf_pwr_mgmt.o ABSOLUTE
    ..\\..\\..\\..\\..\\..\\components\\libraries\\ringbuf\\nrf_ringbuf.c 0x00000000   Number         0  nrf_ringbuf.o ABSOLUTE
    ..\\..\\..\\..\\..\\..\\components\\libraries\\scheduler\\app_scheduler.c 0x00000000   Number         0  app_scheduler.o ABSOLUTE
    ..\\..\\..\\..\\..\\..\\components\\libraries\\sdcard\\app_sdcard.c 0x00000000   Number         0  app_sdcard.o ABSOLUTE
    ..\\..\\..\\..\\..\\..\\components\\libraries\\sortlist\\nrf_sortlist.c 0x00000000   Number         0  nrf_sortlist.o ABSOLUTE
    ..\\..\\..\\..\\..\\..\\components\\libraries\\strerror\\nrf_strerror.c 0x00000000   Number         0  nrf_strerror.o ABSOLUTE
    ..\\..\\..\\..\\..\\..\\components\\libraries\\timer\\app_timer2.c 0x00000000   Number         0  app_timer2.o ABSOLUTE
    ..\\..\\..\\..\\..\\..\\components\\libraries\\timer\\drv_rtc.c 0x00000000   Number         0  drv_rtc.o ABSOLUTE
    ..\\..\\..\\..\\..\\..\\components\\libraries\\uart\\app_uart_fifo.c 0x00000000   Number         0  app_uart_fifo.o ABSOLUTE
    ..\\..\\..\\..\\..\\..\\components\\libraries\\uart\\retarget.c 0x00000000   Number         0  retarget.o ABSOLUTE
    ..\\..\\..\\..\\..\\..\\components\\libraries\\util\\app_error.c 0x00000000   Number         0  app_error.o ABSOLUTE
    ..\\..\\..\\..\\..\\..\\components\\libraries\\util\\app_error_handler_keil.c 0x00000000   Number         0  app_error_handler_keil.o ABSOLUTE
    ..\\..\\..\\..\\..\\..\\components\\libraries\\util\\app_error_weak.c 0x00000000   Number         0  app_error_weak.o ABSOLUTE
    ..\\..\\..\\..\\..\\..\\components\\libraries\\util\\app_util_platform.c 0x00000000   Number         0  app_util_platform.o ABSOLUTE
    ..\\..\\..\\..\\..\\..\\components\\libraries\\util\\nrf_assert.c 0x00000000   Number         0  nrf_assert.o ABSOLUTE
    ..\\..\\..\\..\\..\\..\\components\\softdevice\\common\\nrf_sdh.c 0x00000000   Number         0  nrf_sdh.o ABSOLUTE
    ..\\..\\..\\..\\..\\..\\components\\softdevice\\common\\nrf_sdh_ble.c 0x00000000   Number         0  nrf_sdh_ble.o ABSOLUTE
    ..\\..\\..\\..\\..\\..\\components\\softdevice\\common\\nrf_sdh_soc.c 0x00000000   Number         0  nrf_sdh_soc.o ABSOLUTE
    ..\\..\\..\\..\\..\\..\\external\\fatfs\\port\\diskio_blkdev.c 0x00000000   Number         0  diskio_blkdev.o ABSOLUTE
    ..\\..\\..\\..\\..\\..\\external\\fprintf\\nrf_fprintf.c 0x00000000   Number         0  nrf_fprintf.o ABSOLUTE
    ..\\..\\..\\..\\..\\..\\external\\fprintf\\nrf_fprintf_format.c 0x00000000   Number         0  nrf_fprintf_format.o ABSOLUTE
    ..\\..\\..\\..\\..\\..\\external\\segger_rtt\\SEGGER_RTT.c 0x00000000   Number         0  segger_rtt.o ABSOLUTE
    ..\\..\\..\\..\\..\\..\\external\\segger_rtt\\SEGGER_RTT_printf.c 0x00000000   Number         0  segger_rtt_printf.o ABSOLUTE
    ..\\..\\..\\..\\..\\..\\integration\\nrfx\\legacy\\nrf_drv_clock.c 0x00000000   Number         0  nrf_drv_clock.o ABSOLUTE
    ..\\..\\..\\..\\..\\..\\integration\\nrfx\\legacy\\nrf_drv_spi.c 0x00000000   Number         0  nrf_drv_spi.o ABSOLUTE
    ..\\..\\..\\..\\..\\..\\integration\\nrfx\\legacy\\nrf_drv_uart.c 0x00000000   Number         0  nrf_drv_uart.o ABSOLUTE
    ..\\..\\..\\..\\..\\..\\modules\\nrfx\\drivers\\src\\nrfx_clock.c 0x00000000   Number         0  nrfx_clock.o ABSOLUTE
    ..\\..\\..\\..\\..\\..\\modules\\nrfx\\drivers\\src\\nrfx_gpiote.c 0x00000000   Number         0  nrfx_gpiote.o ABSOLUTE
    ..\\..\\..\\..\\..\\..\\modules\\nrfx\\drivers\\src\\nrfx_spi.c 0x00000000   Number         0  nrfx_spi.o ABSOLUTE
    ..\\..\\..\\..\\..\\..\\modules\\nrfx\\drivers\\src\\nrfx_spim.c 0x00000000   Number         0  nrfx_spim.o ABSOLUTE
    ..\\..\\..\\..\\..\\..\\modules\\nrfx\\drivers\\src\\nrfx_uart.c 0x00000000   Number         0  nrfx_uart.o ABSOLUTE
    ..\\..\\..\\..\\..\\..\\modules\\nrfx\\drivers\\src\\nrfx_uarte.c 0x00000000   Number         0  nrfx_uarte.o ABSOLUTE
    ..\\..\\..\\..\\..\\..\\modules\\nrfx\\drivers\\src\\prs\\nrfx_prs.c 0x00000000   Number         0  nrfx_prs.o ABSOLUTE
    ..\\..\\..\\..\\..\\..\\modules\\nrfx\\soc\\nrfx_atomic.c 0x00000000   Number         0  nrfx_atomic.o ABSOLUTE
    ..\\..\\..\\main.c                       0x00000000   Number         0  main.o ABSOLUTE
    RTE\Device\nRF52832_xxAA\arm_startup_nrf52.s 0x00000000   Number         0  arm_startup_nrf52.o ABSOLUTE
    RTE\Device\nRF52832_xxAA\system_nrf52.c  0x00000000   Number         0  system_nrf52.o ABSOLUTE
    RTE\\Device\\nRF52832_xxAA\\system_nrf52.c 0x00000000   Number         0  system_nrf52.o ABSOLUTE
    cdrcmple.s                               0x00000000   Number         0  cdrcmple.o ABSOLUTE
    dc.s                                     0x00000000   Number         0  dc.o ABSOLUTE
    handlers.s                               0x00000000   Number         0  handlers.o ABSOLUTE
    init.s                                   0x00000000   Number         0  init.o ABSOLUTE
    RESET                                    0x00026000   Section      512  arm_startup_nrf52.o(RESET)
    .ARM.Collect$$$$00000000                 0x00026200   Section        0  entry.o(.ARM.Collect$$$$00000000)
    .ARM.Collect$$$$00000001                 0x00026200   Section        4  entry2.o(.ARM.Collect$$$$00000001)
    .ARM.Collect$$$$00000004                 0x00026204   Section        4  entry5.o(.ARM.Collect$$$$00000004)
    .ARM.Collect$$$$00000008                 0x00026208   Section        0  entry7b.o(.ARM.Collect$$$$00000008)
    .ARM.Collect$$$$0000000A                 0x00026208   Section        0  entry8b.o(.ARM.Collect$$$$0000000A)
    .ARM.Collect$$$$0000000B                 0x00026208   Section        8  entry9a.o(.ARM.Collect$$$$0000000B)
    .ARM.Collect$$$$0000000D                 0x00026210   Section        0  entry10a.o(.ARM.Collect$$$$0000000D)
    .ARM.Collect$$$$0000000F                 0x00026210   Section        0  entry11a.o(.ARM.Collect$$$$0000000F)
    .ARM.Collect$$$$00002712                 0x00026210   Section        4  entry2.o(.ARM.Collect$$$$00002712)
    __lit__00000000                          0x00026210   Data           4  entry2.o(.ARM.Collect$$$$00002712)
    .emb_text                                0x00026214   Section      200  nrf_atfifo.o(.emb_text)
    $v0                                      0x00026214   Number         0  nrf_atfifo.o(.emb_text)
    .emb_text                                0x000262dc   Section      226  nrf_atomic.o(.emb_text)
    $v0                                      0x000262dc   Number         0  nrf_atomic.o(.emb_text)
    .text                                    0x000263c0   Section       36  arm_startup_nrf52.o(.text)
    $v0                                      0x000263c0   Number         0  arm_startup_nrf52.o(.text)
    .text                                    0x000263e4   Section        0  uldiv.o(.text)
    .text                                    0x00026446   Section        0  llshl.o(.text)
    .text                                    0x00026464   Section        0  ctype_o.o(.text)
    .text                                    0x0002646c   Section        0  memcpya.o(.text)
    .text                                    0x00026490   Section        0  memseta.o(.text)
    .text                                    0x000264b4   Section        0  strlen.o(.text)
    .text                                    0x000264c2   Section        0  strcpy.o(.text)
    .text                                    0x000264d4   Section        0  uidiv.o(.text)
    .text                                    0x00026500   Section        0  llushr.o(.text)
    .text                                    0x00026520   Section       36  init.o(.text)
    .text                                    0x00026544   Section        0  __dczerorl2.o(.text)
    i.Button_state                           0x0002659c   Section        0  main.o(i.Button_state)
    i.GPIOTE_IRQHandler                      0x00026664   Section        0  nrfx_gpiote.o(i.GPIOTE_IRQHandler)
    i.POWER_CLOCK_IRQHandler                 0x00026708   Section        0  nrfx_clock.o(i.POWER_CLOCK_IRQHandler)
    i.RTC1_IRQHandler                        0x00026760   Section        0  drv_rtc.o(i.RTC1_IRQHandler)
    i.SEGGER_RTT_Init                        0x00026770   Section        0  segger_rtt.o(i.SEGGER_RTT_Init)
    i.SEGGER_RTT_WriteNoLock                 0x00026774   Section        0  segger_rtt.o(i.SEGGER_RTT_WriteNoLock)
    i.SPIM0_SPIS0_TWIM0_TWIS0_SPI0_TWI0_IRQHandler 0x000267d0   Section        0  nrfx_spim.o(i.SPIM0_SPIS0_TWIM0_TWIS0_SPI0_TWI0_IRQHandler)
    i.SWI2_EGU2_IRQHandler                   0x00026824   Section        0  nrf_sdh.o(i.SWI2_EGU2_IRQHandler)
    i.SysTick_Handler                        0x00026828   Section        0  main.o(i.SysTick_Handler)
    i.SystemInit                             0x00026838   Section        0  system_nrf52.o(i.SystemInit)
    i.TIMER2_IRQHandler                      0x000268bc   Section        0  main.o(i.TIMER2_IRQHandler)
    i.UARTE0_UART0_IRQHandler                0x00026990   Section        0  nrfx_prs.o(i.UARTE0_UART0_IRQHandler)
    i._DoInit                                0x0002699c   Section        0  segger_rtt.o(i._DoInit)
    _DoInit                                  0x0002699d   Thumb Code    76  segger_rtt.o(i._DoInit)
    i._GetAvailWriteSpace                    0x00026a04   Section        0  segger_rtt.o(i._GetAvailWriteSpace)
    _GetAvailWriteSpace                      0x00026a05   Thumb Code    22  segger_rtt.o(i._GetAvailWriteSpace)
    i._WriteBlocking                         0x00026a1a   Section        0  segger_rtt.o(i._WriteBlocking)
    _WriteBlocking                           0x00026a1b   Thumb Code    90  segger_rtt.o(i._WriteBlocking)
    i._WriteNoCheck                          0x00026a74   Section        0  segger_rtt.o(i._WriteNoCheck)
    _WriteNoCheck                            0x00026a75   Thumb Code    66  segger_rtt.o(i._WriteNoCheck)
    i.__0sprintf$1                           0x00026ab8   Section        0  printf1.o(i.__0sprintf$1)
    i.__NVIC_SetPriority                     0x00026ae0   Section        0  main.o(i.__NVIC_SetPriority)
    __NVIC_SetPriority                       0x00026ae1   Thumb Code    32  main.o(i.__NVIC_SetPriority)
    i.__scatterload_copy                     0x00026b00   Section       14  handlers.o(i.__scatterload_copy)
    i.__scatterload_null                     0x00026b0e   Section        2  handlers.o(i.__scatterload_null)
    i.__scatterload_zeroinit                 0x00026b10   Section       14  handlers.o(i.__scatterload_zeroinit)
    i.__sd_nvic_app_accessible_irq           0x00026b20   Section        0  nrf_sdh.o(i.__sd_nvic_app_accessible_irq)
    __sd_nvic_app_accessible_irq             0x00026b21   Thumb Code    32  nrf_sdh.o(i.__sd_nvic_app_accessible_irq)
    i._printf_core                           0x00026b44   Section        0  printf1.o(i._printf_core)
    _printf_core                             0x00026b45   Thumb Code   336  printf1.o(i._printf_core)
    i._sputc                                 0x00026c98   Section        0  printf1.o(i._sputc)
    _sputc                                   0x00026c99   Thumb Code    10  printf1.o(i._sputc)
    i.adv_set_data_size_max_get              0x00026ca2   Section        0  ble_advertising.o(i.adv_set_data_size_max_get)
    adv_set_data_size_max_get                0x00026ca3   Thumb Code    16  ble_advertising.o(i.adv_set_data_size_max_get)
    i.advertising_buttons_configure          0x00026cb2   Section        0  bsp_btn_ble.o(i.advertising_buttons_configure)
    advertising_buttons_configure            0x00026cb3   Thumb Code    54  bsp_btn_ble.o(i.advertising_buttons_configure)
    i.app_error_fault_handler                0x00026ce8   Section        0  app_error_weak.o(i.app_error_fault_handler)
    i.app_error_handler_bare                 0x00026d6c   Section        0  app_error.o(i.app_error_handler_bare)
    i.app_fifo_get                           0x00026d82   Section        0  app_fifo.o(i.app_fifo_get)
    i.app_fifo_put                           0x00026d98   Section        0  app_fifo.o(i.app_fifo_put)
    i.app_sdc_block_read                     0x00026db4   Section        0  app_sdcard.o(i.app_sdc_block_read)
    i.app_sdc_block_write                    0x00026e0c   Section        0  app_sdcard.o(i.app_sdc_block_write)
    i.app_sdc_busy_check                     0x00026e78   Section        0  app_sdcard.o(i.app_sdc_busy_check)
    i.app_sdc_info_get                       0x00026e94   Section        0  app_sdcard.o(i.app_sdc_info_get)
    i.app_sdc_init                           0x00026eac   Section        0  app_sdcard.o(i.app_sdc_init)
    i.app_sdc_uninit                         0x00026f78   Section        0  app_sdcard.o(i.app_sdc_uninit)
    i.app_timer_cnt_get                      0x00026fc0   Section        0  app_timer2.o(i.app_timer_cnt_get)
    i.app_timer_init                         0x00026fcc   Section        0  app_timer2.o(i.app_timer_init)
    i.app_timer_start                        0x00027028   Section        0  app_timer2.o(i.app_timer_start)
    i.app_timer_stop                         0x00027058   Section        0  app_timer2.o(i.app_timer_stop)
    i.app_uart_put                           0x00027064   Section        0  app_uart_fifo.o(i.app_uart_put)
    i.app_util_critical_region_enter         0x000270b8   Section        0  app_util_platform.o(i.app_util_critical_region_enter)
    i.app_util_critical_region_exit          0x00027100   Section        0  app_util_platform.o(i.app_util_critical_region_exit)
    i.apply_config                           0x00027134   Section        0  nrfx_uart.o(i.apply_config)
    apply_config                             0x00027135   Thumb Code   136  nrfx_uart.o(i.apply_config)
    i.apply_config                           0x000271bc   Section        0  nrfx_uarte.o(i.apply_config)
    apply_config                             0x000271bd   Thumb Code   136  nrfx_uarte.o(i.apply_config)
    i.blcm_link_ctx_get                      0x00027244   Section        0  ble_link_ctx_manager.o(i.blcm_link_ctx_get)
    i.ble_advdata_encode                     0x0002728c   Section        0  ble_advdata.o(i.ble_advdata_encode)
    i.ble_advdata_parse                      0x0002740e   Section        0  ble_advdata.o(i.ble_advdata_parse)
    i.ble_advdata_search                     0x0002742e   Section        0  ble_advdata.o(i.ble_advdata_search)
    i.ble_advertising_conn_cfg_tag_set       0x00027474   Section        0  ble_advertising.o(i.ble_advertising_conn_cfg_tag_set)
    i.ble_advertising_init                   0x0002747a   Section        0  ble_advertising.o(i.ble_advertising_init)
    i.ble_advertising_on_ble_evt             0x00027572   Section        0  ble_advertising.o(i.ble_advertising_on_ble_evt)
    i.ble_advertising_start                  0x000275dc   Section        0  ble_advertising.o(i.ble_advertising_start)
    i.ble_conn_state_conn_idx                0x0002780c   Section        0  ble_conn_state.o(i.ble_conn_state_conn_idx)
    i.ble_conn_state_valid                   0x00027820   Section        0  ble_conn_state.o(i.ble_conn_state_valid)
    i.ble_device_addr_encode                 0x00027834   Section        0  ble_advdata.o(i.ble_device_addr_encode)
    ble_device_addr_encode                   0x00027835   Thumb Code    96  ble_advdata.o(i.ble_device_addr_encode)
    i.ble_evt_handler                        0x00027894   Section        0  main.o(i.ble_evt_handler)
    ble_evt_handler                          0x00027895   Thumb Code   174  main.o(i.ble_evt_handler)
    i.ble_evt_handler                        0x00027970   Section        0  bsp_btn_ble.o(i.ble_evt_handler)
    ble_evt_handler                          0x00027971   Thumb Code   106  bsp_btn_ble.o(i.ble_evt_handler)
    i.ble_evt_handler                        0x000279e0   Section        0  ble_conn_params.o(i.ble_evt_handler)
    ble_evt_handler                          0x000279e1   Thumb Code   242  ble_conn_params.o(i.ble_evt_handler)
    i.ble_evt_handler                        0x00027adc   Section        0  ble_conn_state.o(i.ble_evt_handler)
    ble_evt_handler                          0x00027add   Thumb Code   274  ble_conn_state.o(i.ble_evt_handler)
    i.ble_nus_init                           0x00027bf4   Section        0  ble_nus.o(i.ble_nus_init)
    i.ble_nus_on_ble_evt                     0x00027cc8   Section        0  ble_nus.o(i.ble_nus_on_ble_evt)
    i.ble_srv_is_notification_enabled        0x00027d3e   Section        0  ble_srv_common.o(i.ble_srv_is_notification_enabled)
    i.block_dev_handler                      0x00027d48   Section        0  diskio_blkdev.o(i.block_dev_handler)
    block_dev_handler                        0x00027d49   Thumb Code    40  diskio_blkdev.o(i.block_dev_handler)
    i.block_dev_sdc_geometry                 0x00027d74   Section        0  nrf_block_dev_sdc.o(i.block_dev_sdc_geometry)
    block_dev_sdc_geometry                   0x00027d75   Thumb Code     4  nrf_block_dev_sdc.o(i.block_dev_sdc_geometry)
    i.block_dev_sdc_init                     0x00027d78   Section        0  nrf_block_dev_sdc.o(i.block_dev_sdc_init)
    block_dev_sdc_init                       0x00027d79   Thumb Code   104  nrf_block_dev_sdc.o(i.block_dev_sdc_init)
    i.block_dev_sdc_ioctl                    0x00027dec   Section        0  nrf_block_dev_sdc.o(i.block_dev_sdc_ioctl)
    block_dev_sdc_ioctl                      0x00027ded   Thumb Code    32  nrf_block_dev_sdc.o(i.block_dev_sdc_ioctl)
    i.block_dev_sdc_read_req                 0x00027e0c   Section        0  nrf_block_dev_sdc.o(i.block_dev_sdc_read_req)
    block_dev_sdc_read_req                   0x00027e0d   Thumb Code   116  nrf_block_dev_sdc.o(i.block_dev_sdc_read_req)
    i.block_dev_sdc_uninit                   0x00027e88   Section        0  nrf_block_dev_sdc.o(i.block_dev_sdc_uninit)
    block_dev_sdc_uninit                     0x00027e89   Thumb Code    74  nrf_block_dev_sdc.o(i.block_dev_sdc_uninit)
    i.block_dev_sdc_write_req                0x00027edc   Section        0  nrf_block_dev_sdc.o(i.block_dev_sdc_write_req)
    block_dev_sdc_write_req                  0x00027edd   Thumb Code   116  nrf_block_dev_sdc.o(i.block_dev_sdc_write_req)
    i.bsp_board_button_idx_to_pin            0x00027f58   Section        0  boards.o(i.bsp_board_button_idx_to_pin)
    i.bsp_board_led_invert                   0x00027f64   Section        0  boards.o(i.bsp_board_led_invert)
    i.bsp_board_led_off                      0x00027f88   Section        0  boards.o(i.bsp_board_led_off)
    i.bsp_board_led_on                       0x00027f98   Section        0  boards.o(i.bsp_board_led_on)
    i.bsp_board_led_state_get                0x00027fa8   Section        0  boards.o(i.bsp_board_led_state_get)
    i.bsp_board_leds_off                     0x00027fc8   Section        0  boards.o(i.bsp_board_leds_off)
    i.bsp_board_leds_on                      0x00027fda   Section        0  boards.o(i.bsp_board_leds_on)
    i.bsp_board_pin_to_button_idx            0x00027fec   Section        0  boards.o(i.bsp_board_pin_to_button_idx)
    i.bsp_btn_ble_sleep_mode_prepare         0x00028010   Section        0  bsp_btn_ble.o(i.bsp_btn_ble_sleep_mode_prepare)
    i.bsp_button_event_handler               0x00028030   Section        0  bsp.o(i.bsp_button_event_handler)
    bsp_button_event_handler                 0x00028031   Thumb Code   132  bsp.o(i.bsp_button_event_handler)
    i.bsp_event_to_button_action_assign      0x000280c0   Section        0  bsp.o(i.bsp_event_to_button_action_assign)
    i.bsp_indication_set                     0x00028104   Section        0  bsp.o(i.bsp_indication_set)
    i.bsp_led_indication                     0x0002811c   Section        0  bsp.o(i.bsp_led_indication)
    bsp_led_indication                       0x0002811d   Thumb Code   446  bsp.o(i.bsp_led_indication)
    i.bsp_wakeup_button_enable               0x000282e4   Section        0  bsp.o(i.bsp_wakeup_button_enable)
    i.buf_prealloc                           0x000282ec   Section        0  nrf_log_frontend.o(i.buf_prealloc)
    buf_prealloc                             0x000282ed   Thumb Code   140  nrf_log_frontend.o(i.buf_prealloc)
    i.buffer_add                             0x00028380   Section        0  nrf_fprintf_format.o(i.buffer_add)
    buffer_add                               0x00028381   Thumb Code    46  nrf_fprintf_format.o(i.buffer_add)
    i.buffer_is_empty                        0x000283b0   Section        0  nrf_log_frontend.o(i.buffer_is_empty)
    i.channel_port_get                       0x000283c8   Section        0  nrfx_gpiote.o(i.channel_port_get)
    channel_port_get                         0x000283c9   Thumb Code    10  nrfx_gpiote.o(i.channel_port_get)
    i.characteristic_add                     0x000283d8   Section        0  ble_srv_common.o(i.characteristic_add)
    i.check_fs                               0x00028568   Section        0  ff.o(i.check_fs)
    check_fs                                 0x00028569   Thumb Code   102  ff.o(i.check_fs)
    i.clock_clk_started_notify               0x000285d8   Section        0  nrf_drv_clock.o(i.clock_clk_started_notify)
    clock_clk_started_notify                 0x000285d9   Thumb Code    34  nrf_drv_clock.o(i.clock_clk_started_notify)
    i.clock_irq_handler                      0x00028600   Section        0  nrf_drv_clock.o(i.clock_irq_handler)
    clock_irq_handler                        0x00028601   Thumb Code    24  nrf_drv_clock.o(i.clock_irq_handler)
    i.clust2sect                             0x0002861c   Section        0  ff.o(i.clust2sect)
    clust2sect                               0x0002861d   Thumb Code    24  ff.o(i.clust2sect)
    i.compare_func                           0x00028634   Section        0  app_timer2.o(i.compare_func)
    compare_func                             0x00028635   Thumb Code    24  app_timer2.o(i.compare_func)
    i.conn_handle_list_get                   0x0002864c   Section        0  ble_conn_state.o(i.conn_handle_list_get)
    i.conn_int_encode                        0x0002868a   Section        0  ble_advdata.o(i.conn_int_encode)
    conn_int_encode                          0x0002868b   Thumb Code   136  ble_advdata.o(i.conn_int_encode)
    i.conn_params_negotiation                0x00028714   Section        0  ble_conn_params.o(i.conn_params_negotiation)
    conn_params_negotiation                  0x00028715   Thumb Code    68  ble_conn_params.o(i.conn_params_negotiation)
    i.create_chain                           0x0002875c   Section        0  ff.o(i.create_chain)
    create_chain                             0x0002875d   Thumb Code   164  ff.o(i.create_chain)
    i.create_name                            0x00028800   Section        0  ff.o(i.create_name)
    create_name                              0x00028801   Thumb Code   210  ff.o(i.create_name)
    i.data_length_update                     0x000288e4   Section        0  nrf_ble_gatt.o(i.data_length_update)
    data_length_update                       0x000288e5   Thumb Code   110  nrf_ble_gatt.o(i.data_length_update)
    i.default_wait_func                      0x000289a4   Section        0  diskio_blkdev.o(i.default_wait_func)
    default_wait_func                        0x000289a5   Thumb Code     4  diskio_blkdev.o(i.default_wait_func)
    i.dir_find                               0x000289a8   Section        0  ff.o(i.dir_find)
    dir_find                                 0x000289a9   Thumb Code   100  ff.o(i.dir_find)
    i.dir_next                               0x00028a0c   Section        0  ff.o(i.dir_next)
    dir_next                                 0x00028a0d   Thumb Code   244  ff.o(i.dir_next)
    i.dir_register                           0x00028b00   Section        0  ff.o(i.dir_register)
    dir_register                             0x00028b01   Thumb Code   102  ff.o(i.dir_register)
    i.dir_sdi                                0x00028b66   Section        0  ff.o(i.dir_sdi)
    dir_sdi                                  0x00028b67   Thumb Code   130  ff.o(i.dir_sdi)
    i.disk_initialize                        0x00028be8   Section        0  diskio_blkdev.o(i.disk_initialize)
    i.disk_ioctl                             0x00028c68   Section        0  diskio_blkdev.o(i.disk_ioctl)
    i.disk_read                              0x00028ce4   Section        0  diskio_blkdev.o(i.disk_read)
    i.disk_status                            0x00028d60   Section        0  diskio_blkdev.o(i.disk_status)
    i.disk_write                             0x00028d80   Section        0  diskio_blkdev.o(i.disk_write)
    i.diskio_blockdev_register               0x00028e08   Section        0  diskio_blkdev.o(i.diskio_blockdev_register)
    i.dropped_sat16_get                      0x00028e14   Section        0  nrf_log_frontend.o(i.dropped_sat16_get)
    dropped_sat16_get                        0x00028e15   Thumb Code    16  nrf_log_frontend.o(i.dropped_sat16_get)
    i.drv_rtc_compare_disable                0x00028e28   Section        0  drv_rtc.o(i.drv_rtc_compare_disable)
    i.drv_rtc_compare_pending                0x00028e3c   Section        0  drv_rtc.o(i.drv_rtc_compare_pending)
    i.drv_rtc_compare_set                    0x00028e4a   Section        0  drv_rtc.o(i.drv_rtc_compare_set)
    i.drv_rtc_counter_get                    0x00028e9a   Section        0  drv_rtc.o(i.drv_rtc_counter_get)
    i.drv_rtc_init                           0x00028ea4   Section        0  drv_rtc.o(i.drv_rtc_init)
    i.drv_rtc_irq_trigger                    0x00028f7c   Section        0  drv_rtc.o(i.drv_rtc_irq_trigger)
    i.drv_rtc_overflow_enable                0x00028f9a   Section        0  drv_rtc.o(i.drv_rtc_overflow_enable)
    i.drv_rtc_overflow_pending               0x00028fa2   Section        0  drv_rtc.o(i.drv_rtc_overflow_pending)
    i.drv_rtc_start                          0x00028faa   Section        0  drv_rtc.o(i.drv_rtc_start)
    i.drv_rtc_stop                           0x00028fb2   Section        0  drv_rtc.o(i.drv_rtc_stop)
    i.drv_rtc_windowed_compare_set           0x00028fba   Section        0  drv_rtc.o(i.drv_rtc_windowed_compare_set)
    i.evt_enable                             0x00029098   Section        0  drv_rtc.o(i.evt_enable)
    evt_enable                               0x00029099   Thumb Code    18  drv_rtc.o(i.evt_enable)
    i.evt_pending                            0x000290aa   Section        0  drv_rtc.o(i.evt_pending)
    evt_pending                              0x000290ab   Thumb Code    20  drv_rtc.o(i.evt_pending)
    i.f_close                                0x000290be   Section        0  ff.o(i.f_close)
    i.f_mount                                0x000290dc   Section        0  ff.o(i.f_mount)
    i.f_open                                 0x00029128   Section        0  ff.o(i.f_open)
    i.f_opendir                              0x000292dc   Section        0  ff.o(i.f_opendir)
    i.f_sync                                 0x00029340   Section        0  ff.o(i.f_sync)
    i.f_write                                0x000293d0   Section        0  ff.o(i.f_write)
    i.fifo_get                               0x0002954e   Section        0  app_fifo.o(i.fifo_get)
    fifo_get                                 0x0002954f   Thumb Code    20  app_fifo.o(i.fifo_get)
    i.fifo_put                               0x00029562   Section        0  app_fifo.o(i.fifo_put)
    fifo_put                                 0x00029563   Thumb Code    18  app_fifo.o(i.fifo_put)
    i.find_volume                            0x00029574   Section        0  ff.o(i.find_volume)
    find_volume                              0x00029575   Thumb Code   576  ff.o(i.find_volume)
    i.flag_toggle                            0x000297c0   Section        0  ble_conn_state.o(i.flag_toggle)
    flag_toggle                              0x000297c1   Thumb Code    10  ble_conn_state.o(i.flag_toggle)
    i.flags_set                              0x000297ca   Section        0  ble_advertising.o(i.flags_set)
    flags_set                                0x000297cb   Thumb Code    40  ble_advertising.o(i.flags_set)
    i.follow_path                            0x000297f2   Section        0  ff.o(i.follow_path)
    follow_path                              0x000297f3   Thumb Code   116  ff.o(i.follow_path)
    i.get_fat                                0x00029866   Section        0  ff.o(i.get_fat)
    get_fat                                  0x00029867   Thumb Code   190  ff.o(i.get_fat)
    i.get_ldnumber                           0x00029924   Section        0  ff.o(i.get_ldnumber)
    get_ldnumber                             0x00029925   Thumb Code    60  ff.o(i.get_ldnumber)
    i.get_now                                0x00029960   Section        0  app_timer2.o(i.get_now)
    get_now                                  0x00029961   Thumb Code    46  app_timer2.o(i.get_now)
    i.instance_get                           0x00029994   Section        0  ble_conn_params.o(i.instance_get)
    instance_get                             0x00029995   Thumb Code    14  ble_conn_params.o(i.instance_get)
    i.int_print                              0x000299a8   Section        0  nrf_fprintf_format.o(i.int_print)
    int_print                                0x000299a9   Thumb Code   166  nrf_fprintf_format.o(i.int_print)
    i.interrupts_enable                      0x00029a50   Section        0  nrfx_uarte.o(i.interrupts_enable)
    interrupts_enable                        0x00029a51   Thumb Code   132  nrfx_uarte.o(i.interrupts_enable)
    i.invalid_packets_omit                   0x00029ad8   Section        0  nrf_log_frontend.o(i.invalid_packets_omit)
    invalid_packets_omit                     0x00029ad9   Thumb Code    52  nrf_log_frontend.o(i.invalid_packets_omit)
    i.is_conn_params_ok                      0x00029b0c   Section        0  ble_conn_params.o(i.is_conn_params_ok)
    is_conn_params_ok                        0x00029b0d   Thumb Code    68  ble_conn_params.o(i.is_conn_params_ok)
    i.ld_clust                               0x00029b50   Section        0  ff.o(i.ld_clust)
    ld_clust                                 0x00029b51   Thumb Code    38  ff.o(i.ld_clust)
    i.ld_dword                               0x00029b76   Section        0  ff.o(i.ld_dword)
    ld_dword                                 0x00029b77   Thumb Code    22  ff.o(i.ld_dword)
    i.ld_word                                0x00029b8c   Section        0  ff.o(i.ld_word)
    ld_word                                  0x00029b8d   Thumb Code    10  ff.o(i.ld_word)
    i.leds_off                               0x00029b98   Section        0  bsp.o(i.leds_off)
    leds_off                                 0x00029b99   Thumb Code    42  bsp.o(i.leds_off)
    i.link_init                              0x00029bc8   Section        0  nrf_ble_gatt.o(i.link_init)
    link_init                                0x00029bc9   Thumb Code    24  nrf_ble_gatt.o(i.link_init)
    i.log_skip                               0x00029be0   Section        0  nrf_log_frontend.o(i.log_skip)
    log_skip                                 0x00029be1   Thumb Code   150  nrf_log_frontend.o(i.log_skip)
    i.main                                   0x00029c84   Section        0  main.o(i.main)
    i.manuf_specific_data_encode             0x00029de4   Section        0  ble_advdata.o(i.manuf_specific_data_encode)
    manuf_specific_data_encode               0x00029de5   Thumb Code   100  ble_advdata.o(i.manuf_specific_data_encode)
    i.mem_cpy                                0x00029e48   Section        0  ff.o(i.mem_cpy)
    mem_cpy                                  0x00029e49   Thumb Code    18  ff.o(i.mem_cpy)
    i.mem_set                                0x00029e5c   Section        0  ff.o(i.mem_set)
    mem_set                                  0x00029e5d   Thumb Code    14  ff.o(i.mem_set)
    i.memobj_op                              0x00029e6a   Section        0  nrf_memobj.o(i.memobj_op)
    memobj_op                                0x00029e6b   Thumb Code   126  nrf_memobj.o(i.memobj_op)
    i.module_idx_get                         0x00029ee8   Section        0  nrf_log_frontend.o(i.module_idx_get)
    module_idx_get                           0x00029ee9   Thumb Code    42  nrf_log_frontend.o(i.module_idx_get)
    i.move_window                            0x00029f18   Section        0  ff.o(i.move_window)
    move_window                              0x00029f19   Thumb Code    50  ff.o(i.move_window)
    i.name_encode                            0x00029f4a   Section        0  ble_advdata.o(i.name_encode)
    name_encode                              0x00029f4b   Thumb Code   166  ble_advdata.o(i.name_encode)
    i.nrf_atfifo_init                        0x00029ff0   Section        0  nrf_atfifo.o(i.nrf_atfifo_init)
    i.nrf_atfifo_item_alloc                  0x0002a016   Section        0  nrf_atfifo.o(i.nrf_atfifo_item_alloc)
    i.nrf_atfifo_item_free                   0x0002a02c   Section        0  nrf_atfifo.o(i.nrf_atfifo_item_free)
    i.nrf_atfifo_item_get                    0x0002a042   Section        0  nrf_atfifo.o(i.nrf_atfifo_item_get)
    i.nrf_atfifo_item_put                    0x0002a058   Section        0  nrf_atfifo.o(i.nrf_atfifo_item_put)
    i.nrf_atflags_clear                      0x0002a06e   Section        0  nrf_atflags.o(i.nrf_atflags_clear)
    i.nrf_atflags_get                        0x0002a084   Section        0  nrf_atflags.o(i.nrf_atflags_get)
    i.nrf_atflags_set                        0x0002a09a   Section        0  nrf_atflags.o(i.nrf_atflags_set)
    i.nrf_atomic_flag_clear_fetch            0x0002a0ae   Section        0  nrf_atomic.o(i.nrf_atomic_flag_clear_fetch)
    i.nrf_atomic_flag_set                    0x0002a0b4   Section        0  nrf_atomic.o(i.nrf_atomic_flag_set)
    i.nrf_atomic_u32_add                     0x0002a0ba   Section        0  nrf_atomic.o(i.nrf_atomic_u32_add)
    i.nrf_atomic_u32_and                     0x0002a0c6   Section        0  nrf_atomic.o(i.nrf_atomic_u32_and)
    i.nrf_atomic_u32_fetch_and               0x0002a0d2   Section        0  nrf_atomic.o(i.nrf_atomic_u32_fetch_and)
    i.nrf_atomic_u32_fetch_store             0x0002a0dc   Section        0  nrf_atomic.o(i.nrf_atomic_u32_fetch_store)
    i.nrf_atomic_u32_or                      0x0002a0e6   Section        0  nrf_atomic.o(i.nrf_atomic_u32_or)
    i.nrf_atomic_u32_sub                     0x0002a0f2   Section        0  nrf_atomic.o(i.nrf_atomic_u32_sub)
    i.nrf_balloc_alloc                       0x0002a0fe   Section        0  nrf_balloc.o(i.nrf_balloc_alloc)
    i.nrf_balloc_free                        0x0002a142   Section        0  nrf_balloc.o(i.nrf_balloc_free)
    i.nrf_balloc_init                        0x0002a172   Section        0  nrf_balloc.o(i.nrf_balloc_init)
    i.nrf_bitmask_bit_is_set                 0x0002a1a2   Section        0  nrfx_gpiote.o(i.nrf_bitmask_bit_is_set)
    nrf_bitmask_bit_is_set                   0x0002a1a3   Thumb Code    16  nrfx_gpiote.o(i.nrf_bitmask_bit_is_set)
    i.nrf_ble_gatt_on_ble_evt                0x0002a1b4   Section        0  nrf_ble_gatt.o(i.nrf_ble_gatt_on_ble_evt)
    i.nrf_ble_qwr_conn_handle_assign         0x0002a304   Section        0  nrf_ble_qwr.o(i.nrf_ble_qwr_conn_handle_assign)
    i.nrf_ble_qwr_init                       0x0002a31a   Section        0  nrf_ble_qwr.o(i.nrf_ble_qwr_init)
    i.nrf_ble_qwr_on_ble_evt                 0x0002a33e   Section        0  nrf_ble_qwr.o(i.nrf_ble_qwr_on_ble_evt)
    i.nrf_blk_dev_ioctl                      0x0002a3f4   Section        0  diskio_blkdev.o(i.nrf_blk_dev_ioctl)
    nrf_blk_dev_ioctl                        0x0002a3f5   Thumb Code     6  diskio_blkdev.o(i.nrf_blk_dev_ioctl)
    i.nrf_clock_event_check                  0x0002a3fa   Section        0  nrfx_clock.o(i.nrf_clock_event_check)
    nrf_clock_event_check                    0x0002a3fb   Thumb Code    14  nrfx_clock.o(i.nrf_clock_event_check)
    i.nrf_clock_event_clear                  0x0002a408   Section        0  nrfx_clock.o(i.nrf_clock_event_clear)
    nrf_clock_event_clear                    0x0002a409   Thumb Code    16  nrfx_clock.o(i.nrf_clock_event_clear)
    i.nrf_drv_clock_init                     0x0002a418   Section        0  nrf_drv_clock.o(i.nrf_drv_clock_init)
    i.nrf_drv_clock_lfclk_release            0x0002a458   Section        0  nrf_drv_clock.o(i.nrf_drv_clock_lfclk_release)
    i.nrf_drv_spi_init                       0x0002a48c   Section        0  nrf_drv_spi.o(i.nrf_drv_spi_init)
    i.nrf_drv_spi_transfer                   0x0002a4fc   Section        0  app_sdcard.o(i.nrf_drv_spi_transfer)
    nrf_drv_spi_transfer                     0x0002a4fd   Thumb Code    22  app_sdcard.o(i.nrf_drv_spi_transfer)
    i.nrf_drv_uart_init                      0x0002a514   Section        0  nrf_drv_uart.o(i.nrf_drv_uart_init)
    i.nrf_drv_uart_tx                        0x0002a57c   Section        0  app_uart_fifo.o(i.nrf_drv_uart_tx)
    nrf_drv_uart_tx                          0x0002a57d   Thumb Code    26  app_uart_fifo.o(i.nrf_drv_uart_tx)
    i.nrf_fprintf                            0x0002a59c   Section        0  nrf_fprintf.o(i.nrf_fprintf)
    i.nrf_fprintf_buffer_flush               0x0002a5b6   Section        0  nrf_fprintf.o(i.nrf_fprintf_buffer_flush)
    i.nrf_fprintf_fmt                        0x0002a5ce   Section        0  nrf_fprintf_format.o(i.nrf_fprintf_fmt)
    i.nrf_gpio_cfg                           0x0002a7a8   Section        0  main.o(i.nrf_gpio_cfg)
    nrf_gpio_cfg                             0x0002a7a9   Thumb Code    36  main.o(i.nrf_gpio_cfg)
    i.nrf_gpio_cfg                           0x0002a7cc   Section        0  nrfx_uart.o(i.nrf_gpio_cfg)
    nrf_gpio_cfg                             0x0002a7cd   Thumb Code    36  nrfx_uart.o(i.nrf_gpio_cfg)
    i.nrf_gpio_cfg                           0x0002a7f0   Section        0  nrfx_uarte.o(i.nrf_gpio_cfg)
    nrf_gpio_cfg                             0x0002a7f1   Thumb Code    36  nrfx_uarte.o(i.nrf_gpio_cfg)
    i.nrf_gpio_cfg                           0x0002a814   Section        0  nrfx_spim.o(i.nrf_gpio_cfg)
    nrf_gpio_cfg                             0x0002a815   Thumb Code    36  nrfx_spim.o(i.nrf_gpio_cfg)
    i.nrf_gpio_cfg                           0x0002a838   Section        0  app_sdcard.o(i.nrf_gpio_cfg)
    nrf_gpio_cfg                             0x0002a839   Thumb Code    36  app_sdcard.o(i.nrf_gpio_cfg)
    i.nrf_gpio_cfg_default                   0x0002a85c   Section        0  nrfx_uart.o(i.nrf_gpio_cfg_default)
    nrf_gpio_cfg_default                     0x0002a85d   Thumb Code    18  nrfx_uart.o(i.nrf_gpio_cfg_default)
    i.nrf_gpio_cfg_default                   0x0002a86e   Section        0  nrfx_uarte.o(i.nrf_gpio_cfg_default)
    nrf_gpio_cfg_default                     0x0002a86f   Thumb Code    18  nrfx_uarte.o(i.nrf_gpio_cfg_default)
    i.nrf_gpio_cfg_input                     0x0002a880   Section        0  nrfx_uart.o(i.nrf_gpio_cfg_input)
    nrf_gpio_cfg_input                       0x0002a881   Thumb Code    18  nrfx_uart.o(i.nrf_gpio_cfg_input)
    i.nrf_gpio_cfg_input                     0x0002a892   Section        0  nrfx_uarte.o(i.nrf_gpio_cfg_input)
    nrf_gpio_cfg_input                       0x0002a893   Thumb Code    18  nrfx_uarte.o(i.nrf_gpio_cfg_input)
    i.nrf_gpio_cfg_output                    0x0002a8a4   Section        0  main.o(i.nrf_gpio_cfg_output)
    nrf_gpio_cfg_output                      0x0002a8a5   Thumb Code    20  main.o(i.nrf_gpio_cfg_output)
    i.nrf_gpio_cfg_output                    0x0002a8b8   Section        0  nrfx_uart.o(i.nrf_gpio_cfg_output)
    nrf_gpio_cfg_output                      0x0002a8b9   Thumb Code    20  nrfx_uart.o(i.nrf_gpio_cfg_output)
    i.nrf_gpio_cfg_output                    0x0002a8cc   Section        0  nrfx_uarte.o(i.nrf_gpio_cfg_output)
    nrf_gpio_cfg_output                      0x0002a8cd   Thumb Code    20  nrfx_uarte.o(i.nrf_gpio_cfg_output)
    i.nrf_gpio_cfg_output                    0x0002a8e0   Section        0  nrfx_spim.o(i.nrf_gpio_cfg_output)
    nrf_gpio_cfg_output                      0x0002a8e1   Thumb Code    20  nrfx_spim.o(i.nrf_gpio_cfg_output)
    i.nrf_gpio_cfg_sense_set                 0x0002a8f4   Section        0  nrfx_gpiote.o(i.nrf_gpio_cfg_sense_set)
    nrf_gpio_cfg_sense_set                   0x0002a8f5   Thumb Code    34  nrfx_gpiote.o(i.nrf_gpio_cfg_sense_set)
    i.nrf_gpio_latches_read_and_clear        0x0002a918   Section        0  nrfx_gpiote.o(i.nrf_gpio_latches_read_and_clear)
    nrf_gpio_latches_read_and_clear          0x0002a919   Thumb Code    38  nrfx_gpiote.o(i.nrf_gpio_latches_read_and_clear)
    i.nrf_gpio_pin_clear                     0x0002a944   Section        0  nrfx_spim.o(i.nrf_gpio_pin_clear)
    nrf_gpio_pin_clear                       0x0002a945   Thumb Code    14  nrfx_spim.o(i.nrf_gpio_pin_clear)
    i.nrf_gpio_pin_set                       0x0002a952   Section        0  nrfx_spim.o(i.nrf_gpio_pin_set)
    nrf_gpio_pin_set                         0x0002a953   Thumb Code    14  nrfx_spim.o(i.nrf_gpio_pin_set)
    i.nrf_gpio_pin_set                       0x0002a960   Section        0  app_sdcard.o(i.nrf_gpio_pin_set)
    nrf_gpio_pin_set                         0x0002a961   Thumb Code    14  app_sdcard.o(i.nrf_gpio_pin_set)
    i.nrf_gpio_pin_toggle                    0x0002a96e   Section        0  main.o(i.nrf_gpio_pin_toggle)
    nrf_gpio_pin_toggle                      0x0002a96f   Thumb Code    28  main.o(i.nrf_gpio_pin_toggle)
    i.nrf_gpio_pin_write                     0x0002a98a   Section        0  boards.o(i.nrf_gpio_pin_write)
    nrf_gpio_pin_write                       0x0002a98b   Thumb Code    22  boards.o(i.nrf_gpio_pin_write)
    i.nrf_gpiote_event_clear                 0x0002a9a0   Section        0  nrfx_gpiote.o(i.nrf_gpiote_event_clear)
    nrf_gpiote_event_clear                   0x0002a9a1   Thumb Code    16  nrfx_gpiote.o(i.nrf_gpiote_event_clear)
    i.nrf_gpiote_event_is_set                0x0002a9b4   Section        0  nrfx_gpiote.o(i.nrf_gpiote_event_is_set)
    nrf_gpiote_event_is_set                  0x0002a9b5   Thumb Code    12  nrfx_gpiote.o(i.nrf_gpiote_event_is_set)
    i.nrf_log_backend_add                    0x0002a9c4   Section        0  nrf_log_frontend.o(i.nrf_log_backend_add)
    i.nrf_log_backend_rtt_flush              0x0002aa20   Section        0  nrf_log_backend_rtt.o(i.nrf_log_backend_rtt_flush)
    nrf_log_backend_rtt_flush                0x0002aa21   Thumb Code     2  nrf_log_backend_rtt.o(i.nrf_log_backend_rtt_flush)
    i.nrf_log_backend_rtt_init               0x0002aa22   Section        0  nrf_log_backend_rtt.o(i.nrf_log_backend_rtt_init)
    i.nrf_log_backend_rtt_panic_set          0x0002aa26   Section        0  nrf_log_backend_rtt.o(i.nrf_log_backend_rtt_panic_set)
    nrf_log_backend_rtt_panic_set            0x0002aa27   Thumb Code     2  nrf_log_backend_rtt.o(i.nrf_log_backend_rtt_panic_set)
    i.nrf_log_backend_rtt_put                0x0002aa28   Section        0  nrf_log_backend_rtt.o(i.nrf_log_backend_rtt_put)
    nrf_log_backend_rtt_put                  0x0002aa29   Thumb Code    16  nrf_log_backend_rtt.o(i.nrf_log_backend_rtt_put)
    i.nrf_log_backend_serial_put             0x0002aa40   Section        0  nrf_log_backend_serial.o(i.nrf_log_backend_serial_put)
    i.nrf_log_backend_uart_flush             0x0002ab08   Section        0  nrf_log_backend_uart.o(i.nrf_log_backend_uart_flush)
    nrf_log_backend_uart_flush               0x0002ab09   Thumb Code     2  nrf_log_backend_uart.o(i.nrf_log_backend_uart_flush)
    i.nrf_log_backend_uart_init              0x0002ab0a   Section        0  nrf_log_backend_uart.o(i.nrf_log_backend_uart_init)
    i.nrf_log_backend_uart_panic_set         0x0002ab10   Section        0  nrf_log_backend_uart.o(i.nrf_log_backend_uart_panic_set)
    nrf_log_backend_uart_panic_set           0x0002ab11   Thumb Code    36  nrf_log_backend_uart.o(i.nrf_log_backend_uart_panic_set)
    i.nrf_log_backend_uart_put               0x0002ab3c   Section        0  nrf_log_backend_uart.o(i.nrf_log_backend_uart_put)
    nrf_log_backend_uart_put                 0x0002ab3d   Thumb Code    16  nrf_log_backend_uart.o(i.nrf_log_backend_uart_put)
    i.nrf_log_color_id_get                   0x0002ab54   Section        0  nrf_log_frontend.o(i.nrf_log_color_id_get)
    i.nrf_log_default_backends_init          0x0002ab84   Section        0  nrf_log_default_backends.o(i.nrf_log_default_backends_init)
    i.nrf_log_frontend_dequeue               0x0002abb8   Section        0  nrf_log_frontend.o(i.nrf_log_frontend_dequeue)
    i.nrf_log_frontend_std_0                 0x0002adf0   Section        0  nrf_log_frontend.o(i.nrf_log_frontend_std_0)
    i.nrf_log_frontend_std_1                 0x0002adf8   Section        0  nrf_log_frontend.o(i.nrf_log_frontend_std_1)
    i.nrf_log_frontend_std_2                 0x0002ae06   Section        0  nrf_log_frontend.o(i.nrf_log_frontend_std_2)
    i.nrf_log_hexdump_entry_process          0x0002ae18   Section        0  nrf_log_str_formatter.o(i.nrf_log_hexdump_entry_process)
    i.nrf_log_init                           0x0002aec8   Section        0  nrf_log_frontend.o(i.nrf_log_init)
    i.nrf_log_module_cnt_get                 0x0002aef0   Section        0  nrf_log_frontend.o(i.nrf_log_module_cnt_get)
    i.nrf_log_module_name_get                0x0002af04   Section        0  nrf_log_frontend.o(i.nrf_log_module_name_get)
    i.nrf_log_panic                          0x0002af20   Section        0  nrf_log_frontend.o(i.nrf_log_panic)
    i.nrf_log_std_entry_process              0x0002af48   Section        0  nrf_log_str_formatter.o(i.nrf_log_std_entry_process)
    i.nrf_memobj_alloc                       0x0002affe   Section        0  nrf_memobj.o(i.nrf_memobj_alloc)
    i.nrf_memobj_free                        0x0002b05e   Section        0  nrf_memobj.o(i.nrf_memobj_free)
    i.nrf_memobj_get                         0x0002b090   Section        0  nrf_memobj.o(i.nrf_memobj_get)
    i.nrf_memobj_pool_init                   0x0002b098   Section        0  nrf_memobj.o(i.nrf_memobj_pool_init)
    i.nrf_memobj_put                         0x0002b09c   Section        0  nrf_memobj.o(i.nrf_memobj_put)
    i.nrf_memobj_read                        0x0002b0ba   Section        0  nrf_memobj.o(i.nrf_memobj_read)
    i.nrf_memobj_write                       0x0002b0ca   Section        0  nrf_memobj.o(i.nrf_memobj_write)
    i.nrf_qwr_error_handler                  0x0002b0da   Section        0  main.o(i.nrf_qwr_error_handler)
    nrf_qwr_error_handler                    0x0002b0db   Thumb Code     4  main.o(i.nrf_qwr_error_handler)
    i.nrf_ringbuf_init                       0x0002b0de   Section        0  nrf_ringbuf.o(i.nrf_ringbuf_init)
    i.nrf_rtc_event_clear                    0x0002b0fa   Section        0  drv_rtc.o(i.nrf_rtc_event_clear)
    nrf_rtc_event_clear                      0x0002b0fb   Thumb Code    12  drv_rtc.o(i.nrf_rtc_event_clear)
    i.nrf_sdh_ble_app_ram_start_get          0x0002b108   Section        0  nrf_sdh_ble.o(i.nrf_sdh_ble_app_ram_start_get)
    i.nrf_sdh_ble_default_cfg_set            0x0002b11c   Section        0  nrf_sdh_ble.o(i.nrf_sdh_ble_default_cfg_set)
    i.nrf_sdh_ble_enable                     0x0002b24c   Section        0  nrf_sdh_ble.o(i.nrf_sdh_ble_enable)
    i.nrf_sdh_ble_evts_poll                  0x0002b37c   Section        0  nrf_sdh_ble.o(i.nrf_sdh_ble_evts_poll)
    nrf_sdh_ble_evts_poll                    0x0002b37d   Thumb Code    88  nrf_sdh_ble.o(i.nrf_sdh_ble_evts_poll)
    i.nrf_sdh_enable_request                 0x0002b3dc   Section        0  nrf_sdh.o(i.nrf_sdh_enable_request)
    i.nrf_sdh_evts_poll                      0x0002b450   Section        0  nrf_sdh.o(i.nrf_sdh_evts_poll)
    i.nrf_sdh_is_enabled                     0x0002b474   Section        0  nrf_sdh.o(i.nrf_sdh_is_enabled)
    i.nrf_sdh_soc_evts_poll                  0x0002b480   Section        0  nrf_sdh_soc.o(i.nrf_sdh_soc_evts_poll)
    nrf_sdh_soc_evts_poll                    0x0002b481   Thumb Code    56  nrf_sdh_soc.o(i.nrf_sdh_soc_evts_poll)
    i.nrf_section_iter_init                  0x0002b4bc   Section        0  nrf_section_iter.o(i.nrf_section_iter_init)
    i.nrf_section_iter_item_set              0x0002b4c6   Section        0  nrf_section_iter.o(i.nrf_section_iter_item_set)
    nrf_section_iter_item_set                0x0002b4c7   Thumb Code    36  nrf_section_iter.o(i.nrf_section_iter_item_set)
    i.nrf_section_iter_next                  0x0002b4ea   Section        0  nrf_section_iter.o(i.nrf_section_iter_next)
    i.nrf_sortlist_add                       0x0002b50a   Section        0  nrf_sortlist.o(i.nrf_sortlist_add)
    i.nrf_sortlist_peek                      0x0002b52c   Section        0  nrf_sortlist.o(i.nrf_sortlist_peek)
    i.nrf_sortlist_pop                       0x0002b532   Section        0  nrf_sortlist.o(i.nrf_sortlist_pop)
    i.nrf_sortlist_remove                    0x0002b540   Section        0  nrf_sortlist.o(i.nrf_sortlist_remove)
    i.nrf_spim_event_check                   0x0002b55e   Section        0  nrfx_spim.o(i.nrf_spim_event_check)
    nrf_spim_event_check                     0x0002b55f   Thumb Code    10  nrfx_spim.o(i.nrf_spim_event_check)
    i.nrf_strerror_find                      0x0002b568   Section        0  nrf_strerror.o(i.nrf_strerror_find)
    i.nrf_strerror_get                       0x0002b5a0   Section        0  nrf_strerror.o(i.nrf_strerror_get)
    i.nrf_uart_event_check                   0x0002b5b4   Section        0  nrfx_uart.o(i.nrf_uart_event_check)
    nrf_uart_event_check                     0x0002b5b5   Thumb Code    10  nrfx_uart.o(i.nrf_uart_event_check)
    i.nrf_uart_event_clear                   0x0002b5be   Section        0  nrfx_uart.o(i.nrf_uart_event_clear)
    nrf_uart_event_clear                     0x0002b5bf   Thumb Code    12  nrfx_uart.o(i.nrf_uart_event_clear)
    i.nrf_uart_int_enable_check              0x0002b5ca   Section        0  nrfx_uart.o(i.nrf_uart_int_enable_check)
    nrf_uart_int_enable_check                0x0002b5cb   Thumb Code    12  nrfx_uart.o(i.nrf_uart_int_enable_check)
    i.nrf_uarte_event_check                  0x0002b5d6   Section        0  nrfx_uarte.o(i.nrf_uarte_event_check)
    nrf_uarte_event_check                    0x0002b5d7   Thumb Code    10  nrfx_uarte.o(i.nrf_uarte_event_check)
    i.nrf_uarte_event_clear                  0x0002b5e0   Section        0  nrfx_uarte.o(i.nrf_uarte_event_clear)
    nrf_uarte_event_clear                    0x0002b5e1   Thumb Code    12  nrfx_uarte.o(i.nrf_uarte_event_clear)
    i.nrf_wdt_started                        0x0002b5ec   Section        0  nrf_drv_clock.o(i.nrf_wdt_started)
    nrf_wdt_started                          0x0002b5ed   Thumb Code    12  nrf_drv_clock.o(i.nrf_wdt_started)
    i.nrfx_clock_enable                      0x0002b5fc   Section        0  nrfx_clock.o(i.nrfx_clock_enable)
    i.nrfx_clock_init                        0x0002b628   Section        0  nrfx_clock.o(i.nrfx_clock_init)
    i.nrfx_clock_lfclk_stop                  0x0002b648   Section        0  nrfx_clock.o(i.nrfx_clock_lfclk_stop)
    i.nrfx_coredep_delay_us                  0x0002b678   Section        0  drv_rtc.o(i.nrfx_coredep_delay_us)
    nrfx_coredep_delay_us                    0x0002b679   Thumb Code    12  drv_rtc.o(i.nrfx_coredep_delay_us)
    i.nrfx_is_in_ram                         0x0002b688   Section        0  nrfx_uarte.o(i.nrfx_is_in_ram)
    nrfx_is_in_ram                           0x0002b689   Thumb Code    16  nrfx_uarte.o(i.nrfx_is_in_ram)
    i.nrfx_is_in_ram                         0x0002b698   Section        0  nrfx_spim.o(i.nrfx_is_in_ram)
    nrfx_is_in_ram                           0x0002b699   Thumb Code    16  nrfx_spim.o(i.nrfx_is_in_ram)
    i.nrfx_prs_acquire                       0x0002b6a8   Section        0  nrfx_prs.o(i.nrfx_prs_acquire)
    i.nrfx_prs_release                       0x0002b6e2   Section        0  nrfx_prs.o(i.nrfx_prs_release)
    i.nrfx_spim_init                         0x0002b6f4   Section        0  nrfx_spim.o(i.nrfx_spim_init)
    i.nrfx_spim_uninit                       0x0002b860   Section        0  nrfx_spim.o(i.nrfx_spim_uninit)
    i.nrfx_spim_xfer                         0x0002b8f4   Section        0  nrfx_spim.o(i.nrfx_spim_xfer)
    i.nrfx_uart_0_irq_handler                0x0002b958   Section        0  nrfx_uart.o(i.nrfx_uart_0_irq_handler)
    i.nrfx_uart_init                         0x0002b968   Section        0  nrfx_uart.o(i.nrfx_uart_init)
    i.nrfx_uart_tx                           0x0002ba3c   Section        0  nrfx_uart.o(i.nrfx_uart_tx)
    i.nrfx_uart_tx_in_progress               0x0002bae4   Section        0  nrfx_uart.o(i.nrfx_uart_tx_in_progress)
    i.nrfx_uart_uninit                       0x0002bb04   Section        0  nrfx_uart.o(i.nrfx_uart_uninit)
    i.nrfx_uarte_0_irq_handler               0x0002bbc4   Section        0  nrfx_uarte.o(i.nrfx_uarte_0_irq_handler)
    i.nrfx_uarte_init                        0x0002bbd4   Section        0  nrfx_uarte.o(i.nrfx_uarte_init)
    i.nrfx_uarte_tx                          0x0002bc40   Section        0  nrfx_uarte.o(i.nrfx_uarte_tx)
    i.nrfx_uarte_tx_in_progress              0x0002bcec   Section        0  nrfx_uarte.o(i.nrfx_uarte_tx_in_progress)
    i.nrfx_uarte_uninit                      0x0002bd08   Section        0  nrfx_uarte.o(i.nrfx_uarte_uninit)
    i.nus_data_handler                       0x0002be10   Section        0  main.o(i.nus_data_handler)
    nus_data_handler                         0x0002be11   Thumb Code    98  main.o(i.nus_data_handler)
    i.nvmc_config                            0x0002bea8   Section        0  system_nrf52.o(i.nvmc_config)
    i.on_adv_evt                             0x0002bec0   Section        0  main.o(i.on_adv_evt)
    on_adv_evt                               0x0002bec1   Thumb Code    54  main.o(i.on_adv_evt)
    i.on_connect                             0x0002bef6   Section        0  ble_nus.o(i.on_connect)
    on_connect                               0x0002bef7   Thumb Code   106  ble_nus.o(i.on_connect)
    i.on_connected_evt                       0x0002bf60   Section        0  nrf_ble_gatt.o(i.on_connected_evt)
    on_connected_evt                         0x0002bf61   Thumb Code   106  nrf_ble_gatt.o(i.on_connected_evt)
    i.on_exchange_mtu_request_evt            0x0002c008   Section        0  nrf_ble_gatt.o(i.on_exchange_mtu_request_evt)
    on_exchange_mtu_request_evt              0x0002c009   Thumb Code   110  nrf_ble_gatt.o(i.on_exchange_mtu_request_evt)
    i.on_write                               0x0002c0b4   Section        0  ble_nus.o(i.on_write)
    on_write                                 0x0002c0b5   Thumb Code   132  ble_nus.o(i.on_write)
    i.phy_is_valid                           0x0002c138   Section        0  ble_advertising.o(i.phy_is_valid)
    phy_is_valid                             0x0002c139   Thumb Code    18  ble_advertising.o(i.phy_is_valid)
    i.port_event_handle                      0x0002c14c   Section        0  nrfx_gpiote.o(i.port_event_handle)
    port_event_handle                        0x0002c14d   Thumb Code   176  nrfx_gpiote.o(i.port_event_handle)
    i.port_handler_polarity_get              0x0002c200   Section        0  nrfx_gpiote.o(i.port_handler_polarity_get)
    port_handler_polarity_get                0x0002c201   Thumb Code    12  nrfx_gpiote.o(i.port_handler_polarity_get)
    i.postfix_process                        0x0002c210   Section        0  nrf_log_str_formatter.o(i.postfix_process)
    postfix_process                          0x0002c211   Thumb Code    48  nrf_log_str_formatter.o(i.postfix_process)
    i.prefix_process                         0x0002c24c   Section        0  nrf_log_str_formatter.o(i.prefix_process)
    prefix_process                           0x0002c24d   Thumb Code    90  nrf_log_str_formatter.o(i.prefix_process)
    i.prs_box_get                            0x0002c2e4   Section        0  nrfx_prs.o(i.prs_box_get)
    prs_box_get                              0x0002c2e5   Thumb Code    14  nrfx_prs.o(i.prs_box_get)
    i.put_fat                                0x0002c2fc   Section        0  ff.o(i.put_fat)
    put_fat                                  0x0002c2fd   Thumb Code   234  ff.o(i.put_fat)
    i.remove_chain                           0x0002c3e6   Section        0  ff.o(i.remove_chain)
    remove_chain                             0x0002c3e7   Thumb Code   116  ff.o(i.remove_chain)
    i.rtc_irq                                0x0002c45c   Section        0  app_timer2.o(i.rtc_irq)
    rtc_irq                                  0x0002c45d   Thumb Code    88  app_timer2.o(i.rtc_irq)
    i.rtc_schedule                           0x0002c4b8   Section        0  app_timer2.o(i.rtc_schedule)
    rtc_schedule                             0x0002c4b9   Thumb Code    92  app_timer2.o(i.rtc_schedule)
    i.rtc_update                             0x0002c51c   Section        0  app_timer2.o(i.rtc_update)
    rtc_update                               0x0002c51d   Thumb Code   108  app_timer2.o(i.rtc_update)
    i.rx_byte                                0x0002c590   Section        0  nrfx_uart.o(i.rx_byte)
    rx_byte                                  0x0002c591   Thumb Code    50  nrfx_uart.o(i.rx_byte)
    i.rx_done_event                          0x0002c5c2   Section        0  nrfx_uart.o(i.rx_done_event)
    rx_done_event                            0x0002c5c3   Thumb Code    22  nrfx_uart.o(i.rx_done_event)
    i.rx_done_event                          0x0002c5d8   Section        0  nrfx_uarte.o(i.rx_done_event)
    rx_done_event                            0x0002c5d9   Thumb Code    22  nrfx_uarte.o(i.rx_done_event)
    i.saadc_init                             0x0002c5f0   Section        0  main.o(i.saadc_init)
    i.saadc_start                            0x0002c644   Section        0  main.o(i.saadc_start)
    i.sd_data_saving                         0x0002c66c   Section        0  main.o(i.sd_data_saving)
    sd_data_saving                           0x0002c66d   Thumb Code   454  main.o(i.sd_data_saving)
    i.sd_state_evt_handler                   0x0002c9ec   Section        0  nrf_drv_clock.o(i.sd_state_evt_handler)
    sd_state_evt_handler                     0x0002c9ed   Thumb Code    84  nrf_drv_clock.o(i.sd_state_evt_handler)
    i.sdc_cmd                                0x0002ca44   Section        0  app_sdcard.o(i.sdc_cmd)
    sdc_cmd                                  0x0002ca45   Thumb Code   178  app_sdcard.o(i.sdc_cmd)
    i.sdc_handler                            0x0002cafc   Section        0  nrf_block_dev_sdc.o(i.sdc_handler)
    sdc_handler                              0x0002cafd   Thumb Code   148  nrf_block_dev_sdc.o(i.sdc_handler)
    i.sdc_pt_identification                  0x0002cb98   Section        0  app_sdcard.o(i.sdc_pt_identification)
    sdc_pt_identification                    0x0002cb99   Thumb Code   662  app_sdcard.o(i.sdc_pt_identification)
    i.sdc_pt_read                            0x0002ce34   Section        0  app_sdcard.o(i.sdc_pt_read)
    sdc_pt_read                              0x0002ce35   Thumb Code   122  app_sdcard.o(i.sdc_pt_read)
    i.sdc_pt_sub_data_read                   0x0002ceb4   Section        0  app_sdcard.o(i.sdc_pt_sub_data_read)
    sdc_pt_sub_data_read                     0x0002ceb5   Thumb Code   348  app_sdcard.o(i.sdc_pt_sub_data_read)
    i.sdc_pt_write                           0x0002d014   Section        0  app_sdcard.o(i.sdc_pt_write)
    sdc_pt_write                             0x0002d015   Thumb Code   516  app_sdcard.o(i.sdc_pt_write)
    i.sdc_spi_transfer                       0x0002d21c   Section        0  app_sdcard.o(i.sdc_spi_transfer)
    sdc_spi_transfer                         0x0002d21d   Thumb Code    50  app_sdcard.o(i.sdc_spi_transfer)
    i.sdh_request_observer_notify            0x0002d258   Section        0  nrf_sdh.o(i.sdh_request_observer_notify)
    sdh_request_observer_notify              0x0002d259   Thumb Code    44  nrf_sdh.o(i.sdh_request_observer_notify)
    i.sdh_state_observer_notify              0x0002d288   Section        0  nrf_sdh.o(i.sdh_state_observer_notify)
    sdh_state_observer_notify                0x0002d289   Thumb Code    38  nrf_sdh.o(i.sdh_state_observer_notify)
    i.send_error_evt                         0x0002d2b4   Section        0  ble_conn_params.o(i.send_error_evt)
    send_error_evt                           0x0002d2b5   Thumb Code    12  ble_conn_params.o(i.send_error_evt)
    i.serial_tx                              0x0002d2c4   Section        0  nrf_log_backend_rtt.o(i.serial_tx)
    serial_tx                                0x0002d2c5   Thumb Code    70  nrf_log_backend_rtt.o(i.serial_tx)
    i.serial_tx                              0x0002d314   Section        0  nrf_log_backend_uart.o(i.serial_tx)
    serial_tx                                0x0002d315   Thumb Code    54  nrf_log_backend_uart.o(i.serial_tx)
    i.service_data_encode                    0x0002d354   Section        0  ble_advdata.o(i.service_data_encode)
    service_data_encode                      0x0002d355   Thumb Code   136  ble_advdata.o(i.service_data_encode)
    i.set_security_req                       0x0002d3dc   Section        0  ble_srv_common.o(i.set_security_req)
    set_security_req                         0x0002d3dd   Thumb Code    48  ble_srv_common.o(i.set_security_req)
    i.soc_evt_handler                        0x0002d40c   Section        0  nrf_drv_clock.o(i.soc_evt_handler)
    soc_evt_handler                          0x0002d40d   Thumb Code    18  nrf_drv_clock.o(i.soc_evt_handler)
    i.softdevices_evt_irq_enable             0x0002d424   Section        0  nrf_sdh.o(i.softdevices_evt_irq_enable)
    softdevices_evt_irq_enable               0x0002d425   Thumb Code    80  nrf_sdh.o(i.softdevices_evt_irq_enable)
    i.sortlist_pop                           0x0002d47c   Section        0  app_timer2.o(i.sortlist_pop)
    sortlist_pop                             0x0002d47d   Thumb Code     6  app_timer2.o(i.sortlist_pop)
    i.spi_handler                            0x0002d488   Section        0  app_sdcard.o(i.spi_handler)
    spi_handler                              0x0002d489   Thumb Code   434  app_sdcard.o(i.spi_handler)
    i.spim_evt_handler                       0x0002d644   Section        0  nrf_drv_spi.o(i.spim_evt_handler)
    spim_evt_handler                         0x0002d645   Thumb Code    52  nrf_drv_spi.o(i.spim_evt_handler)
    i.spim_xfer                              0x0002d67c   Section        0  nrfx_spim.o(i.spim_xfer)
    spim_xfer                                0x0002d67d   Thumb Code   188  nrfx_spim.o(i.spim_xfer)
    i.st_clust                               0x0002d738   Section        0  ff.o(i.st_clust)
    st_clust                                 0x0002d739   Thumb Code    40  ff.o(i.st_clust)
    i.st_dword                               0x0002d760   Section        0  ff.o(i.st_dword)
    st_dword                                 0x0002d761   Thumb Code    16  ff.o(i.st_dword)
    i.st_word                                0x0002d770   Section        0  ff.o(i.st_word)
    st_word                                  0x0002d771   Thumb Code     8  ff.o(i.st_word)
    i.std_n                                  0x0002d778   Section        0  nrf_log_frontend.o(i.std_n)
    std_n                                    0x0002d779   Thumb Code   140  nrf_log_frontend.o(i.std_n)
    i.sync_fs                                0x0002d80c   Section        0  ff.o(i.sync_fs)
    sync_fs                                  0x0002d80d   Thumb Code   126  ff.o(i.sync_fs)
    i.sync_window                            0x0002d894   Section        0  ff.o(i.sync_window)
    sync_window                              0x0002d895   Thumb Code    82  ff.o(i.sync_window)
    i.timer_expire                           0x0002d8e8   Section        0  app_timer2.o(i.timer_expire)
    timer_expire                             0x0002d8e9   Thumb Code    80  app_timer2.o(i.timer_expire)
    i.timer_init                             0x0002d940   Section        0  main.o(i.timer_init)
    i.timer_req_process                      0x0002d988   Section        0  app_timer2.o(i.timer_req_process)
    timer_req_process                        0x0002d989   Thumb Code   110  app_timer2.o(i.timer_req_process)
    i.timer_req_schedule                     0x0002da00   Section        0  app_timer2.o(i.timer_req_schedule)
    timer_req_schedule                       0x0002da01   Thumb Code    46  app_timer2.o(i.timer_req_schedule)
    i.tx_byte                                0x0002da38   Section        0  nrfx_uart.o(i.tx_byte)
    tx_byte                                  0x0002da39   Thumb Code    32  nrfx_uart.o(i.tx_byte)
    i.tx_done_event                          0x0002da58   Section        0  nrfx_uart.o(i.tx_done_event)
    tx_done_event                            0x0002da59   Thumb Code    26  nrfx_uart.o(i.tx_done_event)
    i.tx_done_event                          0x0002da72   Section        0  nrfx_uarte.o(i.tx_done_event)
    tx_done_event                            0x0002da73   Thumb Code    26  nrfx_uarte.o(i.tx_done_event)
    i.uart_evt_handler                       0x0002da8c   Section        0  nrf_drv_uart.o(i.uart_evt_handler)
    uart_evt_handler                         0x0002da8d   Thumb Code    42  nrf_drv_uart.o(i.uart_evt_handler)
    i.uart_evt_handler                       0x0002dabc   Section        0  nrf_log_backend_uart.o(i.uart_evt_handler)
    uart_evt_handler                         0x0002dabd   Thumb Code     8  nrf_log_backend_uart.o(i.uart_evt_handler)
    i.uart_init                              0x0002dac8   Section        0  nrf_log_backend_uart.o(i.uart_init)
    uart_init                                0x0002dac9   Thumb Code    66  nrf_log_backend_uart.o(i.uart_init)
    i.uart_irq_handler                       0x0002db18   Section        0  nrfx_uart.o(i.uart_irq_handler)
    uart_irq_handler                         0x0002db19   Thumb Code   298  nrfx_uart.o(i.uart_irq_handler)
    i.uarte_evt_handler                      0x0002dc44   Section        0  nrf_drv_uart.o(i.uarte_evt_handler)
    uarte_evt_handler                        0x0002dc45   Thumb Code    42  nrf_drv_uart.o(i.uarte_evt_handler)
    i.uarte_irq_handler                      0x0002dc74   Section        0  nrfx_uarte.o(i.uarte_irq_handler)
    uarte_irq_handler                        0x0002dc75   Thumb Code   274  nrfx_uarte.o(i.uarte_irq_handler)
    i.uint16_encode                          0x0002dd86   Section        0  ble_advdata.o(i.uint16_encode)
    uint16_encode                            0x0002dd87   Thumb Code    10  ble_advdata.o(i.uint16_encode)
    i.unsigned_print                         0x0002dd90   Section        0  nrf_fprintf_format.o(i.unsigned_print)
    unsigned_print                           0x0002dd91   Thumb Code   176  nrf_fprintf_format.o(i.unsigned_print)
    i.use_whitelist                          0x0002de44   Section        0  ble_advertising.o(i.use_whitelist)
    use_whitelist                            0x0002de45   Thumb Code    24  ble_advertising.o(i.use_whitelist)
    i.user_mem_reply                         0x0002de5c   Section        0  nrf_ble_qwr.o(i.user_mem_reply)
    user_mem_reply                           0x0002de5d   Thumb Code    36  nrf_ble_qwr.o(i.user_mem_reply)
    i.uuid_list_encode                       0x0002de80   Section        0  ble_advdata.o(i.uuid_list_encode)
    uuid_list_encode                         0x0002de81   Thumb Code    48  ble_advdata.o(i.uuid_list_encode)
    i.uuid_list_sized_encode                 0x0002deb0   Section        0  ble_advdata.o(i.uuid_list_sized_encode)
    uuid_list_sized_encode                   0x0002deb1   Thumb Code   158  ble_advdata.o(i.uuid_list_sized_encode)
    i.validate                               0x0002df4e   Section        0  ff.o(i.validate)
    validate                                 0x0002df4f   Thumb Code    50  ff.o(i.validate)
    i.wakeup_button_cfg                      0x0002df80   Section        0  bsp.o(i.wakeup_button_cfg)
    wakeup_button_cfg                        0x0002df81   Thumb Code    58  bsp.o(i.wakeup_button_cfg)
    .constdata                               0x0002dfbc   Section       28  main.o(.constdata)
    m_block_dev_sdc                          0x0002dfbc   Data          28  main.o(.constdata)
    .constdata                               0x0002dfd8   Section        8  boards.o(.constdata)
    m_board_led_list                         0x0002dfd8   Data           4  boards.o(.constdata)
    m_board_btn_list                         0x0002dfdc   Data           4  boards.o(.constdata)
    .constdata                               0x0002dfe0   Section       44  bsp.o(.constdata)
    m_bsp_leds_tmr                           0x0002dfe0   Data           4  bsp.o(.constdata)
    m_bsp_alert_tmr                          0x0002dfe4   Data           4  bsp.o(.constdata)
    m_bsp_button_tmr                         0x0002dfe8   Data           4  bsp.o(.constdata)
    app_buttons                              0x0002dfec   Data          32  bsp.o(.constdata)
    .constdata                               0x0002e00c   Section       22  nrf_ble_gatt.o(.constdata)
    .constdata                               0x0002e024   Section       16  ble_nus.o(.constdata)
    .constdata                               0x0002e034   Section        4  nrfx_gpiote.o(.constdata)
    .constdata                               0x0002e038   Section        4  nrfx_uart.o(.constdata)
    irq_handlers                             0x0002e038   Data           4  nrfx_uart.o(.constdata)
    .constdata                               0x0002e03c   Section        4  nrfx_uarte.o(.constdata)
    irq_handlers                             0x0002e03c   Data           4  nrfx_uarte.o(.constdata)
    .constdata                               0x0002e040   Section       16  nrf_drv_spi.o(.constdata)
    .constdata                               0x0002e050   Section        4  nrfx_spim.o(.constdata)
    irq_handlers                             0x0002e050   Data           4  nrfx_spim.o(.constdata)
    .constdata                               0x0002e054   Section       20  app_timer2.o(.constdata)
    m_req_fifo                               0x0002e054   Data           4  app_timer2.o(.constdata)
    m_app_timer_sortlist                     0x0002e05c   Data          12  app_timer2.o(.constdata)
    .constdata                               0x0002e070   Section        6  drv_rtc.o(.constdata)
    delay_machine_code                       0x0002e070   Data           6  drv_rtc.o(.constdata)
    .constdata                               0x0002e076   Section       16  nrf_fprintf_format.o(.constdata)
    _aV2C                                    0x0002e076   Data          16  nrf_fprintf_format.o(.constdata)
    .constdata                               0x0002e088   Section      316  nrf_strerror.o(.constdata)
    m_unknown_str                            0x0002e088   Data          19  nrf_strerror.o(.constdata)
    nrf_strerror_array                       0x0002e09c   Data         296  nrf_strerror.o(.constdata)
    .constdata                               0x0002e1c4   Section       32  app_sdcard.o(.constdata)
    m_spi                                    0x0002e1c4   Data          16  app_sdcard.o(.constdata)
    .constdata                               0x0002e1e4   Section       24  nrf_block_dev_sdc.o(.constdata)
    .constdata                               0x0002e1fc   Section       72  nrf_block_dev_sdc.o(.constdata)
    .constdata                               0x0002e244   Section       12  nrf_log_backend_rtt.o(.constdata)
    .constdata                               0x0002e250   Section        6  nrf_log_backend_rtt.o(.constdata)
    delay_machine_code                       0x0002e250   Data           6  nrf_log_backend_rtt.o(.constdata)
    .constdata                               0x0002e258   Section       12  nrf_log_frontend.o(.constdata)
    m_log_push_ringbuf                       0x0002e258   Data          12  nrf_log_frontend.o(.constdata)
    .constdata                               0x0002e264   Section       12  nrf_log_backend_uart.o(.constdata)
    .constdata                               0x0002e270   Section       32  nrf_log_backend_uart.o(.constdata)
    .constdata                               0x0002e290   Section       16  nrf_sdh.o(.constdata)
    sdh_req_observers_array                  0x0002e290   Data          16  nrf_sdh.o(.constdata)
    .constdata                               0x0002e2a0   Section       40  nrf_sdh.o(.constdata)
    sdh_req_observers                        0x0002e2a4   Data          12  nrf_sdh.o(.constdata)
    sdh_state_observers                      0x0002e2b0   Data          12  nrf_sdh.o(.constdata)
    sdh_stack_observers                      0x0002e2bc   Data          12  nrf_sdh.o(.constdata)
    .constdata                               0x0002e2c8   Section       16  nrf_sdh.o(.constdata)
    sdh_state_observers_array                0x0002e2c8   Data          16  nrf_sdh.o(.constdata)
    .constdata                               0x0002e2d8   Section       16  nrf_sdh.o(.constdata)
    sdh_stack_observers_array                0x0002e2d8   Data          16  nrf_sdh.o(.constdata)
    .constdata                               0x0002e2e8   Section       32  nrf_sdh_ble.o(.constdata)
    sdh_ble_observers_array                  0x0002e2e8   Data          32  nrf_sdh_ble.o(.constdata)
    .constdata                               0x0002e308   Section       16  nrf_sdh_ble.o(.constdata)
    sdh_ble_observers                        0x0002e30c   Data          12  nrf_sdh_ble.o(.constdata)
    .constdata                               0x0002e318   Section       16  nrf_sdh_soc.o(.constdata)
    sdh_soc_observers_array                  0x0002e318   Data          16  nrf_sdh_soc.o(.constdata)
    .constdata                               0x0002e328   Section       12  nrf_sdh_soc.o(.constdata)
    sdh_soc_observers                        0x0002e328   Data          12  nrf_sdh_soc.o(.constdata)
    .constdata                               0x0002e334   Section      129  ctype_o.o(.constdata)
    .constdata                               0x0002e3b8   Section        4  ctype_o.o(.constdata)
    table                                    0x0002e3b8   Data           4  ctype_o.o(.constdata)
    .conststring                             0x0002e3bc   Section       19  main.o(.conststring)
    .conststring                             0x0002e3d0   Section      162  nrf_ble_gatt.o(.conststring)
    .conststring                             0x0002e474   Section     1003  nrf_strerror.o(.conststring)
    .conststring                             0x0002e860   Section      102  nrf_log_str_formatter.o(.conststring)
    .conststring                             0x0002e8c8   Section      463  nrf_sdh_ble.o(.conststring)
    .conststrlit                             0x0002ea98   Section       13  nrf_ble_gatt.o(.conststrlit)
    .conststrlit                             0x0002eaa8   Section        8  ble_nus.o(.conststrlit)
    .conststrlit                             0x0002eab0   Section        6  nrf_drv_clock.o(.conststrlit)
    .conststrlit                             0x0002eab8   Section        6  nrfx_clock.o(.conststrlit)
    .conststrlit                             0x0002eac0   Section        7  nrfx_gpiote.o(.conststrlit)
    .conststrlit                             0x0002eac8   Section        4  nrfx_prs.o(.conststrlit)
    .conststrlit                             0x0002eacc   Section        5  nrfx_uart.o(.conststrlit)
    .conststrlit                             0x0002ead4   Section        6  nrfx_uarte.o(.conststrlit)
    .conststrlit                             0x0002eadc   Section        5  nrfx_spim.o(.conststrlit)
    .conststrlit                             0x0002eae4   Section       11  app_button.o(.conststrlit)
    .conststrlit                             0x0002eaf0   Section       10  app_timer2.o(.conststrlit)
    .conststrlit                             0x0002eafc   Section        9  nrf_pwr_mgmt.o(.conststrlit)
    .conststrlit                             0x0002eb08   Section        9  nrf_sortlist.o(.conststrlit)
    .conststrlit                             0x0002eb14   Section       33  nrf_log_default_backends.o(.conststrlit)
    .conststrlit                             0x0002eb38   Section        4  nrf_log_frontend.o(.conststrlit)
    .conststrlit                             0x0002eb3c   Section        8  nrf_sdh.o(.conststrlit)
    .conststrlit                             0x0002eb44   Section       12  nrf_sdh_ble.o(.conststrlit)
    .conststrlit                             0x0002eb50   Section       12  nrf_sdh_soc.o(.conststrlit)
    log_backends                             0x0002eb7c   Section       32  nrf_log_default_backends.o(log_backends)
    __tagsym$$used                           0x0002eb7c   Number         0  nrf_log_default_backends.o(log_backends)
    rtt_log_backend                          0x0002eb7c   Data          16  nrf_log_default_backends.o(log_backends)
    __tagsym$$used                           0x0002eb8c   Number         0  nrf_log_default_backends.o(log_backends)
    uart_log_backend                         0x0002eb8c   Data          16  nrf_log_default_backends.o(log_backends)
    log_const_data                           0x0002eb9c   Section        8  nrf_ble_gatt.o(log_const_data)
    __tagsym$$used                           0x0002eb9c   Number         0  nrf_ble_gatt.o(log_const_data)
    log_const_data                           0x0002eba4   Section        8  ble_nus.o(log_const_data)
    __tagsym$$used                           0x0002eba4   Number         0  ble_nus.o(log_const_data)
    log_const_data                           0x0002ebac   Section        8  nrf_drv_clock.o(log_const_data)
    __tagsym$$used                           0x0002ebac   Number         0  nrf_drv_clock.o(log_const_data)
    log_const_data                           0x0002ebb4   Section        8  nrfx_clock.o(log_const_data)
    __tagsym$$used                           0x0002ebb4   Number         0  nrfx_clock.o(log_const_data)
    log_const_data                           0x0002ebbc   Section        8  nrfx_gpiote.o(log_const_data)
    __tagsym$$used                           0x0002ebbc   Number         0  nrfx_gpiote.o(log_const_data)
    log_const_data                           0x0002ebc4   Section        8  nrfx_prs.o(log_const_data)
    __tagsym$$used                           0x0002ebc4   Number         0  nrfx_prs.o(log_const_data)
    log_const_data                           0x0002ebcc   Section        8  nrfx_uart.o(log_const_data)
    __tagsym$$used                           0x0002ebcc   Number         0  nrfx_uart.o(log_const_data)
    log_const_data                           0x0002ebd4   Section        8  nrfx_uarte.o(log_const_data)
    __tagsym$$used                           0x0002ebd4   Number         0  nrfx_uarte.o(log_const_data)
    log_const_data                           0x0002ebdc   Section        8  nrfx_spim.o(log_const_data)
    __tagsym$$used                           0x0002ebdc   Number         0  nrfx_spim.o(log_const_data)
    log_const_data                           0x0002ebe4   Section        8  app_button.o(log_const_data)
    __tagsym$$used                           0x0002ebe4   Number         0  app_button.o(log_const_data)
    log_const_data                           0x0002ebec   Section        8  app_timer2.o(log_const_data)
    __tagsym$$used                           0x0002ebec   Number         0  app_timer2.o(log_const_data)
    log_const_data                           0x0002ebf4   Section        8  nrf_pwr_mgmt.o(log_const_data)
    __tagsym$$used                           0x0002ebf4   Number         0  nrf_pwr_mgmt.o(log_const_data)
    log_const_data                           0x0002ebfc   Section        8  nrf_sortlist.o(log_const_data)
    __tagsym$$used                           0x0002ebfc   Number         0  nrf_sortlist.o(log_const_data)
    log_const_data                           0x0002ec04   Section        8  nrf_log_frontend.o(log_const_data)
    __tagsym$$used                           0x0002ec04   Number         0  nrf_log_frontend.o(log_const_data)
    log_const_data                           0x0002ec0c   Section        8  nrf_sdh.o(log_const_data)
    __tagsym$$used                           0x0002ec0c   Number         0  nrf_sdh.o(log_const_data)
    log_const_data                           0x0002ec14   Section        8  nrf_sdh_ble.o(log_const_data)
    __tagsym$$used                           0x0002ec14   Number         0  nrf_sdh_ble.o(log_const_data)
    log_const_data                           0x0002ec1c   Section        8  nrf_sdh_soc.o(log_const_data)
    __tagsym$$used                           0x0002ec1c   Number         0  nrf_sdh_soc.o(log_const_data)
    nrf_balloc                               0x0002ec24   Section       20  nrf_log_frontend.o(nrf_balloc)
    __tagsym$$used                           0x0002ec24   Number         0  nrf_log_frontend.o(nrf_balloc)
    sdh_ble_observers0                       0x0002ec38   Section        8  ble_conn_state.o(sdh_ble_observers0)
    __tagsym$$used                           0x0002ec38   Number         0  ble_conn_state.o(sdh_ble_observers0)
    m_ble_evt_observer                       0x0002ec38   Data           8  ble_conn_state.o(sdh_ble_observers0)
    sdh_ble_observers1                       0x0002ec40   Section       16  main.o(sdh_ble_observers1)
    __tagsym$$used                           0x0002ec40   Number         0  main.o(sdh_ble_observers1)
    m_gatt_obs                               0x0002ec40   Data           8  main.o(sdh_ble_observers1)
    __tagsym$$used                           0x0002ec48   Number         0  main.o(sdh_ble_observers1)
    m_advertising_ble_obs                    0x0002ec48   Data           8  main.o(sdh_ble_observers1)
    sdh_ble_observers1                       0x0002ec50   Section        8  bsp_btn_ble.o(sdh_ble_observers1)
    __tagsym$$used                           0x0002ec50   Number         0  bsp_btn_ble.o(sdh_ble_observers1)
    m_ble_observer                           0x0002ec50   Data           8  bsp_btn_ble.o(sdh_ble_observers1)
    sdh_ble_observers1                       0x0002ec58   Section        8  ble_conn_params.o(sdh_ble_observers1)
    __tagsym$$used                           0x0002ec58   Number         0  ble_conn_params.o(sdh_ble_observers1)
    m_ble_observer                           0x0002ec58   Data           8  ble_conn_params.o(sdh_ble_observers1)
    sdh_ble_observers2                       0x0002ec60   Section       16  main.o(sdh_ble_observers2)
    __tagsym$$used                           0x0002ec60   Number         0  main.o(sdh_ble_observers2)
    m_nus_obs                                0x0002ec60   Data           8  main.o(sdh_ble_observers2)
    __tagsym$$used                           0x0002ec68   Number         0  main.o(sdh_ble_observers2)
    m_qwr_obs                                0x0002ec68   Data           8  main.o(sdh_ble_observers2)
    sdh_ble_observers3                       0x0002ec70   Section        8  main.o(sdh_ble_observers3)
    __tagsym$$used                           0x0002ec70   Number         0  main.o(sdh_ble_observers3)
    m_ble_observer                           0x0002ec70   Data           8  main.o(sdh_ble_observers3)
    sdh_soc_observers0                       0x0002ec78   Section        8  nrf_drv_clock.o(sdh_soc_observers0)
    __tagsym$$used                           0x0002ec78   Number         0  nrf_drv_clock.o(sdh_soc_observers0)
    m_soc_evt_observer                       0x0002ec78   Data           8  nrf_drv_clock.o(sdh_soc_observers0)
    sdh_stack_observers0                     0x0002ec80   Section        8  nrf_sdh_ble.o(sdh_stack_observers0)
    __tagsym$$used                           0x0002ec80   Number         0  nrf_sdh_ble.o(sdh_stack_observers0)
    m_nrf_sdh_ble_evts_poll                  0x0002ec80   Data           8  nrf_sdh_ble.o(sdh_stack_observers0)
    sdh_stack_observers0                     0x0002ec88   Section        8  nrf_sdh_soc.o(sdh_stack_observers0)
    __tagsym$$used                           0x0002ec88   Number         0  nrf_sdh_soc.o(sdh_stack_observers0)
    m_nrf_sdh_soc_evts_poll                  0x0002ec88   Data           8  nrf_sdh_soc.o(sdh_stack_observers0)
    sdh_state_observers0                     0x0002ec90   Section        8  nrf_drv_clock.o(sdh_state_observers0)
    __tagsym$$used                           0x0002ec90   Number         0  nrf_drv_clock.o(sdh_state_observers0)
    m_sd_state_observer                      0x0002ec90   Data           8  nrf_drv_clock.o(sdh_state_observers0)
    .data                                    0x20002ad8   Section       76  main.o(.data)
    m_conn_handle                            0x20002ae4   Data           2  main.o(.data)
    m_ble_nus_max_data_len                   0x20002ae6   Data           2  main.o(.data)
    m_adv_uuids                              0x20002af0   Data           4  main.o(.data)
    data_buffer                              0x20002af8   Data           4  main.o(.data)
    m_nus                                    0x20002afc   Data          28  main.o(.data)
    drives                                   0x20002b18   Data          12  main.o(.data)
    .data                                    0x20002b24   Section        8  main.o(.data)
    m_nus_link_ctx_storage                   0x20002b24   Data           8  main.o(.data)
    .data                                    0x20002b2c   Section        4  main.o(.data)
    m_nus_link_ctx_storage_ctx_data_pool     0x20002b2c   Data           4  main.o(.data)
    .data                                    0x20002b30   Section       16  bsp.o(.data)
    m_stable_state                           0x20002b30   Data           1  bsp.o(.data)
    m_leds_clear                             0x20002b31   Data           1  bsp.o(.data)
    m_alert_on                               0x20002b32   Data           1  bsp.o(.data)
    current_long_push_pin_no                 0x20002b33   Data           1  bsp.o(.data)
    m_indication_type                        0x20002b34   Data           4  bsp.o(.data)
    m_registered_callback                    0x20002b38   Data           4  bsp.o(.data)
    release_event_at_push                    0x20002b3c   Data           4  bsp.o(.data)
    .data                                    0x20002b40   Section        8  bsp_btn_ble.o(.data)
    m_error_handler                          0x20002b40   Data           4  bsp_btn_ble.o(.data)
    m_num_connections                        0x20002b44   Data           4  bsp_btn_ble.o(.data)
    .data                                    0x20002b48   Section        8  ble_conn_params.o(.data)
    m_preferred_conn_params                  0x20002b48   Data           8  ble_conn_params.o(.data)
    .data                                    0x20002b50   Section       12  nrf_drv_uart.o(.data)
    m_handlers                               0x20002b54   Data           4  nrf_drv_uart.o(.data)
    m_contexts                               0x20002b58   Data           4  nrf_drv_uart.o(.data)
    .data                                    0x20002b5c   Section        8  nrfx_clock.o(.data)
    m_clock_cb                               0x20002b5c   Data           8  nrfx_clock.o(.data)
    .data                                    0x20002b64   Section        8  nrfx_prs.o(.data)
    m_prs_box_4                              0x20002b64   Data           8  nrfx_prs.o(.data)
    .data                                    0x20002b70   Section       32  app_timer2.o(.data)
    m_global_active                          0x20002b70   Data           1  app_timer2.o(.data)
    mp_active_timer                          0x20002b74   Data           4  app_timer2.o(.data)
    m_rtc_inst                               0x20002b78   Data           8  app_timer2.o(.data)
    m_base_counter                           0x20002b80   Data           8  app_timer2.o(.data)
    m_stamp64                                0x20002b88   Data           8  app_timer2.o(.data)
    .data                                    0x20002b90   Section        4  app_timer2.o(.data)
    m_app_timer_sortlist_sortlist_cb         0x20002b90   Data           4  app_timer2.o(.data)
    .data                                    0x20002b94   Section       28  app_uart_fifo.o(.data)
    tx_buffer                                0x20002b94   Data           1  app_uart_fifo.o(.data)
    rx_buffer                                0x20002b95   Data           1  app_uart_fifo.o(.data)
    m_rx_ovf                                 0x20002b96   Data           1  app_uart_fifo.o(.data)
    m_event_handler                          0x20002b98   Data           4  app_uart_fifo.o(.data)
    app_uart_inst                            0x20002b9c   Data          20  app_uart_fifo.o(.data)
    .data                                    0x20002bb0   Section       12  drv_rtc.o(.data)
    m_handlers                               0x20002bb0   Data           4  drv_rtc.o(.data)
    m_cb                                     0x20002bb4   Data           8  drv_rtc.o(.data)
    .data                                    0x20002bbc   Section        8  nrf_block_dev_sdc.o(.data)
    m_last_result                            0x20002bbc   Data           1  nrf_block_dev_sdc.o(.data)
    m_active_sdc_dev                         0x20002bc0   Data           4  nrf_block_dev_sdc.o(.data)
    .data                                    0x20002bc4   Section        1  nrf_log_backend_rtt.o(.data)
    m_host_present                           0x20002bc4   Data           1  nrf_log_backend_rtt.o(.data)
    .data                                    0x20002bc8   Section        8  nrf_log_default_backends.o(.data)
    log_backend_cb_rtt_log_backend           0x20002bc8   Data           8  nrf_log_default_backends.o(.data)
    .data                                    0x20002bd0   Section        8  nrf_log_default_backends.o(.data)
    log_backend_cb_uart_log_backend          0x20002bd0   Data           8  nrf_log_default_backends.o(.data)
    .data                                    0x20002bd8   Section        4  nrf_log_frontend.o(.data)
    m_buffer_mask                            0x20002bd8   Data           4  nrf_log_frontend.o(.data)
    .data                                    0x20002bdc   Section        8  nrf_log_frontend.o(.data)
    log_mempool_nrf_balloc_pool_stack        0x20002bdc   Data           8  nrf_log_frontend.o(.data)
    .data                                    0x20002be4   Section        8  nrf_log_frontend.o(.data)
    log_mempool_nrf_balloc_cb                0x20002be4   Data           8  nrf_log_frontend.o(.data)
    .data                                    0x20002bec   Section       64  nrf_log_str_formatter.o(.data)
    m_freq                                   0x20002bec   Data           4  nrf_log_str_formatter.o(.data)
    m_timestamp_div                          0x20002bf0   Data           4  nrf_log_str_formatter.o(.data)
    severity_names                           0x20002bf4   Data          20  nrf_log_str_formatter.o(.data)
    m_colors                                 0x20002c08   Data          36  nrf_log_str_formatter.o(.data)
    .data                                    0x20002c2c   Section       24  nrf_log_backend_uart.o(.data)
    m_xfer_done                              0x20002c2c   Data           1  nrf_log_backend_uart.o(.data)
    m_async_mode                             0x20002c2d   Data           1  nrf_log_backend_uart.o(.data)
    .data                                    0x20002c44   Section        3  nrf_sdh.o(.data)
    m_nrf_sdh_enabled                        0x20002c44   Data           1  nrf_sdh.o(.data)
    m_nrf_sdh_suspended                      0x20002c45   Data           1  nrf_sdh.o(.data)
    m_nrf_sdh_continue                       0x20002c46   Data           1  nrf_sdh.o(.data)
    .data                                    0x20002c47   Section        1  nrf_sdh_ble.o(.data)
    m_stack_is_enabled                       0x20002c47   Data           1  nrf_sdh_ble.o(.data)
    .data                                    0x20002c48   Section        8  diskio_blkdev.o(.data)
    m_drives_count                           0x20002c48   Data           1  diskio_blkdev.o(.data)
    m_drives                                 0x20002c4c   Data           4  diskio_blkdev.o(.data)
    .data                                    0x20002c50   Section        8  ff.o(.data)
    Fsid                                     0x20002c50   Data           2  ff.o(.data)
    FatFs                                    0x20002c54   Data           4  ff.o(.data)
    .data                                    0x20002c58   Section        4  system_nrf52.o(.data)
    __tagsym$$used                           0x20002c58   Number         0  system_nrf52.o(.data)
    .bss                                     0x20002c5c   Section     6800  main.o(.bss)
    fs                                       0x20002c5c   Data         560  main.o(.bss)
    dir                                      0x20002e8c   Data          44  main.o(.bss)
    file1                                    0x20002eb8   Data         552  main.o(.bss)
    file2                                    0x200030e0   Data         552  main.o(.bss)
    m_qwr                                    0x200042ac   Data          12  main.o(.bss)
    m_advertising                            0x200042b8   Data        1076  main.o(.bss)
    .bss                                     0x200046ec   Section       20  main.o(.bss)
    m_gatt                                   0x200046ec   Data          20  main.o(.bss)
    .bss                                     0x20004700   Section       28  main.o(.bss)
    m_block_dev_sdc_work                     0x20004700   Data          28  main.o(.bss)
    .bss                                     0x20004720   Section       32  bsp.o(.bss)
    m_bsp_leds_tmr_data                      0x20004720   Data          32  bsp.o(.bss)
    .bss                                     0x20004740   Section       32  bsp.o(.bss)
    m_bsp_alert_tmr_data                     0x20004740   Data          32  bsp.o(.bss)
    .bss                                     0x20004760   Section       12  bsp.o(.bss)
    m_events_list                            0x20004760   Data          12  bsp.o(.bss)
    .bss                                     0x20004770   Section       32  bsp.o(.bss)
    m_bsp_button_tmr_data                    0x20004770   Data          32  bsp.o(.bss)
    .bss                                     0x20004790   Section       80  ble_conn_params.o(.bss)
    m_timer_data                             0x20004790   Data          32  ble_conn_params.o(.bss)
    m_conn_params_instances                  0x200047b0   Data          20  ble_conn_params.o(.bss)
    m_conn_params_config                     0x200047c4   Data          28  ble_conn_params.o(.bss)
    .bss                                     0x200047e0   Section      124  ble_conn_state.o(.bss)
    m_bcs                                    0x200047e0   Data         124  ble_conn_state.o(.bss)
    .bss                                     0x2000485c   Section       20  nrf_drv_clock.o(.bss)
    m_clock_cb                               0x2000485c   Data          20  nrf_drv_clock.o(.bss)
    .bss                                     0x20004870   Section       92  nrfx_gpiote.o(.bss)
    m_cb                                     0x20004870   Data          92  nrfx_gpiote.o(.bss)
    .bss                                     0x200048cc   Section       44  nrfx_uart.o(.bss)
    m_cb                                     0x200048cc   Data          44  nrfx_uart.o(.bss)
    .bss                                     0x200048f8   Section       36  nrfx_uarte.o(.bss)
    m_cb                                     0x200048f8   Data          36  nrfx_uarte.o(.bss)
    .bss                                     0x2000491c   Section       24  nrf_drv_spi.o(.bss)
    m_handlers                               0x2000491c   Data          12  nrf_drv_spi.o(.bss)
    m_contexts                               0x20004928   Data          12  nrf_drv_spi.o(.bss)
    .bss                                     0x20004934   Section       36  nrfx_spim.o(.bss)
    m_cb                                     0x20004934   Data          36  nrfx_spim.o(.bss)
    .bss                                     0x20004958   Section       16  app_timer2.o(.bss)
    m_req_fifo_inst                          0x20004958   Data          16  app_timer2.o(.bss)
    .bss                                     0x20004968   Section       88  app_timer2.o(.bss)
    m_req_fifo_data                          0x20004968   Data          88  app_timer2.o(.bss)
    .bss                                     0x200049c0   Section       32  app_uart_fifo.o(.bss)
    m_rx_fifo                                0x200049c0   Data          16  app_uart_fifo.o(.bss)
    m_tx_fifo                                0x200049d0   Data          16  app_uart_fifo.o(.bss)
    .bss                                     0x200049e0   Section       12  app_util_platform.o(.bss)
    .bss                                     0x200049ec   Section       92  app_sdcard.o(.bss)
    m_cb                                     0x200049ec   Data          92  app_sdcard.o(.bss)
    .bss                                     0x20004a48   Section       64  nrf_log_backend_rtt.o(.bss)
    m_string_buff                            0x20004a48   Data          64  nrf_log_backend_rtt.o(.bss)
    .bss                                     0x20004a88   Section      192  nrf_log_frontend.o(.bss)
    log_mempool_nrf_balloc_pool_mem          0x20004a88   Data         192  nrf_log_frontend.o(.bss)
    .bss                                     0x20004b48   Section      128  nrf_log_frontend.o(.bss)
    m_log_push_ringbuf_buf                   0x20004b48   Data         128  nrf_log_frontend.o(.bss)
    .bss                                     0x20004bc8   Section       24  nrf_log_frontend.o(.bss)
    m_log_push_ringbuf_cb                    0x20004bc8   Data          24  nrf_log_frontend.o(.bss)
    .bss                                     0x20004be0   Section     1056  nrf_log_frontend.o(.bss)
    m_log_data                               0x20004be0   Data        1056  nrf_log_frontend.o(.bss)
    .bss                                     0x20005000   Section       64  nrf_log_backend_uart.o(.bss)
    m_string_buff                            0x20005000   Data          64  nrf_log_backend_uart.o(.bss)
    .bss                                     0x20005040   Section      648  segger_rtt.o(.bss)
    _acUpBuffer                              0x200050b8   Data         512  segger_rtt.o(.bss)
    _acDownBuffer                            0x200052b8   Data          16  segger_rtt.o(.bss)
    STACK                                    0x200052c8   Section     8192  arm_startup_nrf52.o(STACK)

    Global Symbols

    Symbol Name                              Value     Ov Type        Size  Object(Section)

    BuildAttributes$$THM_ISAv4$E$P$D$K$B$S$7EM$VFPi3$EXTD16$VFPS$VFMA$PE$A:L22UL41UL21$X:L11$S22US41US21$IEEE1$IW$USESV6$~STKCKD$USESV7$~SHL$OSPACE$ROPI$EBA8$MICROLIB$REQ8$EABIv2 0x00000000   Number         0  anon$$obj.o ABSOLUTE
    __ARM_use_no_argv                        0x00000000   Number         0  main.o ABSOLUTE
    _printf_a                                0x00000000   Number         0  stubs.o ABSOLUTE
    _printf_c                                0x00000000   Number         0  stubs.o ABSOLUTE
    _printf_charcount                        0x00000000   Number         0  stubs.o ABSOLUTE
    _printf_d                                0x00000000   Number         0  stubs.o ABSOLUTE
    _printf_e                                0x00000000   Number         0  stubs.o ABSOLUTE
    _printf_f                                0x00000000   Number         0  stubs.o ABSOLUTE
    _printf_flags                            0x00000000   Number         0  stubs.o ABSOLUTE
    _printf_fp_dec                           0x00000000   Number         0  stubs.o ABSOLUTE
    _printf_fp_hex                           0x00000000   Number         0  stubs.o ABSOLUTE
    _printf_g                                0x00000000   Number         0  stubs.o ABSOLUTE
    _printf_i                                0x00000000   Number         0  stubs.o ABSOLUTE
    _printf_int_dec                          0x00000000   Number         0  stubs.o ABSOLUTE
    _printf_l                                0x00000000   Number         0  stubs.o ABSOLUTE
    _printf_lc                               0x00000000   Number         0  stubs.o ABSOLUTE
    _printf_ll                               0x00000000   Number         0  stubs.o ABSOLUTE
    _printf_lld                              0x00000000   Number         0  stubs.o ABSOLUTE
    _printf_lli                              0x00000000   Number         0  stubs.o ABSOLUTE
    _printf_llo                              0x00000000   Number         0  stubs.o ABSOLUTE
    _printf_llu                              0x00000000   Number         0  stubs.o ABSOLUTE
    _printf_llx                              0x00000000   Number         0  stubs.o ABSOLUTE
    _printf_longlong_dec                     0x00000000   Number         0  stubs.o ABSOLUTE
    _printf_longlong_hex                     0x00000000   Number         0  stubs.o ABSOLUTE
    _printf_longlong_oct                     0x00000000   Number         0  stubs.o ABSOLUTE
    _printf_ls                               0x00000000   Number         0  stubs.o ABSOLUTE
    _printf_mbtowc                           0x00000000   Number         0  stubs.o ABSOLUTE
    _printf_n                                0x00000000   Number         0  stubs.o ABSOLUTE
    _printf_o                                0x00000000   Number         0  stubs.o ABSOLUTE
    _printf_p                                0x00000000   Number         0  stubs.o ABSOLUTE
    _printf_percent                          0x00000000   Number         0  stubs.o ABSOLUTE
    _printf_pre_padding                      0x00000000   Number         0  stubs.o ABSOLUTE
    _printf_return_value                     0x00000000   Number         0  stubs.o ABSOLUTE
    _printf_s                                0x00000000   Number         0  stubs.o ABSOLUTE
    _printf_sizespec                         0x00000000   Number         0  stubs.o ABSOLUTE
    _printf_str                              0x00000000   Number         0  stubs.o ABSOLUTE
    _printf_truncate_signed                  0x00000000   Number         0  stubs.o ABSOLUTE
    _printf_truncate_unsigned                0x00000000   Number         0  stubs.o ABSOLUTE
    _printf_u                                0x00000000   Number         0  stubs.o ABSOLUTE
    _printf_wc                               0x00000000   Number         0  stubs.o ABSOLUTE
    _printf_wctomb                           0x00000000   Number         0  stubs.o ABSOLUTE
    _printf_widthprec                        0x00000000   Number         0  stubs.o ABSOLUTE
    _printf_x                                0x00000000   Number         0  stubs.o ABSOLUTE
    __cpp_initialize__aeabi_                  - Undefined Weak Reference
    __cxa_finalize                            - Undefined Weak Reference
    _clock_init                               - Undefined Weak Reference
    _microlib_exit                            - Undefined Weak Reference
    log_dynamic_data$$Base                    - Undefined Reference
    pwr_mgmt_data0$$Base                      - Undefined Reference
    pwr_mgmt_data0$$Limit                     - Undefined Reference
    pwr_mgmt_data1$$Base                      - Undefined Reference
    pwr_mgmt_data1$$Limit                     - Undefined Reference
    pwr_mgmt_data2$$Base                      - Undefined Reference
    pwr_mgmt_data2$$Limit                     - Undefined Reference
    sdh_req_observers0$$Base                  - Undefined Reference
    sdh_req_observers0$$Limit                 - Undefined Reference
    sdh_req_observers1$$Base                  - Undefined Reference
    sdh_req_observers1$$Limit                 - Undefined Reference
    sdh_soc_observers1$$Base                  - Undefined Reference
    sdh_soc_observers1$$Limit                 - Undefined Reference
    sdh_stack_observers1$$Base                - Undefined Reference
    sdh_stack_observers1$$Limit               - Undefined Reference
    sdh_state_observers1$$Base                - Undefined Reference
    sdh_state_observers1$$Limit               - Undefined Reference
    __Vectors_Size                           0x00000200   Number         0  arm_startup_nrf52.o ABSOLUTE
    __Vectors                                0x00026000   Data           4  arm_startup_nrf52.o(RESET)
    __Vectors_End                            0x00026200   Data           0  arm_startup_nrf52.o(RESET)
    __main                                   0x00026201   Thumb Code     0  entry.o(.ARM.Collect$$$$00000000)
    _main_stk                                0x00026201   Thumb Code     0  entry2.o(.ARM.Collect$$$$00000001)
    _main_scatterload                        0x00026205   Thumb Code     0  entry5.o(.ARM.Collect$$$$00000004)
    __main_after_scatterload                 0x00026209   Thumb Code     0  entry5.o(.ARM.Collect$$$$00000004)
    _main_clock                              0x00026209   Thumb Code     0  entry7b.o(.ARM.Collect$$$$00000008)
    _main_cpp_init                           0x00026209   Thumb Code     0  entry8b.o(.ARM.Collect$$$$0000000A)
    _main_init                               0x00026209   Thumb Code     0  entry9a.o(.ARM.Collect$$$$0000000B)
    __rt_final_cpp                           0x00026211   Thumb Code     0  entry10a.o(.ARM.Collect$$$$0000000D)
    __rt_final_exit                          0x00026211   Thumb Code     0  entry11a.o(.ARM.Collect$$$$0000000F)
    __asm___12_nrf_atfifo_c_51f461e1__nrf_atfifo_wspace_req 0x00026215   Thumb Code    56  nrf_atfifo.o(.emb_text)
    __asm___12_nrf_atfifo_c_51f461e1__nrf_atfifo_wspace_close 0x0002624d   Thumb Code    18  nrf_atfifo.o(.emb_text)
    __asm___12_nrf_atfifo_c_51f461e1__nrf_atfifo_rspace_req 0x0002625f   Thumb Code    58  nrf_atfifo.o(.emb_text)
    __asm___12_nrf_atfifo_c_51f461e1__nrf_atfifo_rspace_close 0x00026299   Thumb Code    18  nrf_atfifo.o(.emb_text)
    __asm___12_nrf_atfifo_c_51f461e1__nrf_atfifo_space_clear 0x000262ab   Thumb Code    50  nrf_atfifo.o(.emb_text)
    __asm___12_nrf_atomic_c_85ca2469__nrf_atomic_internal_mov 0x000262dd   Thumb Code    24  nrf_atomic.o(.emb_text)
    __asm___12_nrf_atomic_c_85ca2469__nrf_atomic_internal_orr 0x000262f5   Thumb Code    26  nrf_atomic.o(.emb_text)
    __asm___12_nrf_atomic_c_85ca2469__nrf_atomic_internal_and 0x0002630f   Thumb Code    26  nrf_atomic.o(.emb_text)
    __asm___12_nrf_atomic_c_85ca2469__nrf_atomic_internal_eor 0x00026329   Thumb Code    26  nrf_atomic.o(.emb_text)
    __asm___12_nrf_atomic_c_85ca2469__nrf_atomic_internal_add 0x00026343   Thumb Code    26  nrf_atomic.o(.emb_text)
    __asm___12_nrf_atomic_c_85ca2469__nrf_atomic_internal_sub 0x0002635d   Thumb Code    26  nrf_atomic.o(.emb_text)
    __asm___12_nrf_atomic_c_85ca2469__nrf_atomic_internal_cmp_exch 0x00026377   Thumb Code    42  nrf_atomic.o(.emb_text)
    __asm___12_nrf_atomic_c_85ca2469__nrf_atomic_internal_sub_hs 0x000263a1   Thumb Code    30  nrf_atomic.o(.emb_text)
    Reset_Handler                            0x000263c1   Thumb Code     8  arm_startup_nrf52.o(.text)
    NMI_Handler                              0x000263c9   Thumb Code     2  arm_startup_nrf52.o(.text)
    HardFault_Handler                        0x000263cb   Thumb Code     2  arm_startup_nrf52.o(.text)
    MemoryManagement_Handler                 0x000263cd   Thumb Code     2  arm_startup_nrf52.o(.text)
    BusFault_Handler                         0x000263cf   Thumb Code     2  arm_startup_nrf52.o(.text)
    UsageFault_Handler                       0x000263d1   Thumb Code     2  arm_startup_nrf52.o(.text)
    SVC_Handler                              0x000263d3   Thumb Code     2  arm_startup_nrf52.o(.text)
    DebugMon_Handler                         0x000263d5   Thumb Code     2  arm_startup_nrf52.o(.text)
    PendSV_Handler                           0x000263d7   Thumb Code     2  arm_startup_nrf52.o(.text)
    CCM_AAR_IRQHandler                       0x000263db   Thumb Code     0  arm_startup_nrf52.o(.text)
    COMP_LPCOMP_IRQHandler                   0x000263db   Thumb Code     0  arm_startup_nrf52.o(.text)
    ECB_IRQHandler                           0x000263db   Thumb Code     0  arm_startup_nrf52.o(.text)
    FPU_IRQHandler                           0x000263db   Thumb Code     0  arm_startup_nrf52.o(.text)
    I2S_IRQHandler                           0x000263db   Thumb Code     0  arm_startup_nrf52.o(.text)
    MWU_IRQHandler                           0x000263db   Thumb Code     0  arm_startup_nrf52.o(.text)
    NFCT_IRQHandler                          0x000263db   Thumb Code     0  arm_startup_nrf52.o(.text)
    PDM_IRQHandler                           0x000263db   Thumb Code     0  arm_startup_nrf52.o(.text)
    PWM0_IRQHandler                          0x000263db   Thumb Code     0  arm_startup_nrf52.o(.text)
    PWM1_IRQHandler                          0x000263db   Thumb Code     0  arm_startup_nrf52.o(.text)
    PWM2_IRQHandler                          0x000263db   Thumb Code     0  arm_startup_nrf52.o(.text)
    QDEC_IRQHandler                          0x000263db   Thumb Code     0  arm_startup_nrf52.o(.text)
    RADIO_IRQHandler                         0x000263db   Thumb Code     0  arm_startup_nrf52.o(.text)
    RNG_IRQHandler                           0x000263db   Thumb Code     0  arm_startup_nrf52.o(.text)
    RTC0_IRQHandler                          0x000263db   Thumb Code     0  arm_startup_nrf52.o(.text)
    RTC2_IRQHandler                          0x000263db   Thumb Code     0  arm_startup_nrf52.o(.text)
    SAADC_IRQHandler                         0x000263db   Thumb Code     0  arm_startup_nrf52.o(.text)
    SPIM1_SPIS1_TWIM1_TWIS1_SPI1_TWI1_IRQHandler 0x000263db   Thumb Code     0  arm_startup_nrf52.o(.text)
    SPIM2_SPIS2_SPI2_IRQHandler              0x000263db   Thumb Code     0  arm_startup_nrf52.o(.text)
    SWI0_EGU0_IRQHandler                     0x000263db   Thumb Code     0  arm_startup_nrf52.o(.text)
    SWI1_EGU1_IRQHandler                     0x000263db   Thumb Code     0  arm_startup_nrf52.o(.text)
    SWI3_EGU3_IRQHandler                     0x000263db   Thumb Code     0  arm_startup_nrf52.o(.text)
    SWI4_EGU4_IRQHandler                     0x000263db   Thumb Code     0  arm_startup_nrf52.o(.text)
    SWI5_EGU5_IRQHandler                     0x000263db   Thumb Code     0  arm_startup_nrf52.o(.text)
    TEMP_IRQHandler                          0x000263db   Thumb Code     0  arm_startup_nrf52.o(.text)
    TIMER0_IRQHandler                        0x000263db   Thumb Code     0  arm_startup_nrf52.o(.text)
    TIMER1_IRQHandler                        0x000263db   Thumb Code     0  arm_startup_nrf52.o(.text)
    TIMER3_IRQHandler                        0x000263db   Thumb Code     0  arm_startup_nrf52.o(.text)
    TIMER4_IRQHandler                        0x000263db   Thumb Code     0  arm_startup_nrf52.o(.text)
    WDT_IRQHandler                           0x000263db   Thumb Code     0  arm_startup_nrf52.o(.text)
    __aeabi_uldivmod                         0x000263e5   Thumb Code    98  uldiv.o(.text)
    __aeabi_llsl                             0x00026447   Thumb Code    30  llshl.o(.text)
    _ll_shift_l                              0x00026447   Thumb Code     0  llshl.o(.text)
    __rt_ctype_table                         0x00026465   Thumb Code     4  ctype_o.o(.text)
    __aeabi_memcpy                           0x0002646d   Thumb Code    36  memcpya.o(.text)
    __aeabi_memcpy4                          0x0002646d   Thumb Code     0  memcpya.o(.text)
    __aeabi_memcpy8                          0x0002646d   Thumb Code     0  memcpya.o(.text)
    __aeabi_memset                           0x00026491   Thumb Code    14  memseta.o(.text)
    __aeabi_memset4                          0x00026491   Thumb Code     0  memseta.o(.text)
    __aeabi_memset8                          0x00026491   Thumb Code     0  memseta.o(.text)
    __aeabi_memclr                           0x0002649f   Thumb Code     4  memseta.o(.text)
    __aeabi_memclr4                          0x0002649f   Thumb Code     0  memseta.o(.text)
    __aeabi_memclr8                          0x0002649f   Thumb Code     0  memseta.o(.text)
    _memset$wrapper                          0x000264a3   Thumb Code    18  memseta.o(.text)
    strlen                                   0x000264b5   Thumb Code    14  strlen.o(.text)
    strcpy                                   0x000264c3   Thumb Code    18  strcpy.o(.text)
    __aeabi_uidiv                            0x000264d5   Thumb Code     0  uidiv.o(.text)
    __aeabi_uidivmod                         0x000264d5   Thumb Code    44  uidiv.o(.text)
    __aeabi_llsr                             0x00026501   Thumb Code    32  llushr.o(.text)
    _ll_ushift_r                             0x00026501   Thumb Code     0  llushr.o(.text)
    __scatterload                            0x00026521   Thumb Code    28  init.o(.text)
    __scatterload_rt2                        0x00026521   Thumb Code     0  init.o(.text)
    __decompress                             0x00026545   Thumb Code     0  __dczerorl2.o(.text)
    __decompress1                            0x00026545   Thumb Code    86  __dczerorl2.o(.text)
    Button_state                             0x0002659d   Thumb Code   146  main.o(i.Button_state)
    GPIOTE_IRQHandler                        0x00026665   Thumb Code   154  nrfx_gpiote.o(i.GPIOTE_IRQHandler)
    POWER_CLOCK_IRQHandler                   0x00026709   Thumb Code    82  nrfx_clock.o(i.POWER_CLOCK_IRQHandler)
    RTC1_IRQHandler                          0x00026761   Thumb Code    12  drv_rtc.o(i.RTC1_IRQHandler)
    SEGGER_RTT_Init                          0x00026771   Thumb Code     4  segger_rtt.o(i.SEGGER_RTT_Init)
    SEGGER_RTT_WriteNoLock                   0x00026775   Thumb Code    86  segger_rtt.o(i.SEGGER_RTT_WriteNoLock)
    SPIM0_SPIS0_TWIM0_TWIS0_SPI0_TWI0_IRQHandler 0x000267d1   Thumb Code    76  nrfx_spim.o(i.SPIM0_SPIS0_TWIM0_TWIS0_SPI0_TWI0_IRQHandler)
    SWI2_EGU2_IRQHandler                     0x00026825   Thumb Code     4  nrf_sdh.o(i.SWI2_EGU2_IRQHandler)
    SysTick_Handler                          0x00026829   Thumb Code    10  main.o(i.SysTick_Handler)
    SystemInit                               0x00026839   Thumb Code   112  system_nrf52.o(i.SystemInit)
    TIMER2_IRQHandler                        0x000268bd   Thumb Code   188  main.o(i.TIMER2_IRQHandler)
    UARTE0_UART0_IRQHandler                  0x00026991   Thumb Code     6  nrfx_prs.o(i.UARTE0_UART0_IRQHandler)
    __0sprintf$1                             0x00026ab9   Thumb Code    34  printf1.o(i.__0sprintf$1)
    __1sprintf$1                             0x00026ab9   Thumb Code     0  printf1.o(i.__0sprintf$1)
    __2sprintf                               0x00026ab9   Thumb Code     0  printf1.o(i.__0sprintf$1)
    __scatterload_copy                       0x00026b01   Thumb Code    14  handlers.o(i.__scatterload_copy)
    __scatterload_null                       0x00026b0f   Thumb Code     2  handlers.o(i.__scatterload_null)
    __scatterload_zeroinit                   0x00026b11   Thumb Code    14  handlers.o(i.__scatterload_zeroinit)
    app_error_fault_handler                  0x00026ce9   Thumb Code    86  app_error_weak.o(i.app_error_fault_handler)
    app_error_handler_bare                   0x00026d6d   Thumb Code    22  app_error.o(i.app_error_handler_bare)
    app_fifo_get                             0x00026d83   Thumb Code    22  app_fifo.o(i.app_fifo_get)
    app_fifo_put                             0x00026d99   Thumb Code    26  app_fifo.o(i.app_fifo_put)
    app_sdc_block_read                       0x00026db5   Thumb Code    84  app_sdcard.o(i.app_sdc_block_read)
    app_sdc_block_write                      0x00026e0d   Thumb Code   104  app_sdcard.o(i.app_sdc_block_write)
    app_sdc_busy_check                       0x00026e79   Thumb Code    24  app_sdcard.o(i.app_sdc_busy_check)
    app_sdc_info_get                         0x00026e95   Thumb Code    18  app_sdcard.o(i.app_sdc_info_get)
    app_sdc_init                             0x00026ead   Thumb Code   190  app_sdcard.o(i.app_sdc_init)
    app_sdc_uninit                           0x00026f79   Thumb Code    62  app_sdcard.o(i.app_sdc_uninit)
    app_timer_cnt_get                        0x00026fc1   Thumb Code     6  app_timer2.o(i.app_timer_cnt_get)
    app_timer_init                           0x00026fcd   Thumb Code    70  app_timer2.o(i.app_timer_init)
    app_timer_start                          0x00027029   Thumb Code    48  app_timer2.o(i.app_timer_start)
    app_timer_stop                           0x00027059   Thumb Code    12  app_timer2.o(i.app_timer_stop)
    app_uart_put                             0x00027065   Thumb Code    70  app_uart_fifo.o(i.app_uart_put)
    app_util_critical_region_enter           0x000270b9   Thumb Code    64  app_util_platform.o(i.app_util_critical_region_enter)
    app_util_critical_region_exit            0x00027101   Thumb Code    46  app_util_platform.o(i.app_util_critical_region_exit)
    blcm_link_ctx_get                        0x00027245   Thumb Code    72  ble_link_ctx_manager.o(i.blcm_link_ctx_get)
    ble_advdata_encode                       0x0002728d   Thumb Code   386  ble_advdata.o(i.ble_advdata_encode)
    ble_advdata_parse                        0x0002740f   Thumb Code    32  ble_advdata.o(i.ble_advdata_parse)
    ble_advdata_search                       0x0002742f   Thumb Code    70  ble_advdata.o(i.ble_advdata_search)
    ble_advertising_conn_cfg_tag_set         0x00027475   Thumb Code     6  ble_advertising.o(i.ble_advertising_conn_cfg_tag_set)
    ble_advertising_init                     0x0002747b   Thumb Code   248  ble_advertising.o(i.ble_advertising_init)
    ble_advertising_on_ble_evt               0x00027573   Thumb Code   106  ble_advertising.o(i.ble_advertising_on_ble_evt)
    ble_advertising_start                    0x000275dd   Thumb Code   560  ble_advertising.o(i.ble_advertising_start)
    ble_conn_state_conn_idx                  0x0002780d   Thumb Code    18  ble_conn_state.o(i.ble_conn_state_conn_idx)
    ble_conn_state_valid                     0x00027821   Thumb Code    16  ble_conn_state.o(i.ble_conn_state_valid)
    ble_nus_init                             0x00027bf5   Thumb Code   206  ble_nus.o(i.ble_nus_init)
    ble_nus_on_ble_evt                       0x00027cc9   Thumb Code   118  ble_nus.o(i.ble_nus_on_ble_evt)
    ble_srv_is_notification_enabled          0x00027d3f   Thumb Code     8  ble_srv_common.o(i.ble_srv_is_notification_enabled)
    bsp_board_button_idx_to_pin              0x00027f59   Thumb Code     6  boards.o(i.bsp_board_button_idx_to_pin)
    bsp_board_led_invert                     0x00027f65   Thumb Code    32  boards.o(i.bsp_board_led_invert)
    bsp_board_led_off                        0x00027f89   Thumb Code    10  boards.o(i.bsp_board_led_off)
    bsp_board_led_on                         0x00027f99   Thumb Code    10  boards.o(i.bsp_board_led_on)
    bsp_board_led_state_get                  0x00027fa9   Thumb Code    28  boards.o(i.bsp_board_led_state_get)
    bsp_board_leds_off                       0x00027fc9   Thumb Code    18  boards.o(i.bsp_board_leds_off)
    bsp_board_leds_on                        0x00027fdb   Thumb Code    18  boards.o(i.bsp_board_leds_on)
    bsp_board_pin_to_button_idx              0x00027fed   Thumb Code    30  boards.o(i.bsp_board_pin_to_button_idx)
    bsp_btn_ble_sleep_mode_prepare           0x00028011   Thumb Code    30  bsp_btn_ble.o(i.bsp_btn_ble_sleep_mode_prepare)
    bsp_event_to_button_action_assign        0x000280c1   Thumb Code    64  bsp.o(i.bsp_event_to_button_action_assign)
    bsp_indication_set                       0x00028105   Thumb Code    20  bsp.o(i.bsp_indication_set)
    bsp_wakeup_button_enable                 0x000282e5   Thumb Code     6  bsp.o(i.bsp_wakeup_button_enable)
    buffer_is_empty                          0x000283b1   Thumb Code    18  nrf_log_frontend.o(i.buffer_is_empty)
    characteristic_add                       0x000283d9   Thumb Code   400  ble_srv_common.o(i.characteristic_add)
    conn_handle_list_get                     0x0002864d   Thumb Code    62  ble_conn_state.o(i.conn_handle_list_get)
    disk_initialize                          0x00028be9   Thumb Code   114  diskio_blkdev.o(i.disk_initialize)
    disk_ioctl                               0x00028c69   Thumb Code   118  diskio_blkdev.o(i.disk_ioctl)
    disk_read                                0x00028ce5   Thumb Code   120  diskio_blkdev.o(i.disk_read)
    disk_status                              0x00028d61   Thumb Code    26  diskio_blkdev.o(i.disk_status)
    disk_write                               0x00028d81   Thumb Code   130  diskio_blkdev.o(i.disk_write)
    diskio_blockdev_register                 0x00028e09   Thumb Code     8  diskio_blkdev.o(i.diskio_blockdev_register)
    drv_rtc_compare_disable                  0x00028e29   Thumb Code    20  drv_rtc.o(i.drv_rtc_compare_disable)
    drv_rtc_compare_pending                  0x00028e3d   Thumb Code    14  drv_rtc.o(i.drv_rtc_compare_pending)
    drv_rtc_compare_set                      0x00028e4b   Thumb Code    80  drv_rtc.o(i.drv_rtc_compare_set)
    drv_rtc_counter_get                      0x00028e9b   Thumb Code     8  drv_rtc.o(i.drv_rtc_counter_get)
    drv_rtc_init                             0x00028ea5   Thumb Code   148  drv_rtc.o(i.drv_rtc_init)
    drv_rtc_irq_trigger                      0x00028f7d   Thumb Code    30  drv_rtc.o(i.drv_rtc_irq_trigger)
    drv_rtc_overflow_enable                  0x00028f9b   Thumb Code     8  drv_rtc.o(i.drv_rtc_overflow_enable)
    drv_rtc_overflow_pending                 0x00028fa3   Thumb Code     8  drv_rtc.o(i.drv_rtc_overflow_pending)
    drv_rtc_start                            0x00028fab   Thumb Code     8  drv_rtc.o(i.drv_rtc_start)
    drv_rtc_stop                             0x00028fb3   Thumb Code     8  drv_rtc.o(i.drv_rtc_stop)
    drv_rtc_windowed_compare_set             0x00028fbb   Thumb Code   222  drv_rtc.o(i.drv_rtc_windowed_compare_set)
    f_close                                  0x000290bf   Thumb Code    30  ff.o(i.f_close)
    f_mount                                  0x000290dd   Thumb Code    72  ff.o(i.f_mount)
    f_open                                   0x00029129   Thumb Code   432  ff.o(i.f_open)
    f_opendir                                0x000292dd   Thumb Code    98  ff.o(i.f_opendir)
    f_sync                                   0x00029341   Thumb Code   138  ff.o(i.f_sync)
    f_write                                  0x000293d1   Thumb Code   382  ff.o(i.f_write)
    main                                     0x00029c85   Thumb Code   326  main.o(i.main)
    nrf_atfifo_init                          0x00029ff1   Thumb Code    38  nrf_atfifo.o(i.nrf_atfifo_init)
    nrf_atfifo_item_alloc                    0x0002a017   Thumb Code    22  nrf_atfifo.o(i.nrf_atfifo_item_alloc)
    nrf_atfifo_item_free                     0x0002a02d   Thumb Code    22  nrf_atfifo.o(i.nrf_atfifo_item_free)
    nrf_atfifo_item_get                      0x0002a043   Thumb Code    22  nrf_atfifo.o(i.nrf_atfifo_item_get)
    nrf_atfifo_item_put                      0x0002a059   Thumb Code    22  nrf_atfifo.o(i.nrf_atfifo_item_put)
    nrf_atflags_clear                        0x0002a06f   Thumb Code    22  nrf_atflags.o(i.nrf_atflags_clear)
    nrf_atflags_get                          0x0002a085   Thumb Code    22  nrf_atflags.o(i.nrf_atflags_get)
    nrf_atflags_set                          0x0002a09b   Thumb Code    20  nrf_atflags.o(i.nrf_atflags_set)
    nrf_atomic_flag_clear_fetch              0x0002a0af   Thumb Code     6  nrf_atomic.o(i.nrf_atomic_flag_clear_fetch)
    nrf_atomic_flag_set                      0x0002a0b5   Thumb Code     6  nrf_atomic.o(i.nrf_atomic_flag_set)
    nrf_atomic_u32_add                       0x0002a0bb   Thumb Code    12  nrf_atomic.o(i.nrf_atomic_u32_add)
    nrf_atomic_u32_and                       0x0002a0c7   Thumb Code    12  nrf_atomic.o(i.nrf_atomic_u32_and)
    nrf_atomic_u32_fetch_and                 0x0002a0d3   Thumb Code    10  nrf_atomic.o(i.nrf_atomic_u32_fetch_and)
    nrf_atomic_u32_fetch_store               0x0002a0dd   Thumb Code    10  nrf_atomic.o(i.nrf_atomic_u32_fetch_store)
    nrf_atomic_u32_or                        0x0002a0e7   Thumb Code    12  nrf_atomic.o(i.nrf_atomic_u32_or)
    nrf_atomic_u32_sub                       0x0002a0f3   Thumb Code    12  nrf_atomic.o(i.nrf_atomic_u32_sub)
    nrf_balloc_alloc                         0x0002a0ff   Thumb Code    68  nrf_balloc.o(i.nrf_balloc_alloc)
    nrf_balloc_free                          0x0002a143   Thumb Code    48  nrf_balloc.o(i.nrf_balloc_free)
    nrf_balloc_init                          0x0002a173   Thumb Code    48  nrf_balloc.o(i.nrf_balloc_init)
    nrf_ble_gatt_on_ble_evt                  0x0002a1b5   Thumb Code   270  nrf_ble_gatt.o(i.nrf_ble_gatt_on_ble_evt)
    nrf_ble_qwr_conn_handle_assign           0x0002a305   Thumb Code    22  nrf_ble_qwr.o(i.nrf_ble_qwr_conn_handle_assign)
    nrf_ble_qwr_init                         0x0002a31b   Thumb Code    36  nrf_ble_qwr.o(i.nrf_ble_qwr_init)
    nrf_ble_qwr_on_ble_evt                   0x0002a33f   Thumb Code   182  nrf_ble_qwr.o(i.nrf_ble_qwr_on_ble_evt)
    nrf_drv_clock_init                       0x0002a419   Thumb Code    56  nrf_drv_clock.o(i.nrf_drv_clock_init)
    nrf_drv_clock_lfclk_release              0x0002a459   Thumb Code    48  nrf_drv_clock.o(i.nrf_drv_clock_lfclk_release)
    nrf_drv_spi_init                         0x0002a48d   Thumb Code    98  nrf_drv_spi.o(i.nrf_drv_spi_init)
    nrf_drv_uart_init                        0x0002a515   Thumb Code    90  nrf_drv_uart.o(i.nrf_drv_uart_init)
    nrf_fprintf                              0x0002a59d   Thumb Code    26  nrf_fprintf.o(i.nrf_fprintf)
    nrf_fprintf_buffer_flush                 0x0002a5b7   Thumb Code    24  nrf_fprintf.o(i.nrf_fprintf_buffer_flush)
    nrf_fprintf_fmt                          0x0002a5cf   Thumb Code   474  nrf_fprintf_format.o(i.nrf_fprintf_fmt)
    nrf_log_backend_add                      0x0002a9c5   Thumb Code    86  nrf_log_frontend.o(i.nrf_log_backend_add)
    nrf_log_backend_rtt_init                 0x0002aa23   Thumb Code     4  nrf_log_backend_rtt.o(i.nrf_log_backend_rtt_init)
    nrf_log_backend_serial_put               0x0002aa41   Thumb Code   200  nrf_log_backend_serial.o(i.nrf_log_backend_serial_put)
    nrf_log_backend_uart_init                0x0002ab0b   Thumb Code     6  nrf_log_backend_uart.o(i.nrf_log_backend_uart_init)
    nrf_log_color_id_get                     0x0002ab55   Thumb Code    42  nrf_log_frontend.o(i.nrf_log_color_id_get)
    nrf_log_default_backends_init            0x0002ab85   Thumb Code    46  nrf_log_default_backends.o(i.nrf_log_default_backends_init)
    nrf_log_frontend_dequeue                 0x0002abb9   Thumb Code   528  nrf_log_frontend.o(i.nrf_log_frontend_dequeue)
    nrf_log_frontend_std_0                   0x0002adf1   Thumb Code     8  nrf_log_frontend.o(i.nrf_log_frontend_std_0)
    nrf_log_frontend_std_1                   0x0002adf9   Thumb Code    14  nrf_log_frontend.o(i.nrf_log_frontend_std_1)
    nrf_log_frontend_std_2                   0x0002ae07   Thumb Code    16  nrf_log_frontend.o(i.nrf_log_frontend_std_2)
    nrf_log_hexdump_entry_process            0x0002ae19   Thumb Code   150  nrf_log_str_formatter.o(i.nrf_log_hexdump_entry_process)
    nrf_log_init                             0x0002aec9   Thumb Code    28  nrf_log_frontend.o(i.nrf_log_init)
    nrf_log_module_cnt_get                   0x0002aef1   Thumb Code    10  nrf_log_frontend.o(i.nrf_log_module_cnt_get)
    nrf_log_module_name_get                  0x0002af05   Thumb Code    24  nrf_log_frontend.o(i.nrf_log_module_name_get)
    nrf_log_panic                            0x0002af21   Thumb Code    36  nrf_log_frontend.o(i.nrf_log_panic)
    nrf_log_std_entry_process                0x0002af49   Thumb Code   182  nrf_log_str_formatter.o(i.nrf_log_std_entry_process)
    nrf_memobj_alloc                         0x0002afff   Thumb Code    96  nrf_memobj.o(i.nrf_memobj_alloc)
    nrf_memobj_free                          0x0002b05f   Thumb Code    50  nrf_memobj.o(i.nrf_memobj_free)
    nrf_memobj_get                           0x0002b091   Thumb Code     8  nrf_memobj.o(i.nrf_memobj_get)
    nrf_memobj_pool_init                     0x0002b099   Thumb Code     4  nrf_memobj.o(i.nrf_memobj_pool_init)
    nrf_memobj_put                           0x0002b09d   Thumb Code    30  nrf_memobj.o(i.nrf_memobj_put)
    nrf_memobj_read                          0x0002b0bb   Thumb Code    16  nrf_memobj.o(i.nrf_memobj_read)
    nrf_memobj_write                         0x0002b0cb   Thumb Code    16  nrf_memobj.o(i.nrf_memobj_write)
    nrf_ringbuf_init                         0x0002b0df   Thumb Code    28  nrf_ringbuf.o(i.nrf_ringbuf_init)
    nrf_sdh_ble_app_ram_start_get            0x0002b109   Thumb Code    16  nrf_sdh_ble.o(i.nrf_sdh_ble_app_ram_start_get)
    nrf_sdh_ble_default_cfg_set              0x0002b11d   Thumb Code   272  nrf_sdh_ble.o(i.nrf_sdh_ble_default_cfg_set)
    nrf_sdh_ble_enable                       0x0002b24d   Thumb Code   116  nrf_sdh_ble.o(i.nrf_sdh_ble_enable)
    nrf_sdh_enable_request                   0x0002b3dd   Thumb Code   102  nrf_sdh.o(i.nrf_sdh_enable_request)
    nrf_sdh_evts_poll                        0x0002b451   Thumb Code    32  nrf_sdh.o(i.nrf_sdh_evts_poll)
    nrf_sdh_is_enabled                       0x0002b475   Thumb Code     6  nrf_sdh.o(i.nrf_sdh_is_enabled)
    nrf_section_iter_init                    0x0002b4bd   Thumb Code    10  nrf_section_iter.o(i.nrf_section_iter_init)
    nrf_section_iter_next                    0x0002b4eb   Thumb Code    32  nrf_section_iter.o(i.nrf_section_iter_next)
    nrf_sortlist_add                         0x0002b50b   Thumb Code    34  nrf_sortlist.o(i.nrf_sortlist_add)
    nrf_sortlist_peek                        0x0002b52d   Thumb Code     6  nrf_sortlist.o(i.nrf_sortlist_peek)
    nrf_sortlist_pop                         0x0002b533   Thumb Code    14  nrf_sortlist.o(i.nrf_sortlist_pop)
    nrf_sortlist_remove                      0x0002b541   Thumb Code    30  nrf_sortlist.o(i.nrf_sortlist_remove)
    nrf_strerror_find                        0x0002b569   Thumb Code    52  nrf_strerror.o(i.nrf_strerror_find)
    nrf_strerror_get                         0x0002b5a1   Thumb Code    14  nrf_strerror.o(i.nrf_strerror_get)
    nrfx_clock_enable                        0x0002b5fd   Thumb Code    34  nrfx_clock.o(i.nrfx_clock_enable)
    nrfx_clock_init                          0x0002b629   Thumb Code    26  nrfx_clock.o(i.nrfx_clock_init)
    nrfx_clock_lfclk_stop                    0x0002b649   Thumb Code    38  nrfx_clock.o(i.nrfx_clock_lfclk_stop)
    nrfx_prs_acquire                         0x0002b6a9   Thumb Code    58  nrfx_prs.o(i.nrfx_prs_acquire)
    nrfx_prs_release                         0x0002b6e3   Thumb Code    18  nrfx_prs.o(i.nrfx_prs_release)
    nrfx_spim_init                           0x0002b6f5   Thumb Code   356  nrfx_spim.o(i.nrfx_spim_init)
    nrfx_spim_uninit                         0x0002b861   Thumb Code   138  nrfx_spim.o(i.nrfx_spim_uninit)
    nrfx_spim_xfer                           0x0002b8f5   Thumb Code    94  nrfx_spim.o(i.nrfx_spim_xfer)
    nrfx_uart_0_irq_handler                  0x0002b959   Thumb Code     8  nrfx_uart.o(i.nrfx_uart_0_irq_handler)
    nrfx_uart_init                           0x0002b969   Thumb Code   200  nrfx_uart.o(i.nrfx_uart_init)
    nrfx_uart_tx                             0x0002ba3d   Thumb Code   162  nrfx_uart.o(i.nrfx_uart_tx)
    nrfx_uart_tx_in_progress                 0x0002bae5   Thumb Code    26  nrfx_uart.o(i.nrfx_uart_tx_in_progress)
    nrfx_uart_uninit                         0x0002bb05   Thumb Code   182  nrfx_uart.o(i.nrfx_uart_uninit)
    nrfx_uarte_0_irq_handler                 0x0002bbc5   Thumb Code     8  nrfx_uarte.o(i.nrfx_uarte_0_irq_handler)
    nrfx_uarte_init                          0x0002bbd5   Thumb Code   100  nrfx_uarte.o(i.nrfx_uarte_init)
    nrfx_uarte_tx                            0x0002bc41   Thumb Code   166  nrfx_uarte.o(i.nrfx_uarte_tx)
    nrfx_uarte_tx_in_progress                0x0002bced   Thumb Code    22  nrfx_uarte.o(i.nrfx_uarte_tx_in_progress)
    nrfx_uarte_uninit                        0x0002bd09   Thumb Code   254  nrfx_uarte.o(i.nrfx_uarte_uninit)
    nvmc_config                              0x0002bea9   Thumb Code    14  system_nrf52.o(i.nvmc_config)
    saadc_init                               0x0002c5f1   Thumb Code    72  main.o(i.saadc_init)
    saadc_start                              0x0002c645   Thumb Code    30  main.o(i.saadc_start)
    timer_init                               0x0002d941   Thumb Code    64  main.o(i.timer_init)
    nrf_block_device_sdc_ops                 0x0002e1e4   Data          24  nrf_block_dev_sdc.o(.constdata)
    nrf_log_backend_rtt_api                  0x0002e244   Data          12  nrf_log_backend_rtt.o(.constdata)
    nrf_log_backend_uart_api                 0x0002e264   Data          12  nrf_log_backend_uart.o(.constdata)
    m_ram_start                              0x0002e308   Data           4  nrf_sdh_ble.o(.constdata)
    __ctype_table                            0x0002e334   Data         129  ctype_o.o(.constdata)
    Region$$Table$$Base                      0x0002eb5c   Number         0  anon$$obj.o(Region$$Table)
    Region$$Table$$Limit                     0x0002eb7c   Number         0  anon$$obj.o(Region$$Table)
    log_const_data$$Base                     0x0002eb9c   Number         0  nrf_ble_gatt.o(log_const_data)
    m_nrf_log_nrf_ble_gatt_logs_data_const   0x0002eb9c   Data           8  nrf_ble_gatt.o(log_const_data)
    m_nrf_log_ble_nus_logs_data_const        0x0002eba4   Data           8  ble_nus.o(log_const_data)
    m_nrf_log_clock_logs_data_const          0x0002ebac   Data           8  nrf_drv_clock.o(log_const_data)
    m_nrf_log_CLOCK_logs_data_const          0x0002ebb4   Data           8  nrfx_clock.o(log_const_data)
    m_nrf_log_GPIOTE_logs_data_const         0x0002ebbc   Data           8  nrfx_gpiote.o(log_const_data)
    m_nrf_log_PRS_logs_data_const            0x0002ebc4   Data           8  nrfx_prs.o(log_const_data)
    m_nrf_log_UART_logs_data_const           0x0002ebcc   Data           8  nrfx_uart.o(log_const_data)
    m_nrf_log_UARTE_logs_data_const          0x0002ebd4   Data           8  nrfx_uarte.o(log_const_data)
    m_nrf_log_SPIM_logs_data_const           0x0002ebdc   Data           8  nrfx_spim.o(log_const_data)
    m_nrf_log_app_button_logs_data_const     0x0002ebe4   Data           8  app_button.o(log_const_data)
    m_nrf_log_app_timer_logs_data_const      0x0002ebec   Data           8  app_timer2.o(log_const_data)
    m_nrf_log_pwr_mgmt_logs_data_const       0x0002ebf4   Data           8  nrf_pwr_mgmt.o(log_const_data)
    m_nrf_log_sortlist_logs_data_const       0x0002ebfc   Data           8  nrf_sortlist.o(log_const_data)
    m_nrf_log_app_logs_data_const            0x0002ec04   Data           8  nrf_log_frontend.o(log_const_data)
    m_nrf_log_nrf_sdh_logs_data_const        0x0002ec0c   Data           8  nrf_sdh.o(log_const_data)
    m_nrf_log_nrf_sdh_ble_logs_data_const    0x0002ec14   Data           8  nrf_sdh_ble.o(log_const_data)
    m_nrf_log_nrf_sdh_soc_logs_data_const    0x0002ec1c   Data           8  nrf_sdh_soc.o(log_const_data)
    log_const_data$$Limit                    0x0002ec24   Number         0  nrf_sdh_soc.o(log_const_data)
    log_mempool                              0x0002ec24   Data          20  nrf_log_frontend.o(nrf_balloc)
    sdh_ble_observers0$$Base                 0x0002ec38   Number         0  ble_conn_state.o(sdh_ble_observers0)
    sdh_ble_observers0$$Limit                0x0002ec40   Number         0  ble_conn_state.o(sdh_ble_observers0)
    sdh_ble_observers1$$Base                 0x0002ec40   Number         0  main.o(sdh_ble_observers1)
    sdh_ble_observers1$$Limit                0x0002ec60   Number         0  ble_conn_params.o(sdh_ble_observers1)
    sdh_ble_observers2$$Base                 0x0002ec60   Number         0  main.o(sdh_ble_observers2)
    sdh_ble_observers2$$Limit                0x0002ec70   Number         0  main.o(sdh_ble_observers2)
    sdh_ble_observers3$$Base                 0x0002ec70   Number         0  main.o(sdh_ble_observers3)
    sdh_ble_observers3$$Limit                0x0002ec78   Number         0  main.o(sdh_ble_observers3)
    sdh_soc_observers0$$Base                 0x0002ec78   Number         0  nrf_drv_clock.o(sdh_soc_observers0)
    sdh_soc_observers0$$Limit                0x0002ec80   Number         0  nrf_drv_clock.o(sdh_soc_observers0)
    sdh_stack_observers0$$Base               0x0002ec80   Number         0  nrf_sdh_ble.o(sdh_stack_observers0)
    sdh_stack_observers0$$Limit              0x0002ec90   Number         0  nrf_sdh_soc.o(sdh_stack_observers0)
    sdh_state_observers0$$Base               0x0002ec90   Number         0  nrf_drv_clock.o(sdh_state_observers0)
    sdh_state_observers0$$Limit              0x0002ec98   Number         0  nrf_drv_clock.o(sdh_state_observers0)
    Image$$RW_IRAM1$$Base                    0x20002ad8   Number         0  anon$$obj.o ABSOLUTE
    pre_button_state                         0x20002ad8   Data           1  main.o(.data)
    lastAfterFilterNoiseState                0x20002ad9   Data           1  main.o(.data)
    user_info_written                        0x20002ada   Data           1  main.o(.data)
    write_to_sd_card                         0x20002adb   Data           1  main.o(.data)
    current_button_state                     0x20002adc   Data           1  main.o(.data)
    count_button                             0x20002ade   Data           2  main.o(.data)
    count_EMG_data                           0x20002ae0   Data           2  main.o(.data)
    count_battery_data                       0x20002ae2   Data           2  main.o(.data)
    msTicks                                  0x20002ae8   Data           4  main.o(.data)
    count_sample                             0x20002aec   Data           4  main.o(.data)
    lastDebounceTime                         0x20002af4   Data           4  main.o(.data)
    nrf_drv_uart_use_easy_dma                0x20002b50   Data           1  nrf_drv_uart.o(.data)
    m_uart                                   0x20002c30   Data          20  nrf_log_backend_uart.o(.data)
    SystemCoreClock                          0x20002c58   Data           4  system_nrf52.o(.data)
    EMG_data                                 0x20003308   Data        2001  main.o(.bss)
    Battery_data                             0x20003ad9   Data        2001  main.o(.bss)
    nrf_nvic_state                           0x200049e0   Data          12  app_util_platform.o(.bss)
    _SEGGER_RTT                              0x20005040   Data         120  segger_rtt.o(.bss)
    __initial_sp                             0x200072c8   Data           0  arm_startup_nrf52.o(STACK)



==============================================================================

Memory Map of the image

  Image Entry point : 0x00026201

  Load Region LR_IROM1 (Base: 0x00026000, Size: 0x00008e1c, Max: 0x0005a000, ABSOLUTE, COMPRESSED[0x00008cfc])

    Execution Region ER_IROM1 (Exec base: 0x00026000, Load base: 0x00026000, Size: 0x00008c98, Max: 0x0005a000, ABSOLUTE)

    Exec Addr    Load Addr    Size         Type   Attr      Idx    E Section Name        Object

    0x00026000   0x00026000   0x00000200   Data   RO         6308    RESET               arm_startup_nrf52.o
    0x00026200   0x00026200   0x00000000   Code   RO         6374  * .ARM.Collect$$$$00000000  mc_w.l(entry.o)
    0x00026200   0x00026200   0x00000004   Code   RO         6682    .ARM.Collect$$$$00000001  mc_w.l(entry2.o)
    0x00026204   0x00026204   0x00000004   Code   RO         6685    .ARM.Collect$$$$00000004  mc_w.l(entry5.o)
    0x00026208   0x00026208   0x00000000   Code   RO         6687    .ARM.Collect$$$$00000008  mc_w.l(entry7b.o)
    0x00026208   0x00026208   0x00000000   Code   RO         6689    .ARM.Collect$$$$0000000A  mc_w.l(entry8b.o)
    0x00026208   0x00026208   0x00000008   Code   RO         6690    .ARM.Collect$$$$0000000B  mc_w.l(entry9a.o)
    0x00026210   0x00026210   0x00000000   Code   RO         6692    .ARM.Collect$$$$0000000D  mc_w.l(entry10a.o)
    0x00026210   0x00026210   0x00000000   Code   RO         6694    .ARM.Collect$$$$0000000F  mc_w.l(entry11a.o)
    0x00026210   0x00026210   0x00000004   Code   RO         6683    .ARM.Collect$$$$00002712  mc_w.l(entry2.o)
    0x00026214   0x00026214   0x000000c8   Code   RO         4026    .emb_text           nrf_atfifo.o
    0x000262dc   0x000262dc   0x000000e2   Code   RO         4162    .emb_text           nrf_atomic.o
    0x000263be   0x000263be   0x00000002   PAD
    0x000263c0   0x000263c0   0x00000024   Code   RO         6309    .text               arm_startup_nrf52.o
    0x000263e4   0x000263e4   0x00000062   Code   RO         6377    .text               mc_w.l(uldiv.o)
    0x00026446   0x00026446   0x0000001e   Code   RO         6379    .text               mc_w.l(llshl.o)
    0x00026464   0x00026464   0x00000008   Code   RO         6381    .text               mc_w.l(ctype_o.o)
    0x0002646c   0x0002646c   0x00000024   Code   RO         6409    .text               mc_w.l(memcpya.o)
    0x00026490   0x00026490   0x00000024   Code   RO         6411    .text               mc_w.l(memseta.o)
    0x000264b4   0x000264b4   0x0000000e   Code   RO         6413    .text               mc_w.l(strlen.o)
    0x000264c2   0x000264c2   0x00000012   Code   RO         6417    .text               mc_w.l(strcpy.o)
    0x000264d4   0x000264d4   0x0000002c   Code   RO         6696    .text               mc_w.l(uidiv.o)
    0x00026500   0x00026500   0x00000020   Code   RO         6698    .text               mc_w.l(llushr.o)
    0x00026520   0x00026520   0x00000024   Code   RO         6711    .text               mc_w.l(init.o)
    0x00026544   0x00026544   0x00000056   Code   RO         6725    .text               mc_w.l(__dczerorl2.o)
    0x0002659a   0x0002659a   0x00000002   PAD
    0x0002659c   0x0002659c   0x000000c8   Code   RO            4    i.Button_state      main.o
    0x00026664   0x00026664   0x000000a4   Code   RO         2279    i.GPIOTE_IRQHandler  nrfx_gpiote.o
    0x00026708   0x00026708   0x00000058   Code   RO         2140    i.POWER_CLOCK_IRQHandler  nrfx_clock.o
    0x00026760   0x00026760   0x00000010   Code   RO         3812    i.RTC1_IRQHandler   drv_rtc.o
    0x00026770   0x00026770   0x00000004   Code   RO         5457    i.SEGGER_RTT_Init   segger_rtt.o
    0x00026774   0x00026774   0x0000005c   Code   RO         5471    i.SEGGER_RTT_WriteNoLock  segger_rtt.o
    0x000267d0   0x000267d0   0x00000054   Code   RO         3051    i.SPIM0_SPIS0_TWIM0_TWIS0_SPI0_TWI0_IRQHandler  nrfx_spim.o
    0x00026824   0x00026824   0x00000004   Code   RO         5708    i.SWI2_EGU2_IRQHandler  nrf_sdh.o
    0x00026828   0x00026828   0x00000010   Code   RO            6    i.SysTick_Handler   main.o
    0x00026838   0x00026838   0x00000084   Code   RO         6317    i.SystemInit        system_nrf52.o
    0x000268bc   0x000268bc   0x000000d4   Code   RO            7    i.TIMER2_IRQHandler  main.o
    0x00026990   0x00026990   0x0000000c   Code   RO         2584    i.UARTE0_UART0_IRQHandler  nrfx_prs.o
    0x0002699c   0x0002699c   0x00000068   Code   RO         5475    i._DoInit           segger_rtt.o
    0x00026a04   0x00026a04   0x00000016   Code   RO         5476    i._GetAvailWriteSpace  segger_rtt.o
    0x00026a1a   0x00026a1a   0x0000005a   Code   RO         5478    i._WriteBlocking    segger_rtt.o
    0x00026a74   0x00026a74   0x00000042   Code   RO         5479    i._WriteNoCheck     segger_rtt.o
    0x00026ab6   0x00026ab6   0x00000002   PAD
    0x00026ab8   0x00026ab8   0x00000028   Code   RO         6468    i.__0sprintf$1      mc_w.l(printf1.o)
    0x00026ae0   0x00026ae0   0x00000020   Code   RO            8    i.__NVIC_SetPriority  main.o
    0x00026b00   0x00026b00   0x0000000e   Code   RO         6719    i.__scatterload_copy  mc_w.l(handlers.o)
    0x00026b0e   0x00026b0e   0x00000002   Code   RO         6720    i.__scatterload_null  mc_w.l(handlers.o)
    0x00026b10   0x00026b10   0x0000000e   Code   RO         6721    i.__scatterload_zeroinit  mc_w.l(handlers.o)
    0x00026b1e   0x00026b1e   0x00000002   PAD
    0x00026b20   0x00026b20   0x00000024   Code   RO         5709    i.__sd_nvic_app_accessible_irq  nrf_sdh.o
    0x00026b44   0x00026b44   0x00000154   Code   RO         6473    i._printf_core      mc_w.l(printf1.o)
    0x00026c98   0x00026c98   0x0000000a   Code   RO         6475    i._sputc            mc_w.l(printf1.o)
    0x00026ca2   0x00026ca2   0x00000010   Code   RO         1065    i.adv_set_data_size_max_get  ble_advertising.o
    0x00026cb2   0x00026cb2   0x00000036   Code   RO          798    i.advertising_buttons_configure  bsp_btn_ble.o
    0x00026ce8   0x00026ce8   0x00000084   Code   RO         3327    i.app_error_fault_handler  app_error_weak.o
    0x00026d6c   0x00026d6c   0x00000016   Code   RO         3267    i.app_error_handler_bare  app_error.o
    0x00026d82   0x00026d82   0x00000016   Code   RO         3387    i.app_fifo_get      app_fifo.o
    0x00026d98   0x00026d98   0x0000001a   Code   RO         3390    i.app_fifo_put      app_fifo.o
    0x00026db2   0x00026db2   0x00000002   PAD
    0x00026db4   0x00026db4   0x00000058   Code   RO         4793    i.app_sdc_block_read  app_sdcard.o
    0x00026e0c   0x00026e0c   0x0000006c   Code   RO         4794    i.app_sdc_block_write  app_sdcard.o
    0x00026e78   0x00026e78   0x0000001c   Code   RO         4795    i.app_sdc_busy_check  app_sdcard.o
    0x00026e94   0x00026e94   0x00000018   Code   RO         4796    i.app_sdc_info_get  app_sdcard.o
    0x00026eac   0x00026eac   0x000000cc   Code   RO         4797    i.app_sdc_init      app_sdcard.o
    0x00026f78   0x00026f78   0x00000048   Code   RO         4798    i.app_sdc_uninit    app_sdcard.o
    0x00026fc0   0x00026fc0   0x0000000c   Code   RO         3511    i.app_timer_cnt_get  app_timer2.o
    0x00026fcc   0x00026fcc   0x0000005c   Code   RO         3513    i.app_timer_init    app_timer2.o
    0x00027028   0x00027028   0x00000030   Code   RO         3516    i.app_timer_start   app_timer2.o
    0x00027058   0x00027058   0x0000000c   Code   RO         3517    i.app_timer_stop    app_timer2.o
    0x00027064   0x00027064   0x00000054   Code   RO         3656    i.app_uart_put      app_uart_fifo.o
    0x000270b8   0x000270b8   0x00000048   Code   RO         3732    i.app_util_critical_region_enter  app_util_platform.o
    0x00027100   0x00027100   0x00000034   Code   RO         3733    i.app_util_critical_region_exit  app_util_platform.o
    0x00027134   0x00027134   0x00000088   Code   RO         2638    i.apply_config      nrfx_uart.o
    0x000271bc   0x000271bc   0x00000088   Code   RO         2826    i.apply_config      nrfx_uarte.o
    0x00027244   0x00027244   0x00000048   Code   RO         1435    i.blcm_link_ctx_get  ble_link_ctx_manager.o
    0x0002728c   0x0002728c   0x00000182   Code   RO          947    i.ble_advdata_encode  ble_advdata.o
    0x0002740e   0x0002740e   0x00000020   Code   RO          949    i.ble_advdata_parse  ble_advdata.o
    0x0002742e   0x0002742e   0x00000046   Code   RO          950    i.ble_advdata_search  ble_advdata.o
    0x00027474   0x00027474   0x00000006   Code   RO         1067    i.ble_advertising_conn_cfg_tag_set  ble_advertising.o
    0x0002747a   0x0002747a   0x000000f8   Code   RO         1068    i.ble_advertising_init  ble_advertising.o
    0x00027572   0x00027572   0x0000006a   Code   RO         1070    i.ble_advertising_on_ble_evt  ble_advertising.o
    0x000275dc   0x000275dc   0x00000230   Code   RO         1073    i.ble_advertising_start  ble_advertising.o
    0x0002780c   0x0002780c   0x00000012   Code   RO         1267    i.ble_conn_state_conn_idx  ble_conn_state.o
    0x0002781e   0x0002781e   0x00000002   PAD
    0x00027820   0x00027820   0x00000014   Code   RO         1281    i.ble_conn_state_valid  ble_conn_state.o
    0x00027834   0x00027834   0x00000060   Code   RO          953    i.ble_device_addr_encode  ble_advdata.o
    0x00027894   0x00027894   0x000000dc   Code   RO            9    i.ble_evt_handler   main.o
    0x00027970   0x00027970   0x00000070   Code   RO          799    i.ble_evt_handler   bsp_btn_ble.o
    0x000279e0   0x000279e0   0x000000fc   Code   RO         1185    i.ble_evt_handler   ble_conn_params.o
    0x00027adc   0x00027adc   0x00000118   Code   RO         1282    i.ble_evt_handler   ble_conn_state.o
    0x00027bf4   0x00027bf4   0x000000d4   Code   RO         1729    i.ble_nus_init      ble_nus.o
    0x00027cc8   0x00027cc8   0x00000076   Code   RO         1730    i.ble_nus_on_ble_evt  ble_nus.o
    0x00027d3e   0x00027d3e   0x00000008   Code   RO         1464    i.ble_srv_is_notification_enabled  ble_srv_common.o
    0x00027d46   0x00027d46   0x00000002   PAD
    0x00027d48   0x00027d48   0x0000002c   Code   RO         5918    i.block_dev_handler  diskio_blkdev.o
    0x00027d74   0x00027d74   0x00000004   Code   RO         4933    i.block_dev_sdc_geometry  nrf_block_dev_sdc.o
    0x00027d78   0x00027d78   0x00000074   Code   RO         4934    i.block_dev_sdc_init  nrf_block_dev_sdc.o
    0x00027dec   0x00027dec   0x00000020   Code   RO         4935    i.block_dev_sdc_ioctl  nrf_block_dev_sdc.o
    0x00027e0c   0x00027e0c   0x0000007c   Code   RO         4936    i.block_dev_sdc_read_req  nrf_block_dev_sdc.o
    0x00027e88   0x00027e88   0x00000054   Code   RO         4937    i.block_dev_sdc_uninit  nrf_block_dev_sdc.o
    0x00027edc   0x00027edc   0x0000007c   Code   RO         4938    i.block_dev_sdc_write_req  nrf_block_dev_sdc.o
    0x00027f58   0x00027f58   0x0000000c   Code   RO          462    i.bsp_board_button_idx_to_pin  boards.o
    0x00027f64   0x00027f64   0x00000024   Code   RO          466    i.bsp_board_led_invert  boards.o
    0x00027f88   0x00027f88   0x00000010   Code   RO          467    i.bsp_board_led_off  boards.o
    0x00027f98   0x00027f98   0x00000010   Code   RO          468    i.bsp_board_led_on  boards.o
    0x00027fa8   0x00027fa8   0x00000020   Code   RO          469    i.bsp_board_led_state_get  boards.o
    0x00027fc8   0x00027fc8   0x00000012   Code   RO          470    i.bsp_board_leds_off  boards.o
    0x00027fda   0x00027fda   0x00000012   Code   RO          471    i.bsp_board_leds_on  boards.o
    0x00027fec   0x00027fec   0x00000024   Code   RO          472    i.bsp_board_pin_to_button_idx  boards.o
    0x00028010   0x00028010   0x0000001e   Code   RO          801    i.bsp_btn_ble_sleep_mode_prepare  bsp_btn_ble.o
    0x0002802e   0x0002802e   0x00000002   PAD
    0x00028030   0x00028030   0x00000090   Code   RO          663    i.bsp_button_event_handler  bsp.o
    0x000280c0   0x000280c0   0x00000044   Code   RO          667    i.bsp_event_to_button_action_assign  bsp.o
    0x00028104   0x00028104   0x00000018   Code   RO          668    i.bsp_indication_set  bsp.o
    0x0002811c   0x0002811c   0x000001c8   Code   RO          670    i.bsp_led_indication  bsp.o
    0x000282e4   0x000282e4   0x00000006   Code   RO          672    i.bsp_wakeup_button_enable  bsp.o
    0x000282ea   0x000282ea   0x00000002   PAD
    0x000282ec   0x000282ec   0x00000094   Code   RO         5144    i.buf_prealloc      nrf_log_frontend.o
    0x00028380   0x00028380   0x0000002e   Code   RO         4374    i.buffer_add        nrf_fprintf_format.o
    0x000283ae   0x000283ae   0x00000002   PAD
    0x000283b0   0x000283b0   0x00000018   Code   RO         5145    i.buffer_is_empty   nrf_log_frontend.o
    0x000283c8   0x000283c8   0x00000010   Code   RO         2282    i.channel_port_get  nrfx_gpiote.o
    0x000283d8   0x000283d8   0x00000190   Code   RO         1466    i.characteristic_add  ble_srv_common.o
    0x00028568   0x00028568   0x00000070   Code   RO         6004    i.check_fs          ff.o
    0x000285d8   0x000285d8   0x00000028   Code   RO         1789    i.clock_clk_started_notify  nrf_drv_clock.o
    0x00028600   0x00028600   0x0000001c   Code   RO         1790    i.clock_irq_handler  nrf_drv_clock.o
    0x0002861c   0x0002861c   0x00000018   Code   RO         6005    i.clust2sect        ff.o
    0x00028634   0x00028634   0x00000018   Code   RO         3519    i.compare_func      app_timer2.o
    0x0002864c   0x0002864c   0x0000003e   Code   RO         1283    i.conn_handle_list_get  ble_conn_state.o
    0x0002868a   0x0002868a   0x00000088   Code   RO          954    i.conn_int_encode   ble_advdata.o
    0x00028712   0x00028712   0x00000002   PAD
    0x00028714   0x00028714   0x00000048   Code   RO         1186    i.conn_params_negotiation  ble_conn_params.o
    0x0002875c   0x0002875c   0x000000a4   Code   RO         6006    i.create_chain      ff.o
    0x00028800   0x00028800   0x000000e4   Code   RO         6007    i.create_name       ff.o
    0x000288e4   0x000288e4   0x000000c0   Code   RO         1582    i.data_length_update  nrf_ble_gatt.o
    0x000289a4   0x000289a4   0x00000004   Code   RO         5919    i.default_wait_func  diskio_blkdev.o
    0x000289a8   0x000289a8   0x00000064   Code   RO         6008    i.dir_find          ff.o
    0x00028a0c   0x00028a0c   0x000000f4   Code   RO         6009    i.dir_next          ff.o
    0x00028b00   0x00028b00   0x00000066   Code   RO         6011    i.dir_register      ff.o
    0x00028b66   0x00028b66   0x00000082   Code   RO         6013    i.dir_sdi           ff.o
    0x00028be8   0x00028be8   0x00000080   Code   RO         5920    i.disk_initialize   diskio_blkdev.o
    0x00028c68   0x00028c68   0x0000007c   Code   RO         5921    i.disk_ioctl        diskio_blkdev.o
    0x00028ce4   0x00028ce4   0x0000007c   Code   RO         5922    i.disk_read         diskio_blkdev.o
    0x00028d60   0x00028d60   0x00000020   Code   RO         5923    i.disk_status       diskio_blkdev.o
    0x00028d80   0x00028d80   0x00000088   Code   RO         5925    i.disk_write        diskio_blkdev.o
    0x00028e08   0x00028e08   0x0000000c   Code   RO         5926    i.diskio_blockdev_register  diskio_blkdev.o
    0x00028e14   0x00028e14   0x00000014   Code   RO         5146    i.dropped_sat16_get  nrf_log_frontend.o
    0x00028e28   0x00028e28   0x00000014   Code   RO         3813    i.drv_rtc_compare_disable  drv_rtc.o
    0x00028e3c   0x00028e3c   0x0000000e   Code   RO         3816    i.drv_rtc_compare_pending  drv_rtc.o
    0x00028e4a   0x00028e4a   0x00000050   Code   RO         3817    i.drv_rtc_compare_set  drv_rtc.o
    0x00028e9a   0x00028e9a   0x00000008   Code   RO         3818    i.drv_rtc_counter_get  drv_rtc.o
    0x00028ea2   0x00028ea2   0x00000002   PAD
    0x00028ea4   0x00028ea4   0x000000d8   Code   RO         3819    i.drv_rtc_init      drv_rtc.o
    0x00028f7c   0x00028f7c   0x0000001e   Code   RO         3820    i.drv_rtc_irq_trigger  drv_rtc.o
    0x00028f9a   0x00028f9a   0x00000008   Code   RO         3822    i.drv_rtc_overflow_enable  drv_rtc.o
    0x00028fa2   0x00028fa2   0x00000008   Code   RO         3823    i.drv_rtc_overflow_pending  drv_rtc.o
    0x00028faa   0x00028faa   0x00000008   Code   RO         3824    i.drv_rtc_start     drv_rtc.o
    0x00028fb2   0x00028fb2   0x00000008   Code   RO         3825    i.drv_rtc_stop      drv_rtc.o
    0x00028fba   0x00028fba   0x000000de   Code   RO         3830    i.drv_rtc_windowed_compare_set  drv_rtc.o
    0x00029098   0x00029098   0x00000012   Code   RO         3831    i.evt_enable        drv_rtc.o
    0x000290aa   0x000290aa   0x00000014   Code   RO         3832    i.evt_pending       drv_rtc.o
    0x000290be   0x000290be   0x0000001e   Code   RO         6014    i.f_close           ff.o
    0x000290dc   0x000290dc   0x0000004c   Code   RO         6021    i.f_mount           ff.o
    0x00029128   0x00029128   0x000001b4   Code   RO         6022    i.f_open            ff.o
    0x000292dc   0x000292dc   0x00000062   Code   RO         6023    i.f_opendir         ff.o
    0x0002933e   0x0002933e   0x00000002   PAD
    0x00029340   0x00029340   0x00000090   Code   RO         6031    i.f_sync            ff.o
    0x000293d0   0x000293d0   0x0000017e   Code   RO         6034    i.f_write           ff.o
    0x0002954e   0x0002954e   0x00000014   Code   RO         3393    i.fifo_get          app_fifo.o
    0x00029562   0x00029562   0x00000012   Code   RO         3394    i.fifo_put          app_fifo.o
    0x00029574   0x00029574   0x0000024c   Code   RO         6035    i.find_volume       ff.o
    0x000297c0   0x000297c0   0x0000000a   Code   RO         1284    i.flag_toggle       ble_conn_state.o
    0x000297ca   0x000297ca   0x00000028   Code   RO         1075    i.flags_set         ble_advertising.o
    0x000297f2   0x000297f2   0x00000074   Code   RO         6036    i.follow_path       ff.o
    0x00029866   0x00029866   0x000000be   Code   RO         6037    i.get_fat           ff.o
    0x00029924   0x00029924   0x0000003c   Code   RO         6039    i.get_ldnumber      ff.o
    0x00029960   0x00029960   0x00000034   Code   RO         3520    i.get_now           app_timer2.o
    0x00029994   0x00029994   0x00000014   Code   RO         1187    i.instance_get      ble_conn_params.o
    0x000299a8   0x000299a8   0x000000a6   Code   RO         4375    i.int_print         nrf_fprintf_format.o
    0x00029a4e   0x00029a4e   0x00000002   PAD
    0x00029a50   0x00029a50   0x00000088   Code   RO         2827    i.interrupts_enable  nrfx_uarte.o
    0x00029ad8   0x00029ad8   0x00000034   Code   RO         5147    i.invalid_packets_omit  nrf_log_frontend.o
    0x00029b0c   0x00029b0c   0x00000044   Code   RO         1188    i.is_conn_params_ok  ble_conn_params.o
    0x00029b50   0x00029b50   0x00000026   Code   RO         6040    i.ld_clust          ff.o
    0x00029b76   0x00029b76   0x00000016   Code   RO         6041    i.ld_dword          ff.o
    0x00029b8c   0x00029b8c   0x0000000a   Code   RO         6042    i.ld_word           ff.o
    0x00029b96   0x00029b96   0x00000002   PAD
    0x00029b98   0x00029b98   0x00000030   Code   RO          674    i.leds_off          bsp.o
    0x00029bc8   0x00029bc8   0x00000018   Code   RO         1583    i.link_init         nrf_ble_gatt.o
    0x00029be0   0x00029be0   0x000000a4   Code   RO         5148    i.log_skip          nrf_log_frontend.o
    0x00029c84   0x00029c84   0x00000160   Code   RO           11    i.main              main.o
    0x00029de4   0x00029de4   0x00000064   Code   RO          955    i.manuf_specific_data_encode  ble_advdata.o
    0x00029e48   0x00029e48   0x00000012   Code   RO         6043    i.mem_cpy           ff.o
    0x00029e5a   0x00029e5a   0x00000002   PAD
    0x00029e5c   0x00029e5c   0x0000000e   Code   RO         6044    i.mem_set           ff.o
    0x00029e6a   0x00029e6a   0x0000007e   Code   RO         4414    i.memobj_op         nrf_memobj.o
    0x00029ee8   0x00029ee8   0x00000030   Code   RO         5149    i.module_idx_get    nrf_log_frontend.o
    0x00029f18   0x00029f18   0x00000032   Code   RO         6045    i.move_window       ff.o
    0x00029f4a   0x00029f4a   0x000000a6   Code   RO          956    i.name_encode       ble_advdata.o
    0x00029ff0   0x00029ff0   0x00000026   Code   RO         4030    i.nrf_atfifo_init   nrf_atfifo.o
    0x0002a016   0x0002a016   0x00000016   Code   RO         4031    i.nrf_atfifo_item_alloc  nrf_atfifo.o
    0x0002a02c   0x0002a02c   0x00000016   Code   RO         4032    i.nrf_atfifo_item_free  nrf_atfifo.o
    0x0002a042   0x0002a042   0x00000016   Code   RO         4033    i.nrf_atfifo_item_get  nrf_atfifo.o
    0x0002a058   0x0002a058   0x00000016   Code   RO         4034    i.nrf_atfifo_item_put  nrf_atfifo.o
    0x0002a06e   0x0002a06e   0x00000016   Code   RO         4096    i.nrf_atflags_clear  nrf_atflags.o
    0x0002a084   0x0002a084   0x00000016   Code   RO         4101    i.nrf_atflags_get   nrf_atflags.o
    0x0002a09a   0x0002a09a   0x00000014   Code   RO         4103    i.nrf_atflags_set   nrf_atflags.o
    0x0002a0ae   0x0002a0ae   0x00000006   Code   RO         4164    i.nrf_atomic_flag_clear_fetch  nrf_atomic.o
    0x0002a0b4   0x0002a0b4   0x00000006   Code   RO         4165    i.nrf_atomic_flag_set  nrf_atomic.o
    0x0002a0ba   0x0002a0ba   0x0000000c   Code   RO         4167    i.nrf_atomic_u32_add  nrf_atomic.o
    0x0002a0c6   0x0002a0c6   0x0000000c   Code   RO         4168    i.nrf_atomic_u32_and  nrf_atomic.o
    0x0002a0d2   0x0002a0d2   0x0000000a   Code   RO         4171    i.nrf_atomic_u32_fetch_and  nrf_atomic.o
    0x0002a0dc   0x0002a0dc   0x0000000a   Code   RO         4173    i.nrf_atomic_u32_fetch_store  nrf_atomic.o
    0x0002a0e6   0x0002a0e6   0x0000000c   Code   RO         4177    i.nrf_atomic_u32_or  nrf_atomic.o
    0x0002a0f2   0x0002a0f2   0x0000000c   Code   RO         4179    i.nrf_atomic_u32_sub  nrf_atomic.o
    0x0002a0fe   0x0002a0fe   0x00000044   Code   RO         4298    i.nrf_balloc_alloc  nrf_balloc.o
    0x0002a142   0x0002a142   0x00000030   Code   RO         4299    i.nrf_balloc_free   nrf_balloc.o
    0x0002a172   0x0002a172   0x00000030   Code   RO         4300    i.nrf_balloc_init   nrf_balloc.o
    0x0002a1a2   0x0002a1a2   0x00000010   Code   RO         2283    i.nrf_bitmask_bit_is_set  nrfx_gpiote.o
    0x0002a1b2   0x0002a1b2   0x00000002   PAD
    0x0002a1b4   0x0002a1b4   0x00000150   Code   RO         1590    i.nrf_ble_gatt_on_ble_evt  nrf_ble_gatt.o
    0x0002a304   0x0002a304   0x00000016   Code   RO         1684    i.nrf_ble_qwr_conn_handle_assign  nrf_ble_qwr.o
    0x0002a31a   0x0002a31a   0x00000024   Code   RO         1685    i.nrf_ble_qwr_init  nrf_ble_qwr.o
    0x0002a33e   0x0002a33e   0x000000b6   Code   RO         1686    i.nrf_ble_qwr_on_ble_evt  nrf_ble_qwr.o
    0x0002a3f4   0x0002a3f4   0x00000006   Code   RO         5927    i.nrf_blk_dev_ioctl  diskio_blkdev.o
    0x0002a3fa   0x0002a3fa   0x0000000e   Code   RO         2141    i.nrf_clock_event_check  nrfx_clock.o
    0x0002a408   0x0002a408   0x00000010   Code   RO         2142    i.nrf_clock_event_clear  nrfx_clock.o
    0x0002a418   0x0002a418   0x00000040   Code   RO         1797    i.nrf_drv_clock_init  nrf_drv_clock.o
    0x0002a458   0x0002a458   0x00000034   Code   RO         1801    i.nrf_drv_clock_lfclk_release  nrf_drv_clock.o
    0x0002a48c   0x0002a48c   0x00000070   Code   RO         2986    i.nrf_drv_spi_init  nrf_drv_spi.o
    0x0002a4fc   0x0002a4fc   0x00000016   Code   RO         4799    i.nrf_drv_spi_transfer  app_sdcard.o
    0x0002a512   0x0002a512   0x00000002   PAD
    0x0002a514   0x0002a514   0x00000068   Code   RO         1949    i.nrf_drv_uart_init  nrf_drv_uart.o
    0x0002a57c   0x0002a57c   0x00000020   Code   RO         3658    i.nrf_drv_uart_tx   app_uart_fifo.o
    0x0002a59c   0x0002a59c   0x0000001a   Code   RO         4335    i.nrf_fprintf       nrf_fprintf.o
    0x0002a5b6   0x0002a5b6   0x00000018   Code   RO         4336    i.nrf_fprintf_buffer_flush  nrf_fprintf.o
    0x0002a5ce   0x0002a5ce   0x000001da   Code   RO         4376    i.nrf_fprintf_fmt   nrf_fprintf_format.o
    0x0002a7a8   0x0002a7a8   0x00000024   Code   RO           12    i.nrf_gpio_cfg      main.o
    0x0002a7cc   0x0002a7cc   0x00000024   Code   RO         2639    i.nrf_gpio_cfg      nrfx_uart.o
    0x0002a7f0   0x0002a7f0   0x00000024   Code   RO         2828    i.nrf_gpio_cfg      nrfx_uarte.o
    0x0002a814   0x0002a814   0x00000024   Code   RO         3052    i.nrf_gpio_cfg      nrfx_spim.o
    0x0002a838   0x0002a838   0x00000024   Code   RO         4800    i.nrf_gpio_cfg      app_sdcard.o
    0x0002a85c   0x0002a85c   0x00000012   Code   RO         2640    i.nrf_gpio_cfg_default  nrfx_uart.o
    0x0002a86e   0x0002a86e   0x00000012   Code   RO         2829    i.nrf_gpio_cfg_default  nrfx_uarte.o
    0x0002a880   0x0002a880   0x00000012   Code   RO         2641    i.nrf_gpio_cfg_input  nrfx_uart.o
    0x0002a892   0x0002a892   0x00000012   Code   RO         2830    i.nrf_gpio_cfg_input  nrfx_uarte.o
    0x0002a8a4   0x0002a8a4   0x00000014   Code   RO           13    i.nrf_gpio_cfg_output  main.o
    0x0002a8b8   0x0002a8b8   0x00000014   Code   RO         2642    i.nrf_gpio_cfg_output  nrfx_uart.o
    0x0002a8cc   0x0002a8cc   0x00000014   Code   RO         2831    i.nrf_gpio_cfg_output  nrfx_uarte.o
    0x0002a8e0   0x0002a8e0   0x00000014   Code   RO         3053    i.nrf_gpio_cfg_output  nrfx_spim.o
    0x0002a8f4   0x0002a8f4   0x00000022   Code   RO         2286    i.nrf_gpio_cfg_sense_set  nrfx_gpiote.o
    0x0002a916   0x0002a916   0x00000002   PAD
    0x0002a918   0x0002a918   0x0000002c   Code   RO         2287    i.nrf_gpio_latches_read_and_clear  nrfx_gpiote.o
    0x0002a944   0x0002a944   0x0000000e   Code   RO         3054    i.nrf_gpio_pin_clear  nrfx_spim.o
    0x0002a952   0x0002a952   0x0000000e   Code   RO         3055    i.nrf_gpio_pin_set  nrfx_spim.o
    0x0002a960   0x0002a960   0x0000000e   Code   RO         4801    i.nrf_gpio_pin_set  app_sdcard.o
    0x0002a96e   0x0002a96e   0x0000001c   Code   RO           14    i.nrf_gpio_pin_toggle  main.o
    0x0002a98a   0x0002a98a   0x00000016   Code   RO          475    i.nrf_gpio_pin_write  boards.o
    0x0002a9a0   0x0002a9a0   0x00000014   Code   RO         2289    i.nrf_gpiote_event_clear  nrfx_gpiote.o
    0x0002a9b4   0x0002a9b4   0x00000010   Code   RO         2290    i.nrf_gpiote_event_is_set  nrfx_gpiote.o
    0x0002a9c4   0x0002a9c4   0x0000005c   Code   RO         5150    i.nrf_log_backend_add  nrf_log_frontend.o
    0x0002aa20   0x0002aa20   0x00000002   Code   RO         4997    i.nrf_log_backend_rtt_flush  nrf_log_backend_rtt.o
    0x0002aa22   0x0002aa22   0x00000004   Code   RO         4998    i.nrf_log_backend_rtt_init  nrf_log_backend_rtt.o
    0x0002aa26   0x0002aa26   0x00000002   Code   RO         4999    i.nrf_log_backend_rtt_panic_set  nrf_log_backend_rtt.o
    0x0002aa28   0x0002aa28   0x00000018   Code   RO         5000    i.nrf_log_backend_rtt_put  nrf_log_backend_rtt.o
    0x0002aa40   0x0002aa40   0x000000c8   Code   RO         5066    i.nrf_log_backend_serial_put  nrf_log_backend_serial.o
    0x0002ab08   0x0002ab08   0x00000002   Code   RO         5383    i.nrf_log_backend_uart_flush  nrf_log_backend_uart.o
    0x0002ab0a   0x0002ab0a   0x00000006   Code   RO         5384    i.nrf_log_backend_uart_init  nrf_log_backend_uart.o
    0x0002ab10   0x0002ab10   0x0000002c   Code   RO         5385    i.nrf_log_backend_uart_panic_set  nrf_log_backend_uart.o
    0x0002ab3c   0x0002ab3c   0x00000018   Code   RO         5386    i.nrf_log_backend_uart_put  nrf_log_backend_uart.o
    0x0002ab54   0x0002ab54   0x00000030   Code   RO         5152    i.nrf_log_color_id_get  nrf_log_frontend.o
    0x0002ab84   0x0002ab84   0x00000034   Code   RO         5100    i.nrf_log_default_backends_init  nrf_log_default_backends.o
    0x0002abb8   0x0002abb8   0x00000238   Code   RO         5153    i.nrf_log_frontend_dequeue  nrf_log_frontend.o
    0x0002adf0   0x0002adf0   0x00000008   Code   RO         5155    i.nrf_log_frontend_std_0  nrf_log_frontend.o
    0x0002adf8   0x0002adf8   0x0000000e   Code   RO         5156    i.nrf_log_frontend_std_1  nrf_log_frontend.o
    0x0002ae06   0x0002ae06   0x00000010   Code   RO         5157    i.nrf_log_frontend_std_2  nrf_log_frontend.o
    0x0002ae16   0x0002ae16   0x00000002   PAD
    0x0002ae18   0x0002ae18   0x000000b0   Code   RO         5331    i.nrf_log_hexdump_entry_process  nrf_log_str_formatter.o
    0x0002aec8   0x0002aec8   0x00000028   Code   RO         5162    i.nrf_log_init      nrf_log_frontend.o
    0x0002aef0   0x0002aef0   0x00000014   Code   RO         5163    i.nrf_log_module_cnt_get  nrf_log_frontend.o
    0x0002af04   0x0002af04   0x0000001c   Code   RO         5166    i.nrf_log_module_name_get  nrf_log_frontend.o
    0x0002af20   0x0002af20   0x00000028   Code   RO         5167    i.nrf_log_panic     nrf_log_frontend.o
    0x0002af48   0x0002af48   0x000000b6   Code   RO         5332    i.nrf_log_std_entry_process  nrf_log_str_formatter.o
    0x0002affe   0x0002affe   0x00000060   Code   RO         4415    i.nrf_memobj_alloc  nrf_memobj.o
    0x0002b05e   0x0002b05e   0x00000032   Code   RO         4416    i.nrf_memobj_free   nrf_memobj.o
    0x0002b090   0x0002b090   0x00000008   Code   RO         4417    i.nrf_memobj_get    nrf_memobj.o
    0x0002b098   0x0002b098   0x00000004   Code   RO         4418    i.nrf_memobj_pool_init  nrf_memobj.o
    0x0002b09c   0x0002b09c   0x0000001e   Code   RO         4419    i.nrf_memobj_put    nrf_memobj.o
    0x0002b0ba   0x0002b0ba   0x00000010   Code   RO         4420    i.nrf_memobj_read   nrf_memobj.o
    0x0002b0ca   0x0002b0ca   0x00000010   Code   RO         4421    i.nrf_memobj_write  nrf_memobj.o
    0x0002b0da   0x0002b0da   0x00000004   Code   RO           15    i.nrf_qwr_error_handler  main.o
    0x0002b0de   0x0002b0de   0x0000001c   Code   RO         4573    i.nrf_ringbuf_init  nrf_ringbuf.o
    0x0002b0fa   0x0002b0fa   0x0000000c   Code   RO         3833    i.nrf_rtc_event_clear  drv_rtc.o
    0x0002b106   0x0002b106   0x00000002   PAD
    0x0002b108   0x0002b108   0x00000014   Code   RO         5829    i.nrf_sdh_ble_app_ram_start_get  nrf_sdh_ble.o
    0x0002b11c   0x0002b11c   0x00000130   Code   RO         5830    i.nrf_sdh_ble_default_cfg_set  nrf_sdh_ble.o
    0x0002b24c   0x0002b24c   0x00000130   Code   RO         5831    i.nrf_sdh_ble_enable  nrf_sdh_ble.o
    0x0002b37c   0x0002b37c   0x00000060   Code   RO         5832    i.nrf_sdh_ble_evts_poll  nrf_sdh_ble.o
    0x0002b3dc   0x0002b3dc   0x00000074   Code   RO         5711    i.nrf_sdh_enable_request  nrf_sdh.o
    0x0002b450   0x0002b450   0x00000024   Code   RO         5712    i.nrf_sdh_evts_poll  nrf_sdh.o
    0x0002b474   0x0002b474   0x0000000c   Code   RO         5713    i.nrf_sdh_is_enabled  nrf_sdh.o
    0x0002b480   0x0002b480   0x0000003c   Code   RO         5883    i.nrf_sdh_soc_evts_poll  nrf_sdh_soc.o
    0x0002b4bc   0x0002b4bc   0x0000000a   Code   RO         4631    i.nrf_section_iter_init  nrf_section_iter.o
    0x0002b4c6   0x0002b4c6   0x00000024   Code   RO         4632    i.nrf_section_iter_item_set  nrf_section_iter.o
    0x0002b4ea   0x0002b4ea   0x00000020   Code   RO         4633    i.nrf_section_iter_next  nrf_section_iter.o
    0x0002b50a   0x0002b50a   0x00000022   Code   RO         4666    i.nrf_sortlist_add  nrf_sortlist.o
    0x0002b52c   0x0002b52c   0x00000006   Code   RO         4668    i.nrf_sortlist_peek  nrf_sortlist.o
    0x0002b532   0x0002b532   0x0000000e   Code   RO         4669    i.nrf_sortlist_pop  nrf_sortlist.o
    0x0002b540   0x0002b540   0x0000001e   Code   RO         4670    i.nrf_sortlist_remove  nrf_sortlist.o
    0x0002b55e   0x0002b55e   0x0000000a   Code   RO         3056    i.nrf_spim_event_check  nrfx_spim.o
    0x0002b568   0x0002b568   0x00000038   Code   RO         4722    i.nrf_strerror_find  nrf_strerror.o
    0x0002b5a0   0x0002b5a0   0x00000014   Code   RO         4723    i.nrf_strerror_get  nrf_strerror.o
    0x0002b5b4   0x0002b5b4   0x0000000a   Code   RO         2643    i.nrf_uart_event_check  nrfx_uart.o
    0x0002b5be   0x0002b5be   0x0000000c   Code   RO         2644    i.nrf_uart_event_clear  nrfx_uart.o
    0x0002b5ca   0x0002b5ca   0x0000000c   Code   RO         2645    i.nrf_uart_int_enable_check  nrfx_uart.o
    0x0002b5d6   0x0002b5d6   0x0000000a   Code   RO         2832    i.nrf_uarte_event_check  nrfx_uarte.o
    0x0002b5e0   0x0002b5e0   0x0000000c   Code   RO         2833    i.nrf_uarte_event_clear  nrfx_uarte.o
    0x0002b5ec   0x0002b5ec   0x00000010   Code   RO         1804    i.nrf_wdt_started   nrf_drv_clock.o
    0x0002b5fc   0x0002b5fc   0x0000002c   Code   RO         2147    i.nrfx_clock_enable  nrfx_clock.o
    0x0002b628   0x0002b628   0x00000020   Code   RO         2150    i.nrfx_clock_init   nrfx_clock.o
    0x0002b648   0x0002b648   0x00000030   Code   RO         2153    i.nrfx_clock_lfclk_stop  nrfx_clock.o
    0x0002b678   0x0002b678   0x00000010   Code   RO         3834    i.nrfx_coredep_delay_us  drv_rtc.o
    0x0002b688   0x0002b688   0x00000010   Code   RO         2834    i.nrfx_is_in_ram    nrfx_uarte.o
    0x0002b698   0x0002b698   0x00000010   Code   RO         3057    i.nrfx_is_in_ram    nrfx_spim.o
    0x0002b6a8   0x0002b6a8   0x0000003a   Code   RO         2585    i.nrfx_prs_acquire  nrfx_prs.o
    0x0002b6e2   0x0002b6e2   0x00000012   Code   RO         2586    i.nrfx_prs_release  nrfx_prs.o
    0x0002b6f4   0x0002b6f4   0x0000016c   Code   RO         3060    i.nrfx_spim_init    nrfx_spim.o
    0x0002b860   0x0002b860   0x00000094   Code   RO         3062    i.nrfx_spim_uninit  nrfx_spim.o
    0x0002b8f4   0x0002b8f4   0x00000064   Code   RO         3063    i.nrfx_spim_xfer    nrfx_spim.o
    0x0002b958   0x0002b958   0x00000010   Code   RO         2646    i.nrfx_uart_0_irq_handler  nrfx_uart.o
    0x0002b968   0x0002b968   0x000000d4   Code   RO         2648    i.nrfx_uart_init    nrfx_uart.o
    0x0002ba3c   0x0002ba3c   0x000000a8   Code   RO         2654    i.nrfx_uart_tx      nrfx_uart.o
    0x0002bae4   0x0002bae4   0x00000020   Code   RO         2656    i.nrfx_uart_tx_in_progress  nrfx_uart.o
    0x0002bb04   0x0002bb04   0x000000c0   Code   RO         2657    i.nrfx_uart_uninit  nrfx_uart.o
    0x0002bbc4   0x0002bbc4   0x00000010   Code   RO         2835    i.nrfx_uarte_0_irq_handler  nrfx_uarte.o
    0x0002bbd4   0x0002bbd4   0x0000006c   Code   RO         2837    i.nrfx_uarte_init   nrfx_uarte.o
    0x0002bc40   0x0002bc40   0x000000ac   Code   RO         2841    i.nrfx_uarte_tx     nrfx_uarte.o
    0x0002bcec   0x0002bcec   0x0000001c   Code   RO         2843    i.nrfx_uarte_tx_in_progress  nrfx_uarte.o
    0x0002bd08   0x0002bd08   0x00000108   Code   RO         2844    i.nrfx_uarte_uninit  nrfx_uarte.o
    0x0002be10   0x0002be10   0x00000098   Code   RO           16    i.nus_data_handler  main.o
    0x0002bea8   0x0002bea8   0x00000018   Code   RO         6318    i.nvmc_config       system_nrf52.o
    0x0002bec0   0x0002bec0   0x00000036   Code   RO           17    i.on_adv_evt        main.o
    0x0002bef6   0x0002bef6   0x0000006a   Code   RO         1731    i.on_connect        ble_nus.o
    0x0002bf60   0x0002bf60   0x000000a8   Code   RO         1591    i.on_connected_evt  nrf_ble_gatt.o
    0x0002c008   0x0002c008   0x000000ac   Code   RO         1592    i.on_exchange_mtu_request_evt  nrf_ble_gatt.o
    0x0002c0b4   0x0002c0b4   0x00000084   Code   RO         1732    i.on_write          ble_nus.o
    0x0002c138   0x0002c138   0x00000012   Code   RO         1076    i.phy_is_valid      ble_advertising.o
    0x0002c14a   0x0002c14a   0x00000002   PAD
    0x0002c14c   0x0002c14c   0x000000b4   Code   RO         2323    i.port_event_handle  nrfx_gpiote.o
    0x0002c200   0x0002c200   0x00000010   Code   RO         2324    i.port_handler_polarity_get  nrfx_gpiote.o
    0x0002c210   0x0002c210   0x0000003c   Code   RO         5334    i.postfix_process   nrf_log_str_formatter.o
    0x0002c24c   0x0002c24c   0x00000098   Code   RO         5335    i.prefix_process    nrf_log_str_formatter.o
    0x0002c2e4   0x0002c2e4   0x00000018   Code   RO         2587    i.prs_box_get       nrfx_prs.o
    0x0002c2fc   0x0002c2fc   0x000000ea   Code   RO         6046    i.put_fat           ff.o
    0x0002c3e6   0x0002c3e6   0x00000074   Code   RO         6049    i.remove_chain      ff.o
    0x0002c45a   0x0002c45a   0x00000002   PAD
    0x0002c45c   0x0002c45c   0x0000005c   Code   RO         3521    i.rtc_irq           app_timer2.o
    0x0002c4b8   0x0002c4b8   0x00000064   Code   RO         3522    i.rtc_schedule      app_timer2.o
    0x0002c51c   0x0002c51c   0x00000074   Code   RO         3523    i.rtc_update        app_timer2.o
    0x0002c590   0x0002c590   0x00000032   Code   RO         2658    i.rx_byte           nrfx_uart.o
    0x0002c5c2   0x0002c5c2   0x00000016   Code   RO         2659    i.rx_done_event     nrfx_uart.o
    0x0002c5d8   0x0002c5d8   0x00000016   Code   RO         2845    i.rx_done_event     nrfx_uarte.o
    0x0002c5ee   0x0002c5ee   0x00000002   PAD
    0x0002c5f0   0x0002c5f0   0x00000054   Code   RO           18    i.saadc_init        main.o
    0x0002c644   0x0002c644   0x00000028   Code   RO           19    i.saadc_start       main.o
    0x0002c66c   0x0002c66c   0x00000380   Code   RO           20    i.sd_data_saving    main.o
    0x0002c9ec   0x0002c9ec   0x00000058   Code   RO         1805    i.sd_state_evt_handler  nrf_drv_clock.o
    0x0002ca44   0x0002ca44   0x000000b8   Code   RO         4802    i.sdc_cmd           app_sdcard.o
    0x0002cafc   0x0002cafc   0x0000009c   Code   RO         4939    i.sdc_handler       nrf_block_dev_sdc.o
    0x0002cb98   0x0002cb98   0x0000029c   Code   RO         4803    i.sdc_pt_identification  app_sdcard.o
    0x0002ce34   0x0002ce34   0x00000080   Code   RO         4804    i.sdc_pt_read       app_sdcard.o
    0x0002ceb4   0x0002ceb4   0x00000160   Code   RO         4805    i.sdc_pt_sub_data_read  app_sdcard.o
    0x0002d014   0x0002d014   0x00000208   Code   RO         4806    i.sdc_pt_write      app_sdcard.o
    0x0002d21c   0x0002d21c   0x0000003c   Code   RO         4807    i.sdc_spi_transfer  app_sdcard.o
    0x0002d258   0x0002d258   0x00000030   Code   RO         5718    i.sdh_request_observer_notify  nrf_sdh.o
    0x0002d288   0x0002d288   0x0000002c   Code   RO         5719    i.sdh_state_observer_notify  nrf_sdh.o
    0x0002d2b4   0x0002d2b4   0x00000010   Code   RO         1189    i.send_error_evt    ble_conn_params.o
    0x0002d2c4   0x0002d2c4   0x00000050   Code   RO         5001    i.serial_tx         nrf_log_backend_rtt.o
    0x0002d314   0x0002d314   0x00000040   Code   RO         5387    i.serial_tx         nrf_log_backend_uart.o
    0x0002d354   0x0002d354   0x00000088   Code   RO          957    i.service_data_encode  ble_advdata.o
    0x0002d3dc   0x0002d3dc   0x00000030   Code   RO         1468    i.set_security_req  ble_srv_common.o
    0x0002d40c   0x0002d40c   0x00000018   Code   RO         1806    i.soc_evt_handler   nrf_drv_clock.o
